:020000040800F2
:10000000005000202D8300085F16000861160008CC
:100010006316000865160008671600080000000057
:100020000000000000000000000000006916000849
:100030006B160008000000006D1600086F1600081F
:1000400075830008758300087583000875830008B0
:1000500075830008758300087583000875830008A0
:100060007583000875830008758300087583000890
:100070007583000875830008758300087583000880
:1000800075830008758300087583000879160008D9
:1000900089160008758300087583000875830008B9
:1000A0007583000875830008758300087583000850
:1000B0007583000875830008758300087583000840
:1000C0007583000875830008758300087583000830
:1000D0007583000855610008758300087583000862
:1000E0007583000875830008758300080000000010
:1000F0000000000000000000000000000000000000
:0C01000000000000000000005FF808F1A3
:1001100010F8012B11F8013B012A28BF9A42F7D0B1
:10012000D01A7047034613F8012B002AFBD1181A86
:100130000138704781F0004102E000BF83F00043C6
:1001400030B54FEA41044FEA430594EA050F08BF72
:1001500090EA020F1FBF54EA000C55EA020C7FEA36
:10016000645C7FEA655C00F0E2804FEA5454D4EBB3
:100170005555B8BF6D420CDD2C4480EA020281EA7D
:10018000030382EA000083EA010180EA020281EAB5
:100190000303362D88BF30BD11F0004F4FEA013107
:1001A0004FF4801C4CEA113102D0404261EB410116
:1001B00013F0004F4FEA03334CEA133302D052429C
:1001C00063EB430394EA050F00F0A780A4F1010458
:1001D000D5F1200E0DDB02FA0EFC22FA05F2801892
:1001E00041F1000103FA0EF2801843FA05F3594178
:1001F0000EE0A5F120050EF1200E012A03FA0EFCF7
:1002000028BF4CF0020C43FA05F3C01851EBE37120
:1002100001F0004507D54FF0000EDCF1000C7EEB3D
:1002200000006EEB0101B1F5801F1BD3B1F5001F7B
:100230000CD349085FEA30004FEA3C0C04F101049A
:100240004FEA445212F5800F80F09A80BCF1004FC3
:1002500008BF5FEA500C50F1000041EB045141EA45
:10026000050130BD5FEA4C0C404141EB010111F446
:10027000801FA4F10104E9D191F0000F04BF0146F1
:100280000020B1FA81F308BF2033A3F10B03B3F1CF
:1002900020020CDA0C3208DD02F1140CC2F10C025F
:1002A00001FA0CF021FA02F10CE002F11402D8BFBD
:1002B000C2F1200C01FA02F120FA0CFCDCBF41EA89
:1002C0000C019040E41AA2BF01EB0451294330BD58
:1002D0006FEA04041F3C1CDA0C340EDC04F1140435
:1002E000C4F1200220FA04F001FA02F340EA03000C
:1002F00021FA04F345EA030130BDC4F10C04C4F152
:10030000200220FA02F001FA04F340EA0300294631
:1003100030BD21FA04F0294630BD94F0000F83F47B
:10032000801306BF81F480110134013D4EE77FEA5E
:10033000645C18BF7FEA655C29D094EA050F08BFAA
:1003400090EA020F05D054EA000C04BF194610468B
:1003500030BD91EA030F1EBF0021002030BD5FEACF
:10036000545C05D14000494128BF41F0004130BDF7
:1003700014F580043CBF01F5801130BD01F000454B
:1003800045F0FE4141F470014FF0000030BD7FEABE
:10039000645C1ABF194610467FEA655C1CBF0B46B9
:1003A000024650EA013406BF52EA033591EA030FD0
:1003B00041F4002130BD00BF90F0000F04BF0021C8
:1003C000704730B54FF4806404F132044FF00005FB
:1003D0004FF0000150E700BF90F0000F04BF002174
:1003E000704730B54FF4806404F1320410F00045DA
:1003F00048BF40424FF000013EE700BF42004FEAD5
:10040000E2014FEA31014FEA02701FBF12F07F4351
:1004100093F07F4F81F06051704732F07F4208BF08
:10042000704793F07F4F04BF41F40021704730B50F
:100430004FF4607401F0004521F000411CE700BF5B
:1004400050EA010208BF704730B54FF000050AE0DE
:1004500050EA010208BF704730B511F0004502D5DF
:10046000404261EB41014FF4806404F132045FEAE1
:10047000915C3FF4D8AE4FF003025FEADC0C18BF8A
:1004800003325FEADC0C18BF033202EBDC02C2F17C
:10049000200300FA03FC20FA02F001FA03FE40EA0E
:1004A0000E0021FA02F11444BDE600BF70B54FF012
:1004B000FF0C4CF4E06C1CEA11541DBF1CEA1355F0
:1004C00094EA0C0F95EA0C0F00F0DEF82C4481EA58
:1004D000030621EA4C5123EA4C5350EA013518BF78
:1004E00052EA033541F4801143F4801338D0A0FB65
:1004F00002CE4FF00005E1FB02E506F00042E0FB12
:1005000003E54FF00006E1FB03569CF0000F18BF17
:100510004EF0010EA4F1FF04B6F5007F64F54074BF
:1005200004D25FEA4E0E6D4146EB060642EAC62152
:1005300041EA55514FEAC52040EA5E504FEACE2EBF
:10054000B4F1FD0C88BFBCF5E06F1ED8BEF1004FC2
:1005500008BF5FEA500E50F1000041EB045170BD3E
:1005600006F0004646EA010140EA020081EA030182
:10057000B4EB5C04C2BFD4EB0C0541EA045170BD7E
:1005800041F480114FF0000E013C00F3AB8014F1F8
:10059000360FDEBF002001F0004170BDC4F1000441
:1005A000203C35DA0C341BDC04F11404C4F12005C2
:1005B00000FA05F320FA04F001FA05F240EA02001D
:1005C00001F0004221F0004110EBD37021FA04F653
:1005D00042EB06015EEA430E08BF20EAD37070BD0D
:1005E000C4F10C04C4F1200500FA04F320FA05F06C
:1005F00001FA04F240EA020001F0004110EBD3706E
:1006000041F100015EEA430E08BF20EAD37070BDDD
:10061000C4F1200500FA05F24EEA020E20FA04F3B6
:1006200001FA05F243EA020321FA04F001F0004165
:1006300021FA04F220EA020000EBD3705EEA430ED6
:1006400008BF20EAD37070BD94F0000F0FD101F005
:100650000046400041EB010111F4801F08BF013C3E
:10066000F7D041EA060195F0000F18BF704703F07C
:100670000046520043EB030313F4801F08BF013D03
:10068000F7D043EA0603704794EA0C0F0CEA1355BF
:1006900018BF95EA0C0F0CD050EA410618BF52EA79
:1006A0004306D1D181EA030101F000414FF000007F
:1006B00070BD50EA410606BF1046194652EA43068D
:1006C00019D094EA0C0F02D150EA013613D195EA01
:1006D0000C0F05D152EA03361CBF104619460AD149
:1006E00081EA030101F0004141F0FE4141F4700153
:1006F0004FF0000070BD41F0FE4141F4780170BD43
:1007000070B54FF0FF0C4CF4E06C1CEA11541DBFA7
:100710001CEA135594EA0C0F95EA0C0F00F0A7F8A9
:10072000A4EB050481EA030E52EA03354FEA0131D6
:1007300000F088804FEA03334FF0805545EA1313E9
:1007400043EA12634FEA022245EA111545EA1065B1
:100750004FEA00260EF000419D4208BF964244F148
:10076000FD0404F5407402D25B084FEA3202B61A67
:1007700065EB03055B084FEA32024FF480104FF43B
:10078000002CB6EB020E75EB030E22BFB61A7546AF
:1007900040EA0C005B084FEA3202B6EB020E75EB42
:1007A000030E22BFB61A754640EA5C005B084FEAAA
:1007B0003202B6EB020E75EB030E22BFB61A754677
:1007C00040EA9C005B084FEA3202B6EB020E75EB82
:1007D000030E22BFB61A754640EADC0055EA060E43
:1007E00018D04FEA051545EA16754FEA06164FEA86
:1007F000C30343EA52734FEAC2025FEA1C1CC0D132
:1008000011F4801F0BD141EA00014FF000004FF0BE
:10081000004CB6E711F4801F04BF01430020B4F17F
:10082000FD0C88BFBCF5E06F3FF6AFAEB5EB030C37
:1008300004BFB6EB020C5FEA500C50F1000041EB34
:10084000045170BD0EF0004E4EEA113114EB5C0401
:10085000C2BFD4EB0C0541EA045170BD41F48011D4
:100860004FF0000E013C90E645EA060E8DE60CEADC
:10087000135594EA0C0F08BF95EA0C0F3FF43BAFF9
:1008800094EA0C0F0AD150EA01347FF434AF95EAB0
:100890000C0F7FF425AF104619462CE795EA0C0F94
:1008A00006D152EA03353FF4FDAE1046194622E761
:1008B00050EA410618BF52EA43067FF4C5AE50EA3B
:1008C00041047FF40DAF52EA43057FF4EBAE12E72B
:1008D0004FF0FF3C06E000BF4FF0010C02E000BF0C
:1008E0004FF0010C4DF804CD4FEA410C7FEA6C5CEF
:1008F0004FEA430C18BF7FEA6C5C1BD001B050EA92
:10090000410C0CBF52EA430C91EA030F02BF90EA7C
:10091000020F0020704710F1000F91EA030F58BF3B
:10092000994208BF90422CBFD8176FEAE37040F09D
:10093000010070474FEA410C7FEA6C5C02D150EA3B
:10094000013C07D14FEA430C7FEA6C5CD6D152EAF6
:10095000033CD3D05DF8040B704700BF84461046BB
:1009600062468C461946634600E000BF01B5FFF7BA
:10097000B7FF002848BF10F1000F01BD4DF808ED8A
:10098000FFF7F4FF0CBF012000205DF808FB00BF5B
:100990004DF808EDFFF7EAFF34BF012000205DF8B5
:1009A00008FB00BF4DF808EDFFF7E0FF94BF012002
:1009B00000205DF808FB00BF4DF808EDFFF7CEFF03
:1009C00094BF012000205DF808FB00BF4DF808ED42
:1009D000FFF7C4FF34BF012000205DF808FB00BF13
:1009E0004FEA410C7FEA6C5C02D150EA013C0AD12B
:1009F0004FEA430C7FEA6C5C02D152EA033C02D11D
:100A00004FF0000070474FF0010070474FEA41027D
:100A100012F5001215D211D56FF47873B3EB625250
:100A200012D94FEAC12343F0004343EA505311F077
:100A3000004F23FA02F018BF404270474FF0000009
:100A4000704750EA013005D111F0004008BF6FF047
:100A5000004070474FF00000704700BF4A0011D2BD
:100A600012F5001211D20DD56FF47873B3EB625208
:100A70000ED44FEAC12343F0004343EA505323FA14
:100A800002F070474FF00000704750EA013002D189
:100A90004FF0FF3070474FF0000070474FEA4102BF
:100AA000B2F1E04324BFB3F5001CDCF1FE5C0DD9CC
:100AB00001F0004C4FEAC0024CEA5070B2F1004F16
:100AC00040EB830008BF20F00100704711F0804F19
:100AD00021D113F13872BCBF01F00040704741F4DE
:100AE00080114FEA5252C2F11802C2F1200C10FAE2
:100AF0000CF320FA02F018BF40F001004FEAC123C6
:100B00004FEAD32303FA0CFC40EA0C0023FA02F369
:100B10004FEA4303CCE77FEA625307D150EA01333F
:100B20001EBF4FF0FE4040F44000704701F000400F
:100B300040F0FE4040F40000704700BF80F00040ED
:100B400002E000BF81F0004142001FBF5FEA4103A5
:100B500092EA030F7FEA226C7FEA236C6AD04FEAA5
:100B60001262D2EB1363C1BFD218414048404140EA
:100B7000B8BF5B42192B88BF704710F0004F40F49C
:100B8000000020F07F4018BF404211F0004F41F4B8
:100B9000000121F07F4118BF494292EA030F3FD084
:100BA000A2F1010241FA03FC10EB0C00C3F1200397
:100BB00001FA03F100F0004302D5494260EB400026
:100BC000B0F5000F13D3B0F1807F06D340084FEA91
:100BD000310102F10102FE2A51D2B1F1004F40EB86
:100BE000C25008BF20F0010040EA030070474900EE
:100BF00040EB000010F4000FA2F10102EDD1B0FAB9
:100C000080FCACF1080CB2EB0C0200FA0CF0AABFAD
:100C100000EBC25052421843BCBFD040184370474B
:100C200092F0000F81F4000106BF80F40000013251
:100C3000013BB5E74FEA41037FEA226C18BF7FEA28
:100C4000236C21D092EA030F04D092F0000F08BF6A
:100C50000846704790EA010F1CBF0020704712F051
:100C60007F4F04D1400028BF40F00040704712F190
:100C700000723CBF00F50000704700F0004343F0F5
:100C8000FE4040F4000070477FEA226216BF08462B
:100C90007FEA23630146420206BF5FEA412390EAEE
:100CA000010F40F4800070474FF0000304E000BFE4
:100CB00010F0004348BF40425FEA000C08BF704795
:100CC00043F0964301464FF000001CE050EA010259
:100CD00008BF70474FF000030AE000BF50EA01026E
:100CE00008BF704711F0004302D5404261EB41015B
:100CF0005FEA010C02BF84460146002043F0B64380
:100D000008BFA3F18053A3F50003BCFA8CF2083AA4
:100D1000A3EBC25310DB01FA02FC634400FA02FCAD
:100D2000C2F12002BCF1004F20FA02F243EB0200B4
:100D300008BF20F00100704702F1200201FA02FC16
:100D4000C2F1200250EA4C0021FA02F243EB020009
:100D500008BF20EADC7070474FF0FF0C1CEAD0524D
:100D60001EBF1CEAD15392EA0C0F93EA0C0F6FD00E
:100D70001A4480EA010C400218BF5FEA41211ED0EC
:100D80004FF0006343EA501043EA5111A0FB0131D8
:100D90000CF00040B1F5000F3EBF490041EAD371AD
:100DA0005B0040EA010062F17F02FD2A1DD8B3F129
:100DB000004F40EBC25008BF20F00100704790F098
:100DC000000F0CF0004C08BF49024CEA502040EAEA
:100DD00051207F3AC2BFD2F1FF0340EAC2507047B0
:100DE00040F400004FF00003013A5DDC12F1190FEE
:100DF000DCBF00F000407047C2F10002410021FA60
:100E000002F1C2F1200200FA02FC5FEA310040F177
:100E1000000053EA4C0308BF20EADC70704792F0F0
:100E2000000F00F0004C02BF400010F4000F013A28
:100E3000F9D040EA0C0093F0000F01F0004C02BF23
:100E4000490011F4000F013BF9D041EA0C018FE792
:100E50000CEAD15392EA0C0F18BF93EA0C0F0AD098
:100E600030F0004C18BF31F0004CD8D180EA0100BE
:100E700000F00040704790F0000F17BF90F0004F57
:100E8000084691F0000F91F0004F14D092EA0C0F39
:100E900001D142020FD193EA0C0F03D14B0218BFCC
:100EA000084608D180EA010000F0004040F0FE4012
:100EB00040F40000704740F0FE4040F440007047AE
:100EC0004FF0FF0C1CEAD0521EBF1CEAD15392EA2D
:100ED0000C0F93EA0C0F69D0A2EB030280EA010C1D
:100EE00049024FEA402037D04FF0805343EA1111B6
:100EF00043EA10130CF000408B4238BF5B0042F114
:100F00007D024FF4000C8B4224BF5B1A40EA0C00B8
:100F1000B3EB510F24BFA3EB510340EA5C00B3EBEA
:100F2000910F24BFA3EB910340EA9C00B3EBD10FD8
:100F300024BFA3EBD10340EADC001B0118BF5FEA2A
:100F40001C1CE0D1FD2A3FF650AF8B4240EBC25053
:100F500008BF20F0010070470CF0004C4CEA502014
:100F60007F32C2BFD2F1FF0340EAC250704740F463
:100F700000004FF00003013A37E792F0000F00F055
:100F8000004C02BF400010F4000F013AF9D040EAD3
:100F90000C0093F0000F01F0004C02BF490011F467
:100FA000000F013BF9D041EA0C0195E70CEAD1535F
:100FB00092EA0C0F08D142027FF47DAF93EA0C0F46
:100FC0007FF470AF084676E793EA0C0F04D14B022A
:100FD0003FF44CAF08466EE730F0004C18BF31F0DC
:100FE000004CCAD130F000427FF45CAF31F00043D6
:100FF0007FF43CAF5FE700BF4FF0FF3C06E000BF6F
:101000004FF0010C02E000BF4FF0010C4DF804CD91
:101010004FEA40024FEA41037FEA226C18BF7FEAA1
:10102000236C11D001B052EA530C18BF90EA010FA3
:1010300058BFB2EB030088BFC81738BF6FEAE17032
:1010400018BF40F0010070477FEA226C02D15FEACE
:10105000402C05D17FEA236CE4D15FEA412CE1D03A
:101060005DF8040B704700BF844608466146FFE701
:101070000FB5FFF7C9FF002848BF10F1000F0FBDE3
:101080004DF808EDFFF7F4FF0CBF012000205DF8DC
:1010900008FB00BF4DF808EDFFF7EAFF34BF012061
:1010A00000205DF808FB00BF4DF808EDFFF7E0FFFA
:1010B00094BF012000205DF808FB00BF4DF808ED4B
:1010C000FFF7D2FF94BF012000205DF808FB00BFAE
:1010D0004DF808EDFFF7C8FF34BF012000205DF890
:1010E00008FB00BF4FEA40024FEA41037FEA226C4F
:1010F00002D15FEA402C08D17FEA236C02D15FEA7B
:10110000412C02D14FF0000070474FF001007047B2
:101110004FEA4002B2F1FE4F0FD34FF09E03B3EB04
:1011200012620DD94FEA002343F0004310F0004F44
:1011300023FA02F018BF404270474FF0000070479A
:1011400012F1610F01D1420205D110F0004008BF39
:101150006FF0004070474FF0000070470348044BA9
:10116000834202D0034B03B118477047BC030020F1
:10117000BC0300200000000005480649091A891038
:1011800001EBD171491002D0034B03B118477047EE
:10119000BC030020BC0300200000000010B5064C7A
:1011A000237843B9FFF7DAFF044B13B10448AFF3D8
:1011B00000800123237010BDC00300200000000048
:1011C000C0C8000808B5054B1BB105490548AFF379
:1011D0000080BDE80840FFF7CFBF00BF000000005F
:1011E000C4030020C0C8000808B500F2E730034B74
:1011F000A3FB0030800900F0D3FB08BDD34D621083
:1012000010B584B01C7842F21073029392B201922E
:1012100000910123024604FA03F1054802F05EF84A
:1012200010B9002004B010BD6FF00300FAE700BF52
:10123000000D002010B584B01C7842F210730293A8
:1012400092B2019200910123024604FA03F105488B
:1012500002F0F6F810B9002004B010BD6FF00300E2
:10126000FAE700BF000D00202DE9F04188B000240E
:101270000494059406940794244B9A6942F0100252
:101280009A619A6902F010020092009A9A6942F0FB
:1012900020029A619A6902F020020192019A9A69E9
:1012A00042F004029A619A6902F004020292029AE0
:1012B0009A6942F008029A619B6903F0080303935C
:1012C000039BDFF8508022465821404601F0A2F8E7
:1012D0000F4D22461021284601F09CF85823049314
:1012E0000127059706940226079604A9404600F0B8
:1012F000A5FF102304930597069407960DEB0301B1
:10130000284600F09BFF08B0BDE8F08100100240C5
:10131000000C01400008014008B50E480E4B036068
:101320004FF4827343604FF4004383600023C36033
:1013300002220261012242614FF400728261102296
:10134000C2610362436283620A23C36201F034F91B
:1013500008BD00BFF00D00200030014030B58DB059
:1013600000240494069408940A94019402940F4D66
:101370000F4B2B606C60AC604FF6FF73EB602C6121
:10138000AC6103230393012205920823079309927A
:101390000B9303A9284601F019FB0194029401A9BB
:1013A000284601F0C2FB0DB030BD00BFC00C0020CC
:1013B0000008004008B50848084B03604FF4E133CB
:1013C000436000238360C36003610C224261836138
:1013D000C36101F033FC08BD9C0D002000380140C2
:1013E00030B58BB0002408940994019402940394BE
:1013F0000494059406940794134D144B2B6040F20B
:10140000CF236B60AC6042F21073EB602C61AC6177
:10141000284601F09DFA0821284601F0B3FA10236E
:101420000893099408A9284601F07FFB019442F231
:101430000F73029303940594224601A9284601F0F4
:1014400045FB0BB030BD00BF540D00200004004030
:1014500008B50948094B0360094B436000238360CA
:10146000C3604FF48042026143618361C3610362E0
:1014700001F062FE08BD00BF000D002000580040D2
:10148000A086010030B583B00024ADF804408DF88B
:1014900006400094124D134B2B604FF0FF336B60EE
:1014A0004FF48073AB60284602F0F8FA8DF80440E0
:1014B0008DF805408DF80640012201A9284602F06A
:1014C00006FA01228DF800208DF801208DF8022007
:1014D0008DF803406946284602F05AFA03B030BD41
:1014E000DC0D00200028004010B50446012380F8E0
:1014F0004230052380F84030022380F84130042335
:1015000080F8433001460F2005F07CFB034608B10C
:10151000184610BD04F1400005F052FC034B186062
:101520002146012005F0A8FB0346F1E7980D0020B5
:1015300030B595B000240C940F9410940594069443
:101540000794089409940194029403940494052345
:101550000A934FF480330B9301220D920E920225D1
:10156000119512934FF4E01313930AA800F042FA76
:101570000F230593069507944FF48063089309940D
:10158000294605A800F076FC112301934FF48073DF
:101590000293049401A800F049FD15B030BD00008D
:1015A00010B594B000F0D8F9FFF7C2FFFFF75CFE6A
:1015B000FFF7B2FEFFF7D2FEFFF7FCFEFFF710FFCA
:1015C000FFF746FFFFF75EFF02F0CAFA1D4C00224C
:1015D0001021204600F01EFF4FF47A7000F0E0F971
:1015E00001221021204600F015FF174C1749204614
:1015F00004F09FFD204604F03DFD3B238DF80430B0
:1016000001238DF81030124B0593124B0693124BA9
:10161000079301AB039302A805F0A0FA10B10120D3
:1016200006F0BCFE02A8FFF75FFF10B1012006F034
:10163000B5FE06F0E7FC02A806F00EFD322000F031
:10164000AFF9F8E7000C0140641900209C0D002060
:101650003512000801120008E911000870477047B0
:10166000FEE7FEE7FEE7FEE770477047704708B504
:1016700000F084F908BD000008B5024802F08FFFB1
:1016800008BD00BFF816002008B5024802F087FF29
:1016900008BD00BFF816002082B00E4B9A6942F0D8
:1016A00001029A619A6902F001020092009ADA69D5
:1016B00042F08052DA61DB6903F080530193019BB1
:1016C000054A536823F0E06343F00073536002B0AF
:1016D000704700BF001002400000014010B588B004
:1016E000002304930593069307930268164B9A42CE
:1016F00001D008B010BD154CE36943F48003E361E9
:10170000E36903F480030193019BA36943F0080399
:10171000A361A36903F008030293029B4FF44063A3
:101720000493122305930323079304A9084800F0A8
:1017300085FDE36943F48003E361E36903F4800317
:101740000393039BD5E700BF005800400010024000
:10175000000C014002680C4B9A4200D0704700B563
:1017600083B000F0C7FE094BDA6942F00062DA612B
:10177000DB6903F000630193019B054B01221A60B2
:1017800003B05DF804FB00BF0028004000100240D9
:101790003C04424200B587B00023029303930493B4
:1017A00005930268124B9A4202D007B05DF804FB21
:1017B00003F560439A6942F480529A619A6902F48F
:1017C00080520092009A9A6942F004029A619B69E1
:1017D00003F004030193019BA023029302230393CC
:1017E0000323059302A9034800F028FDDDE700BFAD
:1017F00000300140000801400268094B9A4200D0C5
:10180000704782B003F50333DA6942F00202DA610D
:10181000DB6903F002030193019B02B0704700BF34
:101820000004004000B587B00023029303930493A3
:1018300005930268114B9A4202D007B05DF804FB91
:1018400003F50233DA6942F00402DA61DA6902F080
:1018500004020092009A9A6942F008029A619B6918
:1018600003F008030193019BC02302930123049317
:1018700002A9034800F0E2FCDFE700BF00080040D7
:10188000000C014030B587B000230293039304930A
:10189000059302681B4B9A4201D007B030BD03F597
:1018A00058439A6942F480429A619A6902F48042EC
:1018B0000092009A9A6942F004029A619B6903F0CF
:1018C00004030193019B4FF40073029302230393DB
:1018D000032305930C4D02A9284600F0AFFC4FF4FA
:1018E0008063029300240394049402A9284600F024
:1018F000A5FC22462146252000F0A4FD252000F06D
:10190000D5FDCAE7003801400008014010B5044683
:101910000E4B18784FF47A73B3FBF0F30C4A10684F
:10192000B0FBF3F000F0D0FD68B90F2C01D9012015
:101930000AE0002221464FF0FF3000F083FD054B06
:101940001C60002000E0012010BD00BF040000204A
:101950000C0000200800002008B5074A136843F077
:1019600010031360032000F05BFD0020FFF7CEFFA3
:10197000FFF792FE002008BD00200240034A1168D4
:10198000034B1B780B441360704700BF480E0020C8
:1019900004000020014B1868704700BF480E00206B
:1019A00038B50446FFF7F6FF0546B4F1FF3F02D015
:1019B000044B1B781C44FFF7EDFF401BA042FAD3F9
:1019C00038BD00BF0400002082B0084B1B68084AE5
:1019D000A2FB03235B0A00FB03F0019000BF019B05
:1019E0005A1E0192002BF9D102B070470C00002062
:1019F000D34D6210002800F0F18170B582B004462A
:101A0000036813F0010F2CD0AA4B5B6803F00C03A2
:101A1000042B1DD0A74B5B6803F00C03082B12D0DE
:101A20006368B3F5803F41D0002B55D103F180436B
:101A300003F504331A6822F480321A601A6822F41B
:101A400080221A6037E09B4B5B6813F4803FE7D03D
:101A5000984B1B6813F4003F03D06368002B00F021
:101A6000BF81236813F0020F75D0924B5B6813F0AF
:101A70000C0F5FD08F4B5B6803F00C03082B54D026
:101A80002369002B00F089808B4B01221A60FFF73D
:101A900081FF0546874B1B6813F0020F74D1FFF7D7
:101AA00079FF401B0228F5D903209EE1814A136883
:101AB00043F480331360636843B3FFF76BFF05465D
:101AC0007C4B1B6813F4003FCBD1FFF763FF401B37
:101AD0006428F5D9032088E1B3F5A02F09D0754B10
:101AE0001A6822F480321A601A6822F480221A607E
:101AF000E1E703F18043A3F53C331A6842F4802206
:101B00001A601A6842F480321A60D4E7FFF742FF85
:101B10000546684B1B6813F4003FA2D0FFF73AFF5D
:101B2000401B6428F5D903205FE1624B5B6813F426
:101B3000803FA5D15F4B1B6813F0020F03D02369D0
:101B4000012B40F04F815B4A136823F0F803616971
:101B500043EAC1031360236813F0080F32D0A3696E
:101B6000002B5BD0554B01221A60FFF713FF05468F
:101B7000504B5B6A13F0020F21D1FFF70BFF401BA4
:101B80000228F5D9032030E14A4A136823F0F8030C
:101B9000616943EAC1031360DDE7474B00221A6025
:101BA000FFF7F8FE0546434B1B6813F0020FD2D037
:101BB000FFF7F0FE401B0228F5D9032015E10120B4
:101BC000FFF702FF236813F0040F00F09780394BF2
:101BD000DB6913F0805F33D1364BDA6942F0805213
:101BE000DA61DB6903F080530193019B0125344BDB
:101BF0001B6813F4807F25D0E368012B36D0002BBF
:101C00004CD103F1804303F504331A6A22F0010238
:101C10001A621A6A22F004021A622CE0274B002290
:101C20001A60FFF7B7FE0546224B5B6A13F0020FFE
:101C3000C8D0FFF7AFFE401B0228F5D90320D4E03F
:101C40000025D4E71E4A136843F480731360FFF73E
:101C5000A1FE06461A4B1B6813F4807FCCD1FFF718
:101C600099FE801B6428F5D90320BEE0114A136A4F
:101C700043F001031362E36873B3FFF78BFE06467C
:101C80000C4B1B6A13F0020F37D1FFF783FE801B4A
:101C900041F288339842F3D90320A6E0052B11D0F6
:101CA000044B1A6A22F001021A621A6A22F0040234
:101CB0001A62E0E700100240000042428004424203
:101CC000007000404D4B1A6A42F004021A621A6A10
:101CD00042F001021A62CEE7FFF75CFE0646474B70
:101CE0001B6A13F0020F08D0FFF754FE801B41F26D
:101CF00088339842F3D9032077E0E5B9E369002BF4
:101D000072D03E4A526802F00C02082A56D0022BCA
:101D100017D03B4B00221A60FFF73CFE0446374BBE
:101D20001B6813F0007F47D0FFF734FE001B02282A
:101D3000F5D9032059E0314AD36923F08053D361A8
:101D4000DCE72F4B00221A60FFF724FE05462B4BE1
:101D50001B6813F0007F06D0FFF71CFE401B022813
:101D6000F5D9032041E0236AB3F5803F1AD0234917
:101D70004B6823F47413226A606A024313434B6076
:101D80001F4B01221A60FFF705FE04461B4B1B6820
:101D900013F0007F0ED1FFF7FDFD001B0228F5D9DF
:101DA000032022E0154A536823F40033A1680B4353
:101DB0005360DCE7002018E0002016E0012B16D06D
:101DC0000E4B5B6803F48031226A914211D103F417
:101DD0007013626A93420ED1002006E00120704722
:101DE000012002E0012000E0002002B070BD0120CF
:101DF000FBE70120F9E70120F7E700BF00100240F0
:101E00006000424210B487B0164C94E80F000DF108
:101E1000180C0CE90F00238AADF80430124B5B68F4
:101E200003F00C02082A03D0104807B010BC70471A
:101E3000C3F38342624412F8102C13F4803F0CD099
:101E4000094B5B68C3F34043634413F8143C0748F1
:101E500000FB02F0B0FBF3F0E7E7054800FB02F0FF
:101E6000E3E700BFD8C800080010024000127A0063
:101E700000093D00002800F0A08070B50446534BD7
:101E80001B6803F007038B420BD2504A136823F000
:101E900007030B431360136803F007038B4240F002
:101EA0008E80236813F0020F17D013F0040F04D0B4
:101EB000474A536843F4E0635360236813F0080F04
:101EC00004D0434A536843F460535360404A536814
:101ED00023F0F003A068034353600D46236813F01A
:101EE000010F31D06368012B20D0022B25D0384A56
:101EF000126812F0020F64D035494A6822F00302DA
:101F000013434B60FFF746FD0646314B5B6803F019
:101F10000C036268B3EB820F16D0FFF73BFD801B0A
:101F200041F288339842F0D9032045E0284A1268EC
:101F300012F4003FE0D101203EE0254A126812F081
:101F4000007FD9D1012037E0204B1B6803F0070345
:101F5000AB420AD91D4A136823F007032B431360D1
:101F6000136803F00703AB422DD1236813F0040F6D
:101F700006D0174A536823F4E063E1680B435360CB
:101F8000236813F0080F07D0114A536823F46053F5
:101F9000216943EAC1035360FFF734FF0C4B5B68D0
:101FA000C3F303130B4AD35CD8400B4B18600B4BA5
:101FB0001868FFF7ABFC002070BD012070470120BE
:101FC000FAE70120F8E70120F6E700BF0020024011
:101FD0000010024020C900080C000020080000206A
:101FE000014B1868704700BF0C00002008B5FFF7D0
:101FF000F7FF044B5B68C3F30223034AD35CD8406A
:1020000008BD00BF0010024030C9000808B5FFF746
:10201000E7FF044B5B68C3F3C223034AD35CD84099
:1020200008BD00BF0010024030C9000870B582B082
:102030000446036813F0010F34D03E4BDB6913F004
:10204000805F48D13B4BDA6942F08052DA61DB694C
:1020500003F080530193019B0125374B1B6813F458
:10206000807F3AD0334B1B6A13F4407311D06268FF
:1020700002F440729A420CD02E4A136A23F4407044
:102080002E4901260E6000260E60106213F0010F2B
:1020900037D1284A136A23F4407361680B431362F3
:1020A000002D3FD1236813F0020F06D0214A536858
:1020B00023F44043A1680B435360236813F0100FCF
:1020C00035D01C4A536823F48003E1680B43536006
:1020D000002002B070BD0025BFE7174A136843F423
:1020E00080731360FFF756FC0646134B1B6813F40E
:1020F000807FB7D1FFF74EFC801B6428F5D9032001
:10210000E7E7FFF747FC06460A4B1B6A13F0020F8E
:10211000BFD1FFF73FFC801B41F288339842F3D9CF
:102120000320D6E7D36923F08053D361BAE70020B8
:10213000CFE700BF00100240007000404004424260
:1021400030B587B00546384C94E80F000DF1180CF7
:102150000CE90F00238AADF80430022D51D0102D68
:1021600004D0012D2CD0002007B030BD2F4B5A6871
:102170001B6813F0807F4FD0C2F3834306A90B4442
:1021800013F8100C12F4803F16D0284B5B68C3F391
:1021900040430B4413F8142C254BB3FBF2F300FB24
:1021A00003F0224B5B6813F4800FDDD14000214B1C
:1021B000A3FB00304008D7E71F4B03FB00F0F0E71C
:1021C0001A4B1B6A40F202321A40B2F5817F25D0C9
:1021D00003F44073B3F5007F04D0B3F5407F09D01A
:1021E0000020C1E7114A526A12F0020FF5D049F6F9
:1021F0004040B9E70D4B1B6813F4003F11D100209C
:10220000B2E7FFF703FF094B5B68C3F38133013388
:102210005B00B0FBF3F0A7E70020A5E74FF4004018
:10222000A2E74FF224409FE7ECC8000800100240EC
:1022300000127A00ABAAAAAA00093D00F0B482B04D
:1022400000263546A0E0002A58D0012A10D1CE68D9
:102250000EE06A4FBA4251D048D9694FBA424DD0C8
:1022600007F58037BA4249D0A7F58017BA4245D062
:10227000FF2B57D88446FF2B57D8AC00DCF8002042
:102280000F27A74022EA070206FA04F42243CCF8FB
:1022900000204A6812F0805F75D05A4A946944F071
:1022A00001049461926902F001020192019AAC0862
:1022B000A71C554A52F8272005F00307BF004FF02E
:1022C0000F0C0CFA07FC22EA0C0C504A904232D058
:1022D00002F58062904271D002F5806290426FD028
:1022E00002F58062904224D0042225E0A7F58017F1
:1022F000BA4203D007F58037BA42B9D18A687AB1B9
:10230000012A08D044610826B2E7CE680836AFE754
:10231000CE680C36ACE704610826A9E70026A7E7DB
:102320000426A5E700F1040CA5E7A5F10804A40024
:10233000A4E7032200E00022BA4042EA0C02023481
:10234000314F47F824204A6812F4803F3AD0304C8D
:1023500022681A4322604A6812F4003F38D02C4C9D
:1023600062681A4362604A6812F4801F36D0284CB3
:10237000A2681A43A2604A6812F4001F34D0244CA9
:10238000E2681343E36001350B6833FA05F231D09C
:102390000124AC4023409C42F5D14A68122AB7D0B0
:1023A0003FF657AF022AB0D07FF64DAF032AB5D023
:1023B000112A7FF45DAFCE68043659E70122BBE7EE
:1023C0000222B9E7124C226822EA03022260C2E725
:1023D0000F4C626822EA03026260C4E70C4CA268F8
:1023E00022EA0302A260C6E7094CE26822EA03037C
:1023F000E360C8E702B0F0BC704700BF00002110E6
:1024000000003110001002400000014000080140AF
:10241000000401400AB1016170470904016170477D
:10242000074AD36823F4E0631B041B0C000200F48A
:10243000E060184340F0BF6040F40030D060704767
:1024400000ED00E030B4174BDB68C3F30223C3F1A7
:102450000704042C28BF04241D1D062D01D9033BAD
:1024600000E000234FF0FF3505FA04F421EA0401EF
:10247000994005FA03F322EA03031943002809DB14
:102480000901C9B200F1604000F5614080F8001315
:1024900030BC704700F00F000901C9B2024B19545B
:1024A000F6E700BF00ED00E014ED00E0002807DBD8
:1024B00000F01F02400901239340024A42F82030F5
:1024C000704700BF00E100E00138B0F1807F0AD220
:1024D000064B5860064AF02182F8231000209860CD
:1024E00007221A6070470120704700BF10E000E02B
:1024F00000ED00E0014B01221A60704720000E42FF
:10250000F8B505460F4616461C462B689B6837EA09
:1025100003030CBF01230023B34237D0B4F1FF3FC4
:10252000F3D0FFF737FA069BC01AA04201D2002C65
:10253000EBD12A68536823F0E00353606B68B3F56E
:10254000827F0BD0AB6AB3F5005F14D0012385F80E
:102550005130002385F85030032018E0AB68B3F504
:10256000004F02D0B3F5806FECD12A68136823F0D6
:1025700040031360E6E72A68136823F400531360EE
:102580002A68136843F400531360DFE70020F8BDA6
:1025900010B582B0044600920B4600228021FFF75E
:1025A000AFFF034610B9184602B010BD636D43F08B
:1025B000200363650323F6E7002839D010B50446ED
:1025C0000023836290F85130002B2CD0022384F832
:1025D00051302268136823F0400313606368A268D7
:1025E0001343E26813432269134362691343A269E8
:1025F00002F400721343E2691343226A1343A16A8F
:1026000022680B431360638B226803F0040353605A
:102610002268D36923F40063D3610020606501233D
:1026200084F8513010BD80F85030FFF7B3F8CDE793
:10263000012070472DE9F04182B090F85040012C04
:1026400000F0C4801D46174688460446012380F8E2
:102650005030FFF79FF9064694F85130DBB2012B5A
:1026600040F09C80B8F1000F00F0A280002F00F035
:10267000A180032384F8513000236365C4F83080BF
:10268000A786E786A363A387E38763642364A368BD
:10269000B3F5004F1CD023681A6812F0400F03D125
:1026A0001A6842F040021A60E368B3F5006F15D073
:1026B00063680BB1012F49D1226B236812781A731A
:1026C000236B01332363E38E013B9BB2E3863DE042
:1026D0002268136843F480431360DCE763680BB13E
:1026E000012F15D1226B23681288DA60236B023325
:1026F0002363E38E013B9BB2E38609E0FFF74AF9CF
:10270000801BA84202D3B5F1FF3F55D1002D55D013
:10271000E38E9BB2002B2CD023689A6812F0020F34
:10272000ECD0226B1288DA60236B02332363E38ED2
:10273000013B9BB2E386EBE7FFF72CF9801BA84235
:1027400002D3B5F1FF3F3BD1002D3BD0E28E92B2D8
:102750007AB123689A6812F0020FEDD0226B1278DA
:102760001A73236B01332363E28E013A92B2E2863D
:10277000ECE7324629462046FFF70AFF08B120233E
:102780006365A36833B901932368DA6801929B6893
:102790000193019B636DBBB9002000E0022001237F
:1027A00084F85130002384F8503002B0BDE8F08145
:1027B0000120F4E70120F2E70320F0E70320EEE731
:1027C0000320ECE70320EAE70120E8E70220ECE73A
:1027D00070B4036A23F001030362036A46688269E6
:1027E00022F073020C6844EA020523F002028B68AF
:1027F00013430D4CA04209D00B4CA0420DD04660B3
:1028000085614A684263036270BC704723F0080325
:10281000CA68134323F00403EEE726F440764A69BE
:1028200032438E691643EAE7002C014030B4036A54
:1028300023F480730362036A4568C26922F073025D
:102840000C68224323F400738C6843EA04230F4C82
:10285000A04209D00D4CA0420ED04560C2614A682A
:10286000C263036230BC704723F40063CC6843EA60
:10287000042323F48063EDE725F440554C6945EAD1
:1028800004158C6945EA0415E7E700BF002C0140F8
:1028900030B4036A23F480530362036A4468C26954
:1028A00022F4E6420D6842EA052223F400538D68C3
:1028B00043EA0533074DA84206D04460C2614A6826
:1028C0000264036230BC704724F480444D6944EADA
:1028D0008514F2E7002C01407047000003681B4A92
:1028E00090420AD0B0F1804F07D0A2F594329042C6
:1028F00003D002F58062904203D123F070034A684E
:102900001343124A90420AD0B0F1804F07D0A2F58B
:102910009432904203D002F58062904203D123F4B6
:102920004073CA68134323F080034A69134303606A
:102930008B68C3620B688362044B984202D0012308
:10294000436170470B690363F9E700BF002C014046
:10295000B0B110B5044690F83D3063B1022384F85D
:102960003D30214651F8040BFFF7B8FF012384F8EE
:102970003D30002010BD80F83C30FEF73DFFEDE714
:102980000120704700B338B504460D4690F83D303D
:10299000ABB1022384F83D30214651F8040BFFF718
:1029A0009DFF2268136823F00803136022681368F0
:1029B0002B431360012384F83D30002038BD80F89C
:1029C0003C30FFF789FFE4E701207047002849D039
:1029D000F8B505460C4690F83D30002B3DD002235B
:1029E00085F83D302A68936823F4804323F0070379
:1029F0009360294651F8040BFFF770FF29688A6835
:102A00008E690F6A2068104326F4407626F003068C
:102A1000A268A36942EA0323334323F47C4323F0EF
:102A2000FC03E668E26946EA02261E43226A1303B3
:102A3000226943EA0213334327F02207626864697C
:102A400042EA04123A43886029688B612B681A6253
:102A5000012385F83D300020F8BD80F83C30FEF7BA
:102A6000E1FEBCE70120704730B4036A23F0100395
:102A70000362036A4468826922F4E6420D6842EA0E
:102A8000052223F020038D6843EA05130E4DA8426A
:102A900009D00D4DA8420ED0446082614A6882631D
:102AA000036230BC704723F08003CD6843EA05130E
:102AB00023F04003EDE724F440644D6944EA8504C3
:102AC0008D6944EA8504E7E7002C014090F83C302A
:102AD000012B28D010B50446012380F83C30022396
:102AE00080F83D300C2A0BD8DFE802F0070A0A0A0A
:102AF000110A0A0A150A0A0A19000068FFF768FE97
:102B0000012384F83D30002084F83C0010BD0068AB
:102B1000FFF7AAFFF4E70068FFF788FEF0E7006818
:102B2000FFF7B6FEECE70220704790F83C30012B2F
:102B30001CD070B4012680F83C60022380F83D3040
:102B400002685568936825F070050C682C4323F0E3
:102B500080054B682B4354600268936080F83D60A9
:102B6000002380F83C30184670BC70470220704744
:102B700038B504460268136923F44053C1680B4317
:102B8000136183680269134342691A430168CB6881
:102B900023F4B05323F00C031343CB600268536952
:102BA00023F4407381690B4353610268214B9A42BD
:102BB0001FD0FFF71BFA00EB800000EB800063687A
:102BC0009B00B0FBF3F01C4DA5FB003251096422C1
:102BD00002FB110213013233A5FB03235B0903F04F
:102BE000F00202EB011203F00F03216813448B6023
:102BF00038BDFFF70BFA00EB800000EB8000636844
:102C00009B00B0FBF3F00C4DA5FB00325109642290
:102C100002FB110213013233A5FB03235B0903F00E
:102C2000F00202EB011203F00F03216813448B60E2
:102C3000DEE700BF003801401F85EB5158B310B5E7
:102C4000044690F839300BB3242384F839302268D5
:102C5000D36823F40053D3602046FFF789FF22682E
:102C6000136923F4904313612268536923F02A0304
:102C700053612268D36843F40053D3600020E063BB
:102C8000202384F8393084F83A3010BD80F8383089
:102C9000FEF7F8FDD8E70120704700000F4B1A68D7
:102CA00042F001021A6059680D4A0A405A601A68D7
:102CB00022F0847222F480321A601A6822F4802290
:102CC0001A605A6822F4FE025A604FF41F029A609A
:102CD000044B4FF000629A60704700BF0010024042
:102CE0000000FFF800ED00E003685A6912F4806FFD
:102CF00001D1002070476FF480625A6100230363A2
:102D0000202280F83D2080F83E30026C42F0040220
:102D1000026480F83C3001207047F8B506460C4646
:102D200017461D4622E0FEF735FE069BC01AA84254
:102D300000D8DDB900233363202286F83D2086F8D1
:102D40003E30326C42F02002326486F83C30012082
:102D50001AE033689B6924EA03039BB2B3FA83F356
:102D60005B099F420FD1B5F1FF3FDCD1C4F30743AC
:102D7000012BEED133685B6924EA03039BB2B3FAFB
:102D800083F35B09EDE70020F8BDF8B504460D4676
:102D900016461F463CE01A6842F400721A60236827
:102DA0006FF480625A6100232363202284F83D205F
:102DB00084F83E30226C42F00402226484F83C30F5
:102DC000012033E0FEF7E6FDC01BB04200D8FEB99B
:102DD00000232363202284F83D2084F83E30226CB7
:102DE00042F02002226484F83C3001201EE0236877
:102DF0009B6925EA03039BB2003318BF0123A3B1EB
:102E000023685A6912F4806FC5D1B6F1FF3FD9D15A
:102E1000C5F30743012BEAD123685B6925EA030365
:102E20009BB2003318BF0123E9E70020F8BD70B55D
:102E300004460D46164623685B6913F0800F1CD1CB
:102E40002046FFF751FFD0B9B5F1FF3FF3D0FEF7B1
:102E5000A1FD801BA84201D8002DECD100232363E3
:102E6000202284F83D2084F83E30226C42F020027B
:102E7000226484F83C30012000E0002070BD012075
:102E8000FCE700002DE9F04184B004460E461746E9
:102E900098460B9D0268136843F480731360009595
:102EA0000A9B00224FF00111FFF737FF20B10123E9
:102EB000184604B0BDE8F081236806F0FE061E61E6
:102EC0002B460A9A20492046FFF75FFF08B10123ED
:102ED000EEE70023039323685A6903929B690393E7
:102EE000039B2A460A992046FFF7A1FF034630B903
:102EF000B8F1010F0ED12268FFB21761D8E7236C39
:102F0000042B01D00123D3E72268136843F4007334
:102F10001360F7E723683A0A1A612A460A9920469D
:102F2000FFF785FF034618B92268FFB21761BFE7B4
:102F3000236C042B01D00123BAE72268136843F401
:102F400000731360F7E700BF020001002DE9F041B4
:102F500084B004460E46174698460B9D02681368D7
:102F600043F4806313600268136843F48073136052
:102F700000950A9B00224FF00111FFF7CEFE20B111
:102F80000123184604B0BDE8F081F6B2236806F0CC
:102F9000FE021A612B460A9A36492046FFF7F5FED3
:102FA00008B10123EDE70023039323685A690392D4
:102FB0009B690393039B2A460A992046FFF737FF34
:102FC00080B9B8F1010F18D12368FFB21F612A46FA
:102FD0000A992046FFF72BFF68B3236C042B24D0FB
:102FE0000123CEE7236C042B01D00123C9E722681B
:102FF000136843F400731360F7E723683A0A1A6111
:103000002A460A992046FFF712FF18B92368FFB233
:103010001F61DCE7236C042B01D00123B1E7226898
:10302000136843F400731360F7E72268136843F4EE
:1030300000731360D4E72268136843F4807313604D
:1030400000950A9B00224FF001112046FFF765FE14
:1030500008B1012395E7236846F001061E612B465F
:103060000A9A04492046FFF790FE0346002888D0BC
:10307000012386E70200010070B504460D4616469E
:1030800023685B6913F0040F1CD12046FFF72CFE68
:10309000D0B9B5F1FF3FF3D0FEF77CFC801BA8420E
:1030A00001D8002DECD100232363202284F83D2099
:1030B00084F83E30226C42F02002226484F83C30D6
:1030C000012000E0002070BD0120FCE770B505463E
:1030D0000C4616462B685A6912F0400F29D15A69DE
:1030E00012F0100F15D1FEF755FC801BA04201D83D
:1030F000002CEFD100232B63202285F83D2085F89A
:103100003E302A6C42F020022A6485F83C300120CF
:1031100070BD6FF010025A6100232B63202285F8E6
:103120003D2085F83E302A6C2A6485F83C30012029
:10313000EEE70020ECE70000002800F0C180F8B5C1
:10314000044690F83D30002B6CD0242384F83D30A9
:103150002268136823F001031360FEF747FF6268DB
:10316000594B9A4263D8594B98428CBF0023012394
:10317000002B40F0A780564BA3FB00239B0C21683B
:103180004A6822F03F021A434A6025682A6A22F000
:103190003F0266684C498E424FD8013313432B627D
:1031A0002568E96921F44F4121F0FF016368464A2F
:1031B00093424CD801385B00B0FBF3F0013040F68D
:1031C000FC73184278D0C0F30B030B43EB6121680A
:1031D0000B6823F0C003E269206A024313430B60CB
:1031E00021688B6823F4034323F0FF032269E0681E
:1031F000024313438B602168CB6823F0FF036269AD
:10320000A06902431343CB602268136843F00103B3
:10321000136000202064202384F83D30206384F86C
:103220003E00F8BD80F83C30FEF758FA8DE7294B98
:1032300098428CBF002301239AE74FF4967101FB5B
:1032400003F32549A1FB03139B090133A6E7A268F9
:10325000BAB9461E03EB4307B6FBF7F60136C6F3D1
:103260000B06B6FA86F6760946BBC2B9421E03EBD8
:103270004303B2FBF3F20132C2F30B0242F4004308
:10328000A3E7461E03EB830707EB8707B6FBF7F6BA
:103290000136C6F30B06B6FA86F67609E4E7421E57
:1032A00003EB830303EB8303B2FBF3F20132C2F3BC
:1032B0000B0242F4404388E7042386E7012384E7B6
:1032C000012070470120ACE7A08601007F841E002A
:1032D00083DE1B43FF083D00D34D62102DE9F04112
:1032E00082B004460E4617469846FEF753FB94F804
:1032F0003D30DBB2202B04D00223184602B0BDE8DB
:10330000F08105460090192301224B492046FFF722
:1033100004FD002840F0898094F83C30012B00F037
:103320008680012384F83C3023681A6812F0010F6C
:1033300003D11A6842F001021A602268136823F46C
:1033400000631360212384F83D30402384F83E302D
:1033500000232364089B6362BDF824306385638D7A
:103360002385364BE36201950A9B009343463A4618
:1033700031462046FFF786FD00285AD1238D002BC9
:1033800033D02A460A992046FFF751FD10BB626AE6
:10339000236812781A61616A4B1C6362238D013BBA
:1033A0009BB22385628D013A92B262852268506990
:1033B00010F0040FE2D0002BE0D04B781361636A69
:1033C00001336362238D013B2385638D013B9BB2F7
:1033D0006385D3E7236C042B01D001238DE722689A
:1033E000136843F400731360F7E72A460A992046EE
:1033F000FFF742FE034650B1236C042B01D001239A
:103400007BE72268136843F400731360F7E72168D1
:103410000A6842F400720A60202284F83D200022EB
:1034200084F83E2084F83C2067E7022365E7022306
:1034300063E7012361E700BF020010000000FFFF07
:103440002DE9F04186B004460E4617469846FEF731
:10345000A1FA94F83D30DBB2202B04D0022630468E
:1034600006B0BDE8F08105460090192301228C4981
:103470002046FFF752FC002840F0488194F83C3089
:10348000012B00F04581012384F83C3023681A6841
:1034900012F0010F03D11A6842F001021A6022688B
:1034A000136823F400631360222384F83D30402323
:1034B00084F83E30002323640C9B6362BDF83430F3
:1034C0006385638D2385774BE36201950E9B0093A3
:1034D00043463A4631462046FFF738FD0646002867
:1034E00040F01881238D5BB9029323685A690292D8
:1034F0009A690292029A1A6842F400721A607DE098
:10350000012B0FD0022B21D02268136843F4806373
:1035100013600023059323685A6905929B690593FC
:10352000059B6BE02268136823F48063136072B616
:103530000023039323685A6903929A690392039ABA
:103540001A6842F400721A6062B657E02268136883
:1035500043F40063136072B60023049323685A692E
:1035600004929A690492049A1A6822F480621A609A
:1035700062B643E02A460E992046FFF7A7FD0028D1
:1035800040F0CA8023681A69636A1A70636A01335B
:103590006362238D013B2385638D013B9BB2638571
:1035A0002CE000950E9B00223F492046FFF7B5FB1B
:1035B000002840F0B38072B62268136843F40073A9
:1035C000136023681A69636A1A70636A013363625D
:1035D000238D013B2385638D013B9BB2638562B6DE
:1035E00023681A69636A1A70636A01336362238D00
:1035F000013B2385638D013B9BB26385238D002BAB
:103600007BD0032B52D8012BB4D0022BC9D000950C
:103610000E9B002224492046FFF77FFB00287FD124
:103620002268136823F48063136072B623681A69F2
:10363000636A1A70636A01336362238D013B2385D9
:10364000638D013B9BB2638500950E9B002216495A
:103650002046FFF762FB002864D12268136843F418
:103660000073136023681A69636A1A70636A01330E
:103670006362238D013B2385638D013B9BB2638590
:1036800062B623681A69636A1A70636A01336362F7
:10369000238D013B2385638D013B9BB26385ADE7A1
:1036A000020010000000FFFF040001002A460E99EE
:1036B0002046FFF70BFD002836D123681A69636A9C
:1036C0001A70626A531C6362238D013B2385638DEC
:1036D000013B9BB263852368596911F0040F8DD0BB
:1036E0001B695370636A01336362238D013B238539
:1036F000638D013B9BB2638580E7202384F83D30D6
:10370000002384F83E3084F83C30A8E60226A6E682
:103710000226A4E60126A2E60126A0E601269EE6F0
:1037200001269CE601269AE6012698E630B4026856
:103730009469A5B2D369916988B2854205D0D069F0
:1037400080B240EA014030BC704798B240EA044081
:10375000F9E70368186A5B6A9BB243EA0040704766
:10376000030903EB83035A0000F00F001044C0B2BA
:103770007047000010B400F5FA64022922D801EB6A
:103780004103C1EBC3011F4BA3FB013102EB51020B
:10379000224400F2CF7002EB90031B4AA2FB0020F0
:1037A000A3EB501303EBD01304331848A0FB032002
:1037B0001A1A00EB52008008C0EBC000181AC0B201
:1037C00010BC704701EB4103C1EBC3030D49A1FBE2
:1037D000031302EB5303234403EB94030A4AA2FBB3
:1037E0000412A3EB521303EBD21302330748A0FBDE
:1037F00003201A1A00EB52008008C0EBC000181A10
:10380000DDE700BF398EE3381F85EB51254992244F
:1038100038B50446FEF7BEF8054623685A6812F02C
:10382000200F07D1FEF7B6F8401BB0F57A7FF4D928
:10383000032004E05A6842F010025A60002038BDAC
:1038400038B504460268536823F010035360FEF74E
:10385000A1F8054623685B6813F0200F07D1FEF737
:1038600099F8401BB0F57A7FF4D9032000E00020DE
:1038700038BD38B505460C46FFF7CAFF10B1012325
:10388000184638BD2B68220C9A612B68A4B2DC6103
:103890002846FFF7D5FF03460028F1D00123EFE7C4
:1038A00038B505460C46FFF7B3FF10B101231846A3
:1038B00038BD2B68220C1A622B68A4B25C622846C1
:1038C000FFF7BEFF03460028F1D00123EFE770B5F4
:1038D000002857D00446002956D0037C012B55D030
:1038E0000E460123037402234374BAB90D784B7852
:1038F000C3EB03139A004FF4616303FB05258B7838
:103900001D4429462046FFF7B4FF0646C8B10423EC
:103910006374002323740126304670BD0878FFF7D6
:103920001FFF4FF4616505FB00F57078FFF718FF86
:10393000C0EB001083001D44B078FFF711FF054471
:10394000DFE72268536823F0050353602046FFF742
:1039500000FFB0F1FF3F01D0854204D8012363741A
:1039600000232374D8E700F5A83101F5C071204683
:10397000FFF796FF0028F1D004236374002323741B
:103980000126C9E70126C7E70126C5E70226C3E7E6
:1039900000285AD038B50446002958D0037C012BA2
:1039A00057D00D460123037402234374BAB9CB7870
:1039B000C3734B7843738B788373A27B617BE07B0B
:1039C000FFF7D8FE207328702046FFF7AFFE224B8A
:1039D000984211D8012363740020207438BDC87840
:1039E000FFF7BEFEE0736878FFF7BAFE6073A87851
:1039F000FFF7B6FEA073E0E7184DA5FB00352D0CD0
:103A0000174B03FB150529462046FFF732FF28B167
:103A100004236374002323740120DFE72046FFF7AB
:103A200098FEB0F1FF3FD5D08542D3D900F5A8313B
:103A300001F5C0712046FFF733FF0028CAD00423E8
:103A40006374002323740120C8E70120704701201C
:103A5000C4E70220C2E700BF8F5F010007452EC206
:103A600080510100C0B138B504460268536823F0A4
:103A700008035360FDF78EFF054623685B6813F06B
:103A8000080F07D1FDF786FF401BB0F57A7FF4D908
:103A9000032000E0002038BD0120704700285AD0E4
:103AA00010B50446437C53B1022363742046FFF7EC
:103AB000D9FF40B1042363740123184610BD037479
:103AC000FDF748FEF0E72046FFF7A2FE00282DD1C3
:103AD0002268536823F007035360A36823B11F4A89
:103AE000136B23F0010313631C4AD36A23F460733E
:103AF000A1680B43D3626068B0F1FF3F1AD022681F
:103B0000936823F00F0343EA104393602268D3685D
:103B10001B0C1B0480B20343D3602046FFF790FECA
:103B2000034688B1042363740123C6E70423637446
:103B30000123C2E70120FEF703FB08B10138DEE7ED
:103B4000042363740123B8E70022E2730122627345
:103B5000A2736274B1E7012318467047006C0040FD
:103B600008B500220F49104801F068FB70B90F49F1
:103B70000D4801F07AFB60B90D490B4802F09BF942
:103B800050B9094801F078FB48B908BDFDF766FD5A
:103B9000EDE7FDF763FDEFE7FDF760FDF1E7FDF70A
:103BA0005DFDF2E7100000204C0E002070000020A8
:103BB0006000002012230B80004870472C0000207A
:103BC00004230B80004870474000002000239342EC
:103BD00016D230B40BE0373401F8134000015C001A
:103BE000013400250D550133DBB2934206D2040F98
:103BF000092CF0D8303401F81340EFE730BC70479F
:103C00007047000038B50A4B186804331C68043349
:103C10001B68C01800D138BD064D0822A91CFFF74B
:103C2000D5FF042205F112012046FFF7CFFFF2E78E
:103C3000E8F7FF1F4400002008B51A230B80FFF7A8
:103C4000E1FF014808BD00BF4400002008B50A4656
:103C500028B90549054801F085FF034808BD024918
:103C6000024801F07FFFF8E71011002068C9000842
:103C700010B5044C0A462146034801F073FF204664
:103C800010BD00BF1011002054C9000808B50A4635
:103C900028B90549054801F065FF034808BD0249F8
:103CA000024801F05FFFF8E71011002038C9000852
:103CB00008B50A4628B90549054801F053FF0348ED
:103CC00008BD0249024801F04DFFF8E7101100203D
:103CD00044C90008002070470020704710B5054C0B
:103CE0000146204602F0F6F8204602F013F90020C3
:103CF00010BD00BF4C0E002010B5064C0022064936
:103D0000204602F0DFF80549204602F0E3F80020E3
:103D100010BD00BF4C0E0020041500201013002021
:103D2000094BD3F8B832D3F814320BB101207047E5
:103D300010B50A460146044C204602F0C3F820465E
:103D400002F0CEF810BD00BF4C0E0020022807D8AC
:103D5000DFE800F0020604000020704701207047F1
:103D6000022070470268124B9A4200D0704700B59B
:103D700083B003F5DA33DA6942F40002DA61DB6911
:103D800003F400030193019B002211461320FEF768
:103D900059FB1320FEF78AFB002211461420FEF780
:103DA00051FB1420FEF782FB03B05DF804FB00BF5B
:103DB000005C004008B500F50C71D0F8680201F015
:103DC00074FA08BD08B500EB4113D3F83C21D0F8D4
:103DD000680201F098FA08BD08B500EB4113DA6BF0
:103DE000D0F8680201F0D9FA08BD08B5D0F8680229
:103DF00001F07CFB08BD10B504468368022B09D195
:103E00000121D4F8680201F05AFBD4F8680201F0ED
:103E10002EFB10BDFDF722FCF2E7000010B50446B2
:103E2000D0F8680201F04EFBA36923B1024A13697E
:103E300043F00603136110BD00ED00E008B5D0F8B3
:103E4000680201F048FB08BD10B504461D48C0F8E3
:103E50006842C4F8C0021C4B03600823436002237D
:103E6000836000238361C361036200F091F830BB7B
:103E7000182300221146D4F8C00200F0B7FC5823E2
:103E800000228021D4F8C00200F0B0FCC023002240
:103E90008121D4F8C00200F0A9FC4FF488730022FD
:103EA0000121D4F8C00200F0A1FC4FF4807300227D
:103EB0008221D4F8C00200F099FC002010BDFDF76B
:103EC000CDFBD5E7F8160020005C004008B5D0F81F
:103ED000C00200F0D7F8FFF739FF08BD10B51C4647
:103EE00013462246D0F8C00200F0F7F8FFF72EFF85
:103EF00010BD08B5D0F8C00200F027F9FFF726FF83
:103F000008BD08B5D0F8C00200F002FCFFF71EFFA4
:103F100008BD08B5D0F8C00200F031FCFFF716FF6D
:103F200008BDD0F8C03211F0800F06D101F07F013A
:103F300003EB411191F82A01704701F07F0103EB77
:103F4000411191F82A00704708B5D0F8C00200F07E
:103F5000B0F8FFF7FBFE08BD08B5D0F8C00200F0CE
:103F600048F9FFF7F3FE08BD08B5D0F8C00200F02D
:103F70001AF9FFF7EBFE08BD08B5D0F8C00200F053
:103F800031F908BD00487047DC03002070477047D6
:103F9000F0B587B0002873D0044690F82932D3B129
:103FA000032384F82932206800F047FC254655F8A1
:103FB000107B6E460FCD0FC62B683360231D0ECBD2
:103FC000384600F02BFC58B1022384F82932012531
:103FD000284607B0F0BD80F82832FFF7C3FEDFE7C0
:103FE0000021206800F033FC00236068834212D275
:103FF00004EB4312012182F8291082F82830D3867D
:10400000002182F82B109163D1639A1C5201A150B8
:104010000133DBB2E9E70023984213D904EB4311E3
:10402000002281F8292181F8283181F82B21C1F85B
:104030003821C1F83C2103F10A01490162500133E2
:10404000DBB2E9E7254655F8107B6E460FCD0FC66B
:104050002B683360231D0ECB384600F0FAFB054673
:1040600020B1022384F829320125B1E7002384F826
:104070002430012384F82932206800F01CFFA7E7D0
:104080000125A5E790F82832012B10D010B5044681
:10409000012180F82812FFF77AFF206800F009FF5D
:1040A000206800F0C2FB002084F8280210BD022026
:1040B000704790F82832012B0DD010B5044601232B
:1040C00080F8283280F82410006800F0ECFE002010
:1040D00084F8280210BD0220704770B511F0800FDF
:1040E00023D101F007056D0105F5947404440544DE
:1040F000002685F8296101F0070121702261E37033
:10410000627802B1E181022B1AD090F82832012B9B
:1041100019D00546012380F828322146006800F0B6
:10412000AEFB002085F8280270BD01F007056D0187
:1041300005F1280404440544012685F82960DAE7DE
:1041400000232371E1E70220EEE710B511F0800FA4
:104150001CD101F007035B0103F594720244034490
:10416000002483F8294101F00703137090F82832E6
:10417000012B16D00446012380F82832114600682E
:1041800000F031FD002084F8280210BD01F0070383
:104190005B0103F1280202440344012483F829400F
:1041A000E1E70220F1E770B501F007056C0104F5C5
:1041B000947101440444C4F83C2105F10A025201FF
:1041C000861883500023736084F8293184F82851BD
:1041D00025B9006800F08BFE002070BD006800F07B
:1041E00086FEF9E701F007010A3100EB411148684A
:1041F000704770B501F007056C0104F12801014416
:104200000444E263AA1C52018618835000237360A1
:10421000012384F8293084F8285025B9006800F07B
:1042200066FE002070BD006800F061FEF9E7F8B599
:104230000446A8E003889BB223F4E14323F0700313
:104240006FEA43436FEA53439BB203802268B2F89C
:10425000503094F8281003EBC103023302EB430300
:10426000B3F80034C3F309036364E26B1344E363FC
:1042700000212046FFF7B0FD94F82430002B00F019
:104280008280236C002B7ED194F82430226843F086
:104290008003A2F84C30002384F8243073E0B0F897
:1042A000503094F8282103EBC203063300EB43039C
:1042B000B3F80034C3F30903C4F84431B4F82E2131
:1042C00004F50C7100F0A3FF2268138823F070033B
:1042D0001B051B0D43F0800313802046FFF76AFD8A
:1042E00051E03E2A09D8510812F0010F00D00131E7
:1042F000890289B2A3F80C14A1E0510912F01F0F32
:1043000000D101396FEAC1626FEA524292B2A3F85A
:104310000C2494E030F82560B6B216F4004F40F05B
:104320009D8016F0800F2ED0226832F825309BB287
:1043300023F4E14323F070036FEA43436FEA5343EE
:104340009BB222F825302268B2F8503004EB4510B9
:1043500090F8281003EBC103023302EB4303B3F8D8
:104360000024C2F30902AB1C5B01E1184A60C16B77
:104370000A44C263E358002B40F0078190F82810EC
:104380002046FFF729FD2068B0F8443013F4004FB1
:1043900000F00381B0F844309BB213F00F05B9D19F
:1043A00013F0100F3FF446AF03889BB213F4006F75
:1043B0007FF475AF13F4004FE5D0038823F070034A
:1043C0001B051B0D43F0800303802068B0F85030BC
:1043D00094F8282103EBC203063300EB4303B3F840
:1043E0000034C3F30903C4F844318BB1D4F83C1151
:1043F00071B1B4F82E2100F00AFFD4F84421D4F8AA
:104400003C311344C4F83C3100212046FFF7DAFC6C
:104410002368B3F850201344D4F83821002A7FF4DD
:1044200060AFB3F80C2492B222F4F84292B2A3F82F
:104430000C24B3F80C2442F40042A3F80C242268A4
:1044400013889BB223F4804323F0700383F440531A
:1044500043F4004343F08003138094E730F82530A1
:1044600023F070031B051B0D43F0800320F825305B
:1044700004EB451393F83431D3B92068B0F85030C9
:1044800004EB451292F8282103EBC203063300EB3C
:104490004303B3F80074C7F309078FB304EB451166
:1044A0003B46B1F82E21D1F83C1100F0B0FE27E0D8
:1044B000206804EB451393F8282130F8223013F4D8
:1044C000804F43D0B0F8503003EBC203023300EB0F
:1044D0004303B3F80074C7F309076FBB226804EB0A
:1044E000451393F8281132F821309BB223F4E043AE
:1044F00023F0700343F4004343F0C00322F821305B
:1045000005F10A035B01E1184A683A444A6004EB8A
:104510004511D1F83C213A44C1F83C21E3581BB184
:10452000D1F838118F4228D204EB451393F82811A3
:104530002046FFF747FCF4E604EB45113B46B1F893
:104540003021D1F83C1100F062FEC7E7B0F85030DE
:1045500003EBC203063300EB4303B3F80074C7F365
:104560000907002FBAD004EB45113B46B1F83221C0
:10457000D1F83C1100F04BFEB0E704EB451191F887
:1045800028112046FFF70FFECBE604EB451595F802
:1045900028102046FFF72DFEF5E60020F8BD10B5E7
:1045A0000446006800F089FC10F4004F45D12068F3
:1045B00000F083FC10F4806F43D1206800F07DFC94
:1045C00010F4804F08D02268B2F844309BB223F434
:1045D00080439BB2A2F84430206800F06EFC10F4D7
:1045E000005F08D02268B2F844309BB223F4005335
:1045F0009BB2A2F84430206800F05FFC10F4805FAA
:1046000030D1206800F059FC10F4006F49D12068C7
:1046100000F053FC10F4007F6DD1206800F04DFCD9
:1046200010F4807F08D02268B2F844309BB223F4A3
:1046300080739BB2A2F8443010BD2046FFF7F7FD0F
:10464000B5E72268B2F844309BB223F480639BB292
:10465000A2F844302046FFF7CEFB00212046FFF7AA
:1046600028FDAAE72268B2F840309BB223F0040389
:104670009BB2A2F840302268B2F840309BB223F0DF
:1046800008039BB2A2F840302046FFF7D7FB226810
:10469000B2F844309BB223F480539BB2A2F844306A
:1046A000AFE72268B2F8403043F00803A2F8403088
:1046B0002268B2F844309BB223F400639BB2A2F8A4
:1046C00044302268B2F8403043F00403A2F840308E
:1046D000206800F0F2FB10F4805F08D02268B2F886
:1046E00044309BB223F480539BB2A2F8443020465E
:1046F000FFF794FB8BE72268B2F844309BB223F4B7
:1047000000739BB2A2F844302046FFF76EFB84E7AB
:1047100038B501F0070543689D422CD811F0800F91
:104720001AD14B0103F5947101440344002283F82C
:10473000292101238B700D7090F82832012B1CD099
:104740000446012380F82832006800F036FB65B18A
:10475000002084F8280238BD6B0103F128010144D0
:104760000344012283F82920E3E704F50C71206853
:1047700000F0A6FBECE70120EDE70220EBE701F0FB
:104780000F0243689A422DD810B511F0800F1ED148
:1047900001F007035B0103F5947202440344002413
:1047A00083F829410023937001F00703137090F8F8
:1047B0002832012B18D00446012380F828321146F4
:1047C000006800F01FFB002084F8280210BD01F0F3
:1047D00007035B0103F1280202440344012483F828
:1047E0002940DFE7012070470220EFE711F0800F3A
:1047F00009D001F0070149012831014442B90A7387
:10480000CB8000207047490101F594710144F5E720
:1048100001220A730B811B0C4B81F2E784B001A8C3
:1048200080E80E00002004B07047B0F8403043F438
:104830003F43A0F8403000207047B0F8403023F4E8
:104840007C535B045B0CA0F84030002070470020D4
:10485000704784B038B505AC84E80E000123A0F899
:1048600040300024A0F84040A0F84440A0F8504058
:10487000FFF7DBFF2046BDE8384004B0704730B496
:1048800003460C7830F8242092B222F4EC4222F055
:10489000700292B2C87803285AD8DFE800F04D556C
:1048A0000251002048F280052A4323F824200C7886
:1048B00033F8242092B222F4E04222F07002224324
:1048C0002A4323F824200A7B002A40F0B1804A784A
:1048D000002A4ED0B3F850201A440C7802EB041290
:1048E000CC8864086400A2F800440C7833F82420D3
:1048F00012F0400F0CD033F8242092B222F4E042A0
:1049000022F0700242F4004242F0C00223F8242058
:10491000CA78012A1ED0097833F8212092B222F4F5
:10492000E04222F0400282F0200242F4004242F0D3
:10493000800223F8212060E042F400720020B1E7F9
:1049400042F4C0620020ADE742F480620020A9E793
:104950000120A7E7097833F8212092B222F4E0423F
:1049600022F0400242F4004242F0800223F821206B
:1049700043E0B3F850201A440C7802EB0412CC88C0
:1049800064086400A2F80844B3F850201A440C7874
:1049900002EB04120C6994BBB2F80C44A4B224F4E8
:1049A000F844A4B2A2F80C44B2F80C4444F4004415
:1049B000A2F80C440C7833F8242012F4804F0CD069
:1049C00033F8242092B222F4E04222F0700242F442
:1049D000404242F0800223F82420097833F8212055
:1049E00092B222F4804222F0700282F4405242F4E9
:1049F000004242F0800223F8212030BC70473E2C58
:104A000009D8650814F0010F00D00135AD02ADB230
:104A1000A2F80C54CEE7650914F01F0F00D1013D38
:104A20006FEAC5646FEA5444A4B2A2F80C44C1E72B
:104A30000C7833F8242092B222F4E04222F0700283
:104A400042F4014242F0800223F82420B3F85020BF
:104A50001A440C7802EB04120C8964086400A2F872
:104A60000044B3F850201A440C7802EB04124C892D
:104A700064086400A2F808444A78002A4ED10C78F1
:104A800033F8242012F4804F0CD033F8242092B253
:104A900022F4E04222F0700242F4404242F08002EE
:104AA00023F824200C7833F8242012F0400F0CD087
:104AB00033F8242092B222F4E04222F0700242F451
:104AC000004242F0C00223F824200C7833F824205E
:104AD00092B222F4E04222F0700242F4004242F02C
:104AE000C00223F824200D7833F8252092B222F456
:104AF000804222F0700282F4405248F28004224345
:104B000023F82520097833F8212092B222F4E042DC
:104B100022F04002224323F821206EE70C7833F87C
:104B2000242012F4804F0CD033F8242092B222F4C7
:104B3000E04222F0700242F4404242F0800223F848
:104B400024200C7833F8242012F0400F0CD033F8D6
:104B5000242092B222F4E04222F0700242F4004299
:104B600042F0C00223F824200C7833F8242092B2BB
:104B700022F4E04222F0700242F4404242F080020D
:104B800023F82420CA78012A1ED00C7833F8242078
:104B900092B222F4E04222F0400282F0200242F47B
:104BA000004242F0800223F82420097833F82120C3
:104BB00092B222F4804222F0700242F4004242F0AB
:104BC000800223F8212018E70C7833F8242092B2D1
:104BD00022F4E04222F0400242F4004242F080021D
:104BE00023F82420E1E70B7B002B46D14B7813B34D
:104BF0000A7830F8223013F0400F0CD030F8223011
:104C00009BB223F4E04323F0700343F4004343F0EA
:104C1000C00320F822300A7830F822309BB223F407
:104C2000E04323F0400343F4004343F0800320F8C3
:104C30002230002070470A7830F8223013F4804F79
:104C40000CD030F822309BB223F4E04323F0700301
:104C500043F4404343F0800320F822300A7830F8D0
:104C600022309BB223F4804323F0700343F40043CB
:104C700043F0800320F82230DBE710B44B78002BA0
:104C80004ED10A7830F8223013F4804F0CD030F82F
:104C900022309BB223F4E04323F0700343F44043FB
:104CA00043F0800320F822300A7830F8223013F0E5
:104CB000400F0CD030F822309BB223F4E04323F0B5
:104CC000700343F4004343F0C00320F822300A7815
:104CD00030F822309BB223F4E04323F0700343F416
:104CE000004343F0C00320F822300B7830F8232033
:104CF00092B222F4804222F0700248F280042243F1
:104D000020F823200A7830F822309BB223F4E043C5
:104D100023F04003234320F82230002010BC7047CA
:104D20000A7830F8223013F4804F0CD030F822305B
:104D30009BB223F4E04323F0700343F4404343F079
:104D4000800320F822300A7830F8223013F0400F28
:104D50000CD030F822309BB223F4E04323F07003F0
:104D600043F4004343F0C00320F822300A7830F8BF
:104D700022309BB223F4E04323F0700343F440431A
:104D800043F0800320F822300B7830F8232092B2D1
:104D900022F4E04222F0400248F28004224320F84C
:104DA00023200A7830F822309BB223F4804323F08A
:104DB0007003234320F82230AFE74B788BB10A7899
:104DC00030F822309BB223F4E04323F0400383F019
:104DD000100343F4004343F0800320F82230002006
:104DE00070470A7830F822309BB223F4804323F0D6
:104DF000700383F4805343F4004343F0800320F8AE
:104E00002230ECE70B7B002B4BD14B7833B30A7885
:104E100030F8223013F0400F0CD030F822309BB223
:104E200023F4E04323F0700343F4004343F0C00352
:104E300020F82230CB78012B33D00A7830F822309A
:104E40009BB223F4E04323F0400383F0200343F4B8
:104E5000004343F0800320F8223022E00A7830F843
:104E6000223013F4804F0CD030F822309BB223F460
:104E7000E04323F0700343F4404343F0800320F801
:104E800022300A7830F822309BB223F4804323F09A
:104E9000700383F4405343F4004343F0800320F84D
:104EA00022300020704711B98023A0F84C30002038
:104EB00070470020704700207047B0F844007047EA
:104EC0000020704701335B0800EB420202F580626C
:104ED00063B110B40C78487844EA002422F8044BFB
:104EE0000231013B002BF5D110BC7047704770B503
:104EF0004E78012E33D08A690B699A4240F2FC80C9
:104F0000D21A8A610A7B002A40F01381B0F850203F
:104F100002440C7802EB0412002B40F0F180B2F84E
:104F20000C349BB223F4F8439BB2A2F80C34B2F8D1
:104F30000C3443F40043A2F80C340A7830F82230E1
:104F40009BB223F4804323F0700383F4405343F473
:104F5000004343F0800320F82230002070BD8A69AE
:104F60000B699A4222D9D21A8A610C4605460A7BFD
:104F700002B30A7830F8221011F0400F72D0002EE0
:104F800040D1B0F85010014401EB02120BBBB2F853
:104F90000C1489B221F4F84189B2A2F80C14B2F8C9
:104FA0000C1441F40041A2F80C1433E000238B618F
:104FB0001346DAE79EB23346CA884969FFF782FF93
:104FC000B5F850302B44227803EB0213A3F80464A5
:104FD00037E03E2B09D8590813F0010F00D00131FA
:104FE000890289B2A2F80C1414E0590913F01F0FBA
:104FF00000D101396FEAC1616FEA514189B2A2F86B
:105000000C1407E0B0F85010014401EB021299B201
:10501000A2F80C1462899BB261692846FFF752FF1F
:105020006378002B57D1227835F822309BB223F4D5
:10503000E04323F0700343F4004343F0C00325F83A
:105040002230227835F822309BB223F4E04323F05B
:10505000400383F0300343F4004343F0800325F81A
:1050600022307AE76EBBB0F85010014401EB021217
:1050700073B9B2F8041489B221F4F84189B2A2F8E4
:105080000414B2F8041441F40041A2F8041420E01E
:105090003E2B09D8590813F0010F00D001318902C5
:1050A00089B2A2F8041414E0590913F01F0F00D1BB
:1050B00001396FEAC1616FEA514189B2A2F8041463
:1050C00007E0B0F85010014401EB021299B2A2F8C7
:1050D000041422899FE7012BB3D1227835F82230BE
:1050E0009BB223F4E04323F0700343F4404343F0C6
:1050F000800325F82230A4E700238B61134601E7E3
:105100003E2B09D85C0813F0010F00D00134A40233
:10511000A4B2A2F80C4410E75C0913F01F0F00D1F1
:10512000013C6FEAC4646FEA5444A4B2A2F80C4490
:1051300003E7A6B9B0F8502002440C7802EB041241
:1051400033BBB2F80444A4B224F4F844A4B2A2F8E5
:105150000444B2F8044444F40044A2F804444A78F5
:10516000002A47D1B0F8502002440C7802EB041218
:105170003BBBB2F80C349BB223F4F8439BB2A2F8C9
:105180000C34B2F80C3443F40043A2F80C34D4E6E7
:105190003E2B09D85C0813F0010F00D00134A402A3
:1051A000A4B2A2F80444DAE75C0913F01F0F00D19F
:1051B000013C6FEAC4646FEA5444A4B2A2F8044408
:1051C000CDE73E2B09D85C0813F0010F00D0013465
:1051D000A402A4B2A2F80C44AFE65C0913F01F0FBE
:1051E00000D1013C6FEAC4636FEA53439BB2A2F85B
:1051F0000C34A2E6012A7FF4A0AEB0F8502002449D
:105200000C7802EB04129BB2A2F80C3495E630B491
:105210005D0800EB420202F5806245B132F8044BB2
:10522000A4B20C70240A4C700231013DF5E713F072
:10523000010F01D013880B7030BC704798B108B5CE
:105240000346D0F8B40210B10020C3F8B40209B18B
:10525000C3F8B0121846012380F89C320270FEF7A2
:10526000F3FD002008BD0220704719B1C0F8B41248
:10527000002070470220704708B5FEF727FE002087
:1052800008BD08B5D0F8B43233B11B68984708B9E7
:10529000002008BD0220FCE70220FAE708B5D0F89C
:1052A000B4325B689847002008BD38B5044600F565
:1052B0002A75284600F03BF90123C4F89432B4F86B
:1052C000AE32C4F8983294F8A81201F01F03012BF3
:1052D0000FD05AB23AB1022B10D001F08001204613
:1052E000FEF70FFE03E02946204600F0CFFA00202B
:1052F00038BD2946204600F0FDFAF8E72946204649
:1053000000F028FBF3E738B50446A9BB1046D4F8F3
:105310009432032B03D0052B25D0002038E0D4F89D
:105320006031D4F8642193420DD99B1AC4F86031DE
:105330009A4206D99AB20146204600F052FC00205B
:1053400026E092B2F7E7D4F8B4321B691BB194F8A7
:105350009C22032A04D0204600F04BFC002017E0DA
:1053600020469847F7E70025C4F89452294620467E
:10537000FEF7C7FD28460BE00A46D0F8B4329B6919
:105380003BB190F89C12032905D1114698470020A3
:1053900038BD0220FCE70220FAE710B504460029D8
:1053A00054D11046D4F89432022B0CD0042B00D0E8
:1053B0001BB980212046FEF7A4FD94F8A032012BF2
:1053C00040D0002010BD236A626A93421BD8E16975
:1053D000B1FBF2F302FB13132BB98A4203D8D4F8C2
:1053E000983299421DD3D4F8B432DB681BB194F8DB
:1053F0009C22032A23D080212046FEF782FD2046EE
:1054000000F002FCD9E79A1A226292B201462046C5
:1054100000F0D0FB00231A4619462046FEF7A4FDF3
:10542000CBE700221146204600F0C4FB0021C4F85F
:1054300098120B460A462046FEF796FDBDE7204629
:105440009847D8E7002084F8A002BBE70A46D0F8C6
:10545000B4325B693BB190F89C12032905D1114627
:1054600098470020AEE70220ACE70220AAE770B51B
:105470000446402300221146FEF730FD0125C4F802
:1054800058514026C4F864613346002280212046EA
:10549000FEF724FDA561666284F89C520023C4F8DF
:1054A00094326360C4F8A432D4F8B8322BB1D4F883
:1054B000B4325B68002120469847002070BD01741B
:1054C0000020704790F89C3280F89D32042380F8C9
:1054D0009C320020704790F89C32042B01D00020B1
:1054E000704790F89D3280F89C32F8E708B590F844
:1054F0009C32032B01D0002008BDD0F8B432DB6908
:10550000002BF8D09847F6E7002302781AB1013350
:10551000DBB20130F9E71846704708B54B88012B1C
:1055200000D008BDC0F8A43200F063FBF9E70B78A7
:1055300003704B7843708B78CA7803EB0223438067
:105540000B794A7903EB022383808B79CA7903EBC9
:105550000223C380704710B504468021FEF7D1FCBA
:1055600000212046FEF7CDFC10BD30B583B00546C6
:105570000C460023ADF806304A88130A013B062B7F
:1055800000F2A480DFE803F004182CA2A2869300A6
:10559000D0F8B0321B680DF10601007C9847BDF8C9
:1055A00006201AB1E388002B40F09480E388002B9A
:1055B00000F09A8003B030BD037C43B9D0F8B43218
:1055C0009B6A0DF10600984702234370E7E7D0F885
:1055D000B432DB6A0DF10600984702234370DEE720
:1055E000D2B2052A52D8DFE802F003101D2A374450
:1055F000D0F8B0325B6823B10DF10601007C98470A
:10560000CDE72146FFF7A7FFD4E7D0F8B0329B687B
:1056100023B10DF10601007C9847C0E72146FFF752
:105620009AFFC7E7D0F8B032DB6823B10DF106016D
:10563000007C9847B3E72146FFF78DFFBAE7D0F823
:10564000B0321B6923B10DF10601007C9847A6E733
:105650002146FFF780FFADE7D0F8B0325B6923B198
:105660000DF10601007C984799E72146FFF773FF8B
:10567000A0E7D0F8B0329B6923B10DF10601007CA0
:1056800098478CE72146FFF766FF93E72146FFF72F
:1056900062FF8FE7037C33B9D0F8B4325B6B0DF156
:1056A000060098477BE72146FFF755FF82E7037C1A
:1056B00043B9D0F8B4321B6B0DF1060098470723AD
:1056C00043706CE72146FFF746FF73E72146FFF77B
:1056D00042FF6FE79A4228BF1A46ADF806200146FE
:1056E000284600F05AFA61E7284600F082FA61E79E
:1056F00038B504468B88F3B9CB88E3B94B887F2B48
:1057000019D803F07F0590F89C32032B0CD080F859
:105710009E522946FEF718FC204600F06AFA35B181
:10572000022384F89C3209E0FFF715FF06E001230D
:1057300084F89C3202E02046FFF70DFF38BD0000E0
:1057400038B504460D468978284B197001290ED8C2
:1057500090F89C32022B0ED0032B21D02946FFF764
:10576000FAFE224B19782046FFF798FD02E0294601
:10577000FFF7F1FE38BD81B14160032380F89C3210
:10578000FFF77FFD022803D0204600F032FAF1E750
:1057900029462046FFF7DFFEECE700F02AFAE9E7AA
:1057A00089B1436899421DD0D9B2FFF777FD0F4BFD
:1057B000197861602046FFF764FD02280DD020466D
:1057C00000F017FAD6E7022380F89C324160FFF719
:1057D00065FD204600F00DFACCE729462046FFF78C
:1057E000BAFEC7E700F005FAC4E700BFFC050020D9
:1057F00008B5CB88012B0CD190F89C325AB29AB1E3
:10580000022B09D9032B0FD10122011D00F0C5F98C
:1058100001E0FFF7A0FE08BD0146002341F8083F64
:10582000012200F0BAF9F6E7FFF795FEF3E708B5B5
:1058300090F89C32013B022B12D8CB88022B0CD162
:105840000123C360D0F8A4320BB10323C36002224A
:1058500000F10C0100F0A1F908BDFFF77CFEFBE7A9
:10586000FFF779FEF8E708B590F89C32013B022B70
:1058700009D84B88012B00D008BD0023C0F8A43202
:1058800000F0B7F9F8E7FFF766FEF5E708B50B7823
:1058900003F06003202B05D0402B03D043B1FFF76A
:1058A0005AFE03E0D0F8B4329B689847002008BD48
:1058B0004B78092B1BD8DFE803F011171A141A08CC
:1058C000051A0E0BFFF751FEF0E7FFF711FFEDE7AA
:1058D000FFF736FFEAE7FFF78BFFE7E7FFF7A7FFE2
:1058E000E4E7FFF71AFEE1E7FFF7BDFFDEE7FFF7AA
:1058F00032FEDBE738B505460C460B7803F0600353
:10590000202B06D0402B04D01BB1FFF724FE002033
:1059100038BD95F89C32013B022B16D82379012B18
:105920000ED8D5F8B4329B68214628469847E388BC
:10593000002BECD10028EAD1284600F05AF9E6E71E
:1059400021462846FFF707FEE1E721462846FFF7F4
:1059500002FEDCE738B504468A880B7803F0600362
:10596000202B08D0D0B2402B05D05BB12046FFF7EA
:10597000F2FD002005E0D4F8B4329B682046984739
:10598000002038BD202B13D04B78012B39D05DB2CD
:10599000002D64D0032B40F0DE8094F89C32022B63
:1059A0000CD0032B1CD02046FFF7D5FD0020E8E7E4
:1059B000D4F8B4329B6820469847E2E708B18028C3
:1059C00004D12046FFF7C7FD0020DAE70146204654
:1059D000FEF797FA80212046FEF793FA0020D0E7E1
:1059E0004B8823B918B1802801D0CB8823B1204639
:1059F00000F0FFF80020C4E701462046FEF781FAD8
:105A0000F5E794F89C32022B06D0032B16D02046E3
:105A1000FFF7A1FD0020B4E708B1802804D120469B
:105A2000FFF799FD0020ACE701462046FEF769FA32
:105A300080212046FEF765FA0020A2E74B88002B64
:105A400040F08E8010F07F0F04D1204600F0D1F896
:105A5000002096E701462046FEF75BFAF5E794F84A
:105A60009C32022B06D0032B2AD02046FFF773FD71
:105A7000002086E708B1802813D112F0800F15D1DD
:105A800000F07F0000EB8000830003F5A871214443
:105A9000043100250D600222204600F07EF82846E1
:105AA0006FE72046FFF757FD00206AE700F07F0010
:105AB00000EB8000830003F1100121440431E8E78A
:105AC00052B2002A1FDB00F00F0303EB83039D009B
:105AD0002544D5F8583123B3002A27DB00F07F0294
:105AE00002EB8202930003F5A8752544043508B142
:105AF000802825D100232B6002222946204600F071
:105B00004CF800203DE700F00F0303EB83039D00FA
:105B10002544AB69002BDFD12046FFF71CFD002098
:105B20002FE72046FFF717FD00202AE700F07F024D
:105B300002EB8202930003F1100525440435D6E7F9
:105B400001462046FEF7EDF910B101232B60D3E7A3
:105B500000232B60D0E72046FFF7FDFC002010E774
:105B600000200EE7C0B170B50D4616460446FFF79B
:105B7000CBFC013040003080287003236B7002237F
:105B8000217841B101345A1CD2B2E9540233DBB25C
:105B90000021A954F4E770BD704710B513460222E6
:105BA000C0F89422C36103620A460021FEF7D4F9CB
:105BB000002010BD08B513460A460021FEF7CCF9B7
:105BC000002008BD10B513460322C0F89422C0F887
:105BD0005C31C0F860310A460021FEF7C5F90020AB
:105BE00010BD08B513460A460021FEF7BDF9002096
:105BF00008BD08B50423C0F8943200231A4619469C
:105C0000FEF7AAF9002008BD08B50523C0F89432B4
:105C100000231A461946FEF7A7F9002008BD10B563
:105C2000D0F8B842D0F8BC325BB194F80002FF283B
:105C300007D09B6894F8012221469847FF2384F8F7
:105C40000032002010BD000043230380004870474D
:105C5000A80000204323038000487047EC00002088
:105C600043230380004870473C0100200A2303803F
:105C7000004870473001002038B50446D0F8B852CB
:105C8000FEF77AF9C5F80C02D4F8B8324BB1D4F863
:105C9000BC32DB6805F50371D5F804029847002093
:105CA00038BD0220FCE738B5D0F8B822D0F8C05291
:105CB000E2B101EB8104A3000344DB693BB105EBD6
:105CC0004115AD6BB3FBF5F405FB143323B1002391
:105CD000C2F81432002038BD01EB81029300034466
:105CE0000022DA611346FEF737F9F3E70220F2E704
:105CF00070B582B005460C46D0F8B86200238DF826
:105D00000730ADF804300B7813F0600227D0202A5A
:105D100056D1CA88DAB113F0800F0CD0D0F8BC325B
:105D20009B68314660789847E28831462846FFF7FD
:105D300034FF002047E04B7886F800328B7986F8F4
:105D40000132CA883146FFF73DFF00203BE0D0F822
:105D5000BC329B68002248789847002033E04B789B
:105D60000A2B14D00B2B21D01BB1FFF7F4FB022020
:105D700029E090F89C32032B03D0FFF7ECFB0220C4
:105D800021E0022201A9FFF708FF00201BE090F8A4
:105D90009C32032B03D0FFF7DEFB022013E001222D
:105DA0000DF10701FFF7F9FE00200CE090F89C329E
:105DB000032B01D1002006E0FFF7CDFB022002E01B
:105DC000FFF7C9FB022002B070BD38B5044681213F
:105DD000FEF78FF80025E56201212046FEF789F8DD
:105DE000C4F86C5182212046FEF783F82564D4F86C
:105DF000B8324BB1D4F8BC325B689847D4F8B802DB
:105E0000FEF7C4F8C4F8B852002038BD38B50446CF
:105E1000037CABBB4FF4007302228121FEF75EF8D6
:105E20000125E5624FF40073022229462046FEF761
:105E300055F8C4F86C510823032282212046FEF74E
:105E40004DF8012323644FF40770FEF79BF80546D5
:105E5000C4F8B80268B3D4F8BC321B689847002372
:105E6000C5F81432C5F81832237CCBB94FF400734F
:105E7000D5F8042201212046FEF776F8002038BD2F
:105E8000402302228121FEF729F80125E562402303
:105E9000022229462046FEF721F8C4F86C51CAE7D1
:105EA0004023D5F8042201212046FEF75DF80020AA
:105EB000E5E70120E3E719B1C0F8BC120020704704
:105EC00002207047D0F8B832C3F80812C3F8102285
:105ED00000207047D0F8B832C3F804120020704791
:105EE000D0F8B822A2B108B5D2F814320BB1012013
:105EF00008BD0123C2F81432D2F810320363B2F89D
:105F00001032D2F808228121FEF726F80020EFE7B0
:105F100002207047D0F8B82292B108B5037C43B98B
:105F20004FF40073D2F804220121FEF71DF800207F
:105F300008BD4023D2F804220121FEF715F8F6E748
:105F4000022070470268D36823F08003D360D0F842
:105F500004345A1CC0F8042403441971B0F80E34F8
:105F600001339BB2A0F80E34D0F80434B3F5806F3F
:105F700002D30023C0F80434D0F80424D0F8083445
:105F80009A4208D0012380F80C340268D36843F0A9
:105F90008003D3607047D0F808340133C0F8083468
:105FA000D0F80834B3F5806FECD30023C0F8083480
:105FB000E8E703460168CA6822F02002CA6090F848
:105FC0001828C2B9D0F81018D0F81428914208D374
:105FD000D0F8100880B2D3F8142892B2801A80B298
:105FE0000BE0D0F81008D3F81428801A80B200F51E
:105FF000806080B201E04FF480601A68D36843F09B
:106000002003D360704703460168CA6822F020026B
:10601000CA6093F818288AB9D3F81018D3F814284E
:1060200091420BD11968CA6842F02002CA6030BFA1
:106030001968CA6822F02002CA60EAE7D3F8142877
:106040001A4492F81004C0B2002283F81828D3F83A
:1060500014280132C3F81428D3F81428B2F5806F3D
:1060600002D30022C3F814281A68D36843F020032F
:10607000D36070470268D36843F02003D360704751
:1060800030B472B603681A6812F0200F1AD059683B
:10609000C9B290F81848ACB9D0F81048651CC0F8DF
:1060A0001058044484F81014D0F81018B1F5806F1B
:1060B00002D30021C0F81018D0F81048D0F81418F6
:1060C0008C4224D012F0800F2CD0D0F80414D0F8D9
:1060D000082491421FD0D0F80824511CC0F808149D
:1060E00002441279D2B25A60B0F80E349BB22BB18E
:1060F000B0F80E34013B9BB2A0F80E34D0F808344F
:10610000B3F5806F0ED30023C0F808340AE00121F4
:1061100080F81818D6E7DA6822F08002DA600023E7
:1061200080F80C3462B630BC704708B5FFF70AFF40
:1061300008BD01600023C0F80434C0F8083480F8BA
:106140000C34A0F80E34C0F81038C0F8143880F8B9
:106150001838704708B50248FFF792FF08BD00BF26
:106160006419002090F9003023F01C03CA789200D3
:1061700002F01C0213430370704790F9003003F0E3
:106180001F030A7943EA42130370704790F9003005
:1061900023F01C030A78920002F01C0213430370E0
:1061A000704790F9003003F01F034A7843EA421326
:1061B00003707047037803F007038B708378C3F391
:1061C00082030B7083785B094B70C378C3F382033F
:1061D000CB70C3785B090B71704700002DE9F84F55
:1061E0000C464068FAF7E8F8804689460022364BAC
:1061F000FAF75CF906460F462088FAF7DDF8824682
:106200008B460022314BFAF751F902460B463046D5
:106210003946F9F793FF06460F46B4F90200FAF73C
:10622000DBF832463B46FAF741F906460F460022B4
:10623000274B40464946FAF739F9804689460022FD
:10624000244B50465946FAF731F902460B46404670
:106250004946F9F773FF02460B46FAF727F98046DD
:106260008946B4F90400FAF7B7F802460B464046EF
:106270004946FAF71BF902460B4630463946F9F70C
:106280005FFF06460F46FAF7C1FB60620022124B21
:1062900030463946FAF734FA04460D4600220F4BD1
:1062A000FAF776FB48B900220D4B20462946FAF74B
:1062B0008DFB20B100240A4D01E00024074D20464B
:1062C0002946BDE8F88F00BF0000103F0000503F96
:1062D0000000E03E0000203F0000B440000044C049
:1062E00000405540000000002DE9F84F05460C46DF
:1062F000486AFAF771F80022874BFAF7D7F80022BC
:10630000864BF9F71BFF06460F4602460B46FAF787
:10631000CDF880468946B4F91000FAF75DF80246D8
:106320000B4640464946FAF7C1F800224FF07C532D
:10633000FAF7BCF880468946B4F90E00FAF74CF833
:1063400032463B46FAF7B2F802460B46F9F7F8FE3A
:1063500042464B46F9F7F4FE0022714BFAF7A6F8D5
:1063600080468946B4F90C00FAF736F800226D4BE6
:10637000FAF79CF802460B4640464946F9F7E0FE1C
:1063800080468946B4F90A00FAF726F832463B46B9
:10639000FAF78CF832463B46FAF788F800224FF0BD
:1063A0007B53FAF783F882468B46B4F90800FAF774
:1063B00013F832463B46FAF779F852465B46F9F74E
:1063C000BFFE00224FF07B53FAF770F800224FF027
:1063D0007C53FAF76BF80022534BF9F7B1FE0646EF
:1063E0000F46E088F9F7E8FF02460B46304639468B
:1063F000FAF75CF882468B4600220023FAF7E6FAA9
:1064000000286FD02868F9F7D7FF02460B46002016
:106410004649F9F793FE06460F460022444B404694
:106420004946FAF743F802460B4630463946F9F733
:1064300085FE33A3D3E90023FAF738F852465B46CA
:10644000FAF75EF906460F46B4F91600F9F7C4FFED
:1064500032463B46FAF72AF832463B46FAF726F828
:1064600000224FF07853FAF721F880468946B4F9B4
:106470001400F9F7B1FF32463B46FAF717F800224D
:106480004FF07C53FAF712F802460B464046494655
:10649000F9F756FE80468946B4F91200F9F79CFFD9
:1064A00002460B4640464946F9F74AFE0022214B78
:1064B000F9F7FCFF32463B46F9F742FE04460D462B
:1064C00011A3D3E90023FAF763FA90B910A3D3E933
:1064D000002320462946FAF779FA30B10CA5D5E910
:1064E000004502E008A5D5E9004520462946BDE85B
:1064F000F88F05A5D5E90045F7E700BFAFF30080A9
:1065000000000000006AB84000000000004CDD40C0
:106510000000000000DBFA400000E03F0040EF40D8
:106520000000D03F0000F0400000F03F000030418C
:106530000000303F0000B03F2DE9F04784B08046B6
:106540008A46486AF9F748FF0022524BF9F7F6FDF0
:1065500006460F46BAF91E00F9F73EFF00224E4BE1
:10656000F9F7A4FF04460D46BAF92000F9F734FF05
:1065700000224A4BF9F79AFF32463B46F9F796FF5D
:1065800002460B4620462946F9F7DAFD04460D4639
:10659000D8F80800F9F710FF22462B46F9F7CEFD90
:1065A000CDE90001BAF91A00F9F716FF00223C4BB9
:1065B000F9F77CFFCDE902019AF81C00F9F7FCFE1F
:1065C0000022384BF9F772FF32463B46F9F76EFF6F
:1065D0000022354BF9F7B4FD04460D469AF9220026
:1065E000F9F7FAFE00222F4BF9F760FF32463B46DF
:1065F000F9F75CFF22462B46F9F758FF00222A4B99
:10660000F9F79EFD80468946DDE90223DDE90001B8
:10661000F9F74CFF06460F4642464B4620462946B0
:10662000F9F744FF02460B4630463946F9F73EFF7C
:1066300004460D469AF81800F9F7BEFE22462B468E
:10664000F9F734FF00224FF07B53F9F72FFF024692
:106650000B4600201449F9F771FD22462B46F9F745
:1066600025FF04460D460022104BFAF7AFF948B952
:106670000022002320462946FAF78AF920B1002497
:10668000002501E00024094D2046294604B0BDE85C
:10669000F08700BF00C0F240000050400000103FF3
:1066A0000000F03E0000503E0000F03F0000594066
:1066B00070B401249C4209D26500013D065D4E552F
:1066C000155D01F814500134E4B2F3E770BC704773
:1066D0004278037843EA02230B83C278837843EA43
:1066E00002234B834279037943EA02238B83C279E5
:1066F000837943EA0223CB83427A037A43EA022373
:106700000B84C27A837A43EA02234B84427B037B65
:1067100043EA02238B84C27B837B43EA0223CB843C
:10672000427C037C43EA02230B85C27C837C43EAE0
:1067300002234B85427D037D43EA02238B85C27D84
:10674000837D43EA0223CB85437E81F83030704756
:106750004278037843EA02234B86837881F8343009
:1067600090F903309BB21B011BB2027902F00F02B9
:106770001343CB8690F905309BB21B011BB2027903
:1067800043EA12130B8790F9063081F83A307047CC
:10679000084201D0012070470020704750B1C26804
:1067A0005AB1026962B143690BB1002070474FF0E2
:1067B000FF3070474FF0FF3070474FF0FF307047A9
:1067C0004FF0FF3070472DE9F84305460E469146DD
:1067D0001C461846FFF7E2FF90B980469EB1237A27
:1067E000012B01D045F08005E76863684A463146D1
:1067F0002846B84784F8450040B94046BDE8F883CC
:106800004FF0FF38F9E74FF0FF38F6E76FF0030875
:10681000F3E730B589B00446002301930293039354
:10682000049305930693ADF81C3003461A2201A980
:106830008820FFF7C8FF054610B1284609B030BDD3
:10684000214601A8FFF744FF2346072201A9E120C2
:10685000FFF7B9FF05460028EFD1214601A8FFF751
:1068600077FFEAE72DE9F04186B005460F4614466A
:106870001E460A2A00D90A243046FFF78FFF8046B9
:1068800058BB6DB37FB38CB33B788DF80430337A4B
:10689000012B09D000239C4206D9E95C01F07F015D
:1068A000E9540133DBB2F6E7012C0CD8A2B2376908
:1068B000736801A92878B84786F84500C8B94046EA
:1068C00006B0BDE8F08123463A4601A92846FFF705
:1068D000EFFE6400013CA2B2E9E74FF0FF38EEE7BB
:1068E0004FF0FF38EBE74FF0FF38E8E76FF00208B2
:1068F000E5E76FF00308E2E710B582B00C46F2233B
:106900008DF80530837803F007038DF807300B46C8
:1069100001220DF107010DF10500FFF7A3FF03466A
:1069200010B1184602B010BDF4208DF805002346C2
:1069300001220DF10601FFF746FF03460028F0D1C2
:10694000234601220DF106010DF10500FFF78AFF34
:106950000346E6E770B582B005460E461446F420BD
:106960008DF80700134601220DF10601FFF72BFFFA
:10697000034670B915F0010F0ED115F0020F11D1B9
:10698000234601220DF106010DF10700FFF76AFF12
:106990000346184602B070BD31460DF10600FFF700
:1069A000F5FBEAE731460DF10600FFF7FAFBE7E7F2
:1069B00070B504460D46164610F0040F04D10120B0
:1069C00014F0030F05D170BD11462846FFF794FF60
:1069D000F6E7324629462046FFF7BCFFF3E770B5DD
:1069E00082B005460E461446F5208DF80700134682
:1069F00001220DF10601FFF7E6FE034670B915F01E
:106A0000080F0ED115F0100F11D1234601220DF100
:106A100006010DF10700FFF725FF0346184602B0F7
:106A200070BD31460DF10600FFF79CFBEAE73146E9
:106A30000DF10600FFF7A1FBE7E738B504460D4668
:106A40000A4601461F20FFF7B3FF034608B1184668
:106A500038BD2A4621461F20FFF7C1FF0346F6E74F
:106A600030B583B005460C46F4208DF807000B4680
:106A700001220DF10601FFF7A6FE034610B11846EC
:106A800003B030BD9DF8060020F0030040B205F0D1
:106A9000030528438DF80600234601220DF1060167
:106AA0000DF10700FFF7DEFE0346E8E738B50446C0
:106AB0000D460846FFF772FE58B96CB12B4601220D
:106AC0002146F420FFF77FFE237803F003032370B1
:106AD00038BD4FF0FF30FBE74FF0FF30F8E730B53F
:106AE00083B00446E0238DF8073000238DF806308C
:106AF000B6238DF80530FFF751FE034610B1184656
:106B000003B030BD234601220DF105010DF1070050
:106B1000FFF7A8FE03460028F1D1052500E0154641
:106B2000636961684FF4FA609847234601220DF1CA
:106B30000601F320FFF747FE034638B96A1ED2B2BA
:106B400025B19DF8061011F0010FE8D19DF806203F
:106B500012F0010FD3D06FF00503D0E770B582B00B
:106B6000054600238DF80730FFF718FE064648B3A8
:106B7000304602B070BD2846FFF74BFE06461CE0CB
:106B80006B6969684FF47A709847013CE4B2A4B12C
:106B90002B4601220DF10701D020FFF714FE064617
:106BA0000028EDD19DF80730602BE9D12B702846E5
:106BB000FFF795FF06460028DDD0002CD8D16FF0F6
:106BC0000106D5E70524E2E710B584B00446034684
:106BD000042203A9F220FFF7F6FD034610B1184680
:106BE00004B010BD01A903A8FFF7E4FA2046FFF79F
:106BF00076FF03460028F2D1214601A8FFF71DFFCA
:106C00000346ECE770B582B006460D460846FFF72E
:106C1000C5FD044610B1204602B070BD29460DF1F5
:106C20000700FFF743FF044610B99DF80730B3B9DA
:106C3000002CF0D131460720FFF7AAFDA0B9002CA7
:106C4000E9D131461820FFF7A3FD0028E3D02A46FA
:106C500005F140013046FFF7C2FE0446DBE7284657
:106C6000FFF7B2FF0446E3E72A4605F1400130464C
:106C7000FFF79EFE0446E2E730B583B005460C46BA
:106C80000846FFF78BFD034610B1184603B030BD30
:106C900021460DF10700FFF709FF034610B99DF8E3
:106CA00007203AB9002BF0D121462846FFF7D8FE3D
:106CB0000346EAE72046FFF787FF0346F2E710B4F2
:106CC000047843781B01827843EA043343EA1213C1
:106CD0000B60C47803791B01427943EA043343EA29
:106CE00012134B608279C37943EA02238B6010BC94
:106CF000704761B3F8B50F4662B373B31E461446CE
:106D0000054600220023C4E90223C4E90023C4E9A4
:106D1000042310F0070F13D115F0010F05D03146F1
:106D20003846FFF7E1FAC4E9000115F0040F17D067
:106D300031463846FFF700FCC4E904010020F8BDE5
:106D400031463846FFF74AFAC4E90201E4E74FF05A
:106D5000FF3070474FF0FF30F1E74FF0FF30EEE7C4
:106D60000020ECE770B586B006460D4614460023B9
:106D7000049305930193029303931046FFF70EFDCE
:106D8000C0B9D5B12346082204A9F720FFF71BFD9F
:106D9000034610B1184606B070BD01A904A8FFF75C
:106DA0008EFF04F118032A4601A93046FFF7A1FF20
:106DB0000346EFE74FF0FF33ECE74FF0FF33E9E72F
:106DC00082B002461C4B93E803000090ADF804101B
:106DD0005378052B04D802A90B4413F8083C00E0B3
:106DE00010231178052904D802A8014411F8081CC1
:106DF00000E010219278052A04D802A8024412F873
:106E0000080C00E0102040F6FC0202FB03F303F242
:106E1000E24302FB01F101F23F210B4402FB00F2CD
:106E200002F23F200344054880FB0320DB17C3EB3D
:106E3000A01002B0704700BF00C90008D34D621017
:106E400008B528B10268117002680132026008BDFD
:106E50000846FFF76AF9FAE72DE9F04107460E46C2
:106E6000151E06DD0A460021107880B1013101327D
:106E7000FAE74FF0200813F001041CD00024317809
:106E800011B33846FFF7DCFF01340136F7E7A942BA
:106E900001DA6D1A00E0002513F0020F02D14FF065
:106EA0002008E8E74FF03008E5E741463846FFF7AD
:106EB000C7FF0134013D002DF7DCE0E741463846CD
:106EC000FFF7BEFF0134013D002DF7DC2046BDE891
:106ED000F081F0B585B007460C9859B11E460C46B6
:106EE00013B10A2A13D0002600238DF80F300DF1BC
:106EF0000F0518E030238DF8043000238DF805309D
:106F00000B9B0A9A01A93846FFF7A6FF29E0002942
:106F100001DB0026E8E74C420126E5E7303305F8BF
:106F2000013DB4FBF2F44CB1B4FBF2F302FB1343AA
:106F3000092BF3DDA0F13A010B44EFE756B10A9BB0
:106F40001BB10B9B13F0020F0DD12D2305F8013C53
:106F5000013D00260B9B0A9A29463846FFF77CFF25
:106F6000304405B0F0BD2D213846FFF769FF0A9B7C
:106F7000013B0A93EEE7000070B588B006460C4668
:106F800005920025A9E0611C6378002B00F0AE801B
:106F9000252B00F095802D2B07D000230A78302A6E
:106FA00006D1013143F00203F8E7A11C0123F5E704
:106FB0002A2A2BD1059A101D059012684C1C2178A5
:106FC0006C2925D02178732924D064292DD07829E3
:106FD0003AD0582947D0752954D0632961D06E29F9
:106FE0007AD1059B1A1D05921B681D6074E002EBA7
:106FF00082025400A0F13002224401310878A0F14D
:107000003004E4B2092CF2D90C46D8E70022F5E7A7
:107010000134D7E70599081D0590096801B937497A
:107020003046FFF719FF054456E00599081D059005
:107030000968612002900193009201230A223046E0
:10704000FFF747FF054447E00599081D05900968CB
:107050006120029001930092002310223046FFF736
:1070600038FF054438E00599081D0590096841205E
:10707000029001930092002310223046FFF729FF6F
:10708000054429E00599081D0590096861200290D2
:107090000193009200230A223046FFF71AFF0544AD
:1070A0001AE00599081D059009788DF81C1000213B
:1070B0008DF81D1007A93046FFF7CEFE05440BE002
:1070C0000C460FE00D213046FFF7BAFE013521785E
:1070D0003046FFF7B5FE01350134237833B1252B57
:1070E0003FF451AF23780A2BF1D1EBE716B13368A7
:1070F00000221A70284608B070BD00BF80C9000881
:107100000EB400B584B0019005AA52F8041B039296
:1071100001A8FFF731FF04B05DF804EB03B070473E
:10712000303840B27047000010B50446FFF7F8FF52
:1071300000280DDA0A4BE35C03F00303012B09D0AE
:10714000E4B2A4F16103DBB2052B05D9002000E015
:10715000C0B210BD2034F3E7573CE0B2F9E700BFFE
:10716000A1D4000800000000F8B507460846F9F76A
:107170009FFD0446002300251EE0F9F799FD2146F6
:10718000F9F7EAFD01462846F9F7DEFC05464FF01F
:107190007E512046F9F7D6FC20F00040F9F72EF991
:1071A0000BA3D3E90023F9F7F3FB78B90A4920468A
:1071B000F9F786FE044633465E1CF85C2E28FAD0AA
:1071C000FFF7AEFF0028D8DC2846F8BD034CF2E7F5
:1071D0007B14AE47E17A843F00002041ABAA2A3EEF
:1071E00070B5064600242546012D0BDC3078FFF7EC
:1071F00097FF002805DB04EB84046300C418013505
:10720000F2E70024204670BD08B5002102F0C0F965
:1072100008BD2DE9F04395B006460F469046002381
:107220001D46FC1E9C4203DDF25C55400133F8E72D
:10723000BB1EF05CFFF778FF00015FFA80F9013FA9
:10724000F05DFFF771FF4844C0B2854240F089808D
:107250000523002100E001339C420BDDF25C2C2A67
:10726000F9D15A1C324414A800EB810040F8502C8C
:107270000131F0E7B378522B01D0012072E0F378AE
:107280004D2B01D001206DE03379432B01D001203B
:1072900068E0019C237888F80030412B01D0012060
:1072A00060E008F10106009B1A68C8F801209B887D
:1072B000A8F805300A210298FFF756FFC8F8140015
:1072C000039B1B7888F8113064210498FFF74CFF6A
:1072D000C8F81800059B1B7888F810300698FFF74F
:1072E00093FFC8F820000798FFF78EFFC8F81C002E
:1072F00008F107052368C8F80730A388A8F80B3001
:1073000008F10500FFF76CFFC8F8240008F103003E
:10731000FFF766FFC8F828003046FFF761FFC8F89E
:107320002C002846FFF75CFFC8F8300008F1090080
:10733000FFF756FF0138C8F8340008F10B00FFF7DB
:107340004FFF6430C8F838000023C8F8443008F113
:10735000240001F04BF9C8E91201012088F80F0060
:1073600000E0002015B0BDE8F08300002DE9F843EF
:1073700080460E4604E024281DD02C4B00221A60C3
:107380003046FEF716FE00284CD03046FEF73BFE96
:107390000746274B1B78002BEDD0012BF0D10D2891
:1073A0000DD0224B1B684F2B14D8591C1F4A11605B
:1073B000204AD054E4E71E4B01221A70DDE71B4C33
:1073C000424621681B48FFF724FF0023184A137028
:1073D000236028E00024164B1C7000E00134254691
:1073E000124A13689C4215D2124A125D242AF5D122
:1073F000611C5D1BDFF83C902A464944484601F079
:1074000005F86A1C094B1A6009F80570084B01223F
:107410001A70E3E7064B1B78002BB1D1134600220C
:107420001A60ADE70020BDE8F88300BF0006002029
:107430000406002080210020002A26DB70B4457954
:10744000954224DD002B25DB04799C4224DD1F2995
:1074500000D82021A1F12004E4B25F2C0CD886686A
:10746000A1F1200404FB0524345DB02906D044FAC0
:1074700003F000F001000BE00024F6E7806805EB64
:10748000450569010A44845CF1E70020704700204B
:1074900070BC70470020FBE70020F9E7002A28DBDA
:1074A00070B44579954226DD002B27DB04799C4298
:1074B00026DD01F07F0411F0600F00D12024C17996
:1074C00001F11F06A64200DA2024203C04FB05221D
:1074D00003FB05F303FB0123002B08DBDB108168B2
:1074E000C85C02F00702104100F0010004E007331D
:1074F000F4E700207047002070BC70470020FBE7D5
:107500000020F9E7012800D070474FF6FF73994239
:10751000FAD10C4B07221A7105225A7106229A7170
:107520006022DA710849996008491960084B1221F4
:1075300019710A2159719971DA71064A9A60064ADD
:107540001A60E1E71406002088C90008F4D3000897
:107550000806002070CB0008E8D3000808B54FF6F5
:10756000FF710120FFF7CEFF08BDB0F90030B1F97F
:10757000002002800B8070470028B8BF404200B254
:1075800070477047FEE7000030B4074D056041606A
:107590008260C36000230361436183610123037739
:1075A000029B036230BC704700D40008704708B5E6
:1075B00003681B69984708BDF0B583B0ADF80610A5
:1075C000ADF80420002973DB4268914270DABDF9FE
:1075D0000460002E6CDB8768BE4269DA1D460446F3
:1075E0008369022B1DD0032B26D0012B0BD0237FC8
:1075F000012B2FD9237F002B43D0032B44D8002D00
:107600005AD0012141E001A90DF10600FFF7ADFFBD
:107610006368BDF806209B1A9BB2013BADF80630AB
:10762000E5E7521A92B2013AADF80620BB1B9BB2B5
:10763000013BADF80430DAE701A90DF10600FFF7D0
:1076400094FFA368BDF804209B1A9BB2013BADF8E0
:107650000430CCE7206ABDF904201346002A0EDB73
:10766000DB106668BDF9061006FB031302F0070283
:1076700001219140C25C22EA0102C254BAE7D31D43
:10768000EEE7BDB1002100E00021206ABDF9042031
:107690001346002A12DBDB106568BDF9064005FBC6
:1076A000034302F0070201FA02F2C15C4A40C254ED
:1076B00003B0F0BD0121E8E70021E6E7D31DEAE7CA
:1076C000F8B5044603689B68002198472368DB6887
:1076D0002121204698472368DB68002120469847EF
:1076E0002368DB68E1680139C9B2204698472368FE
:1076F000DB682221204698472368DB68002120466A
:1077000098472368DB68A268402A08D003212046F6
:107710009847E368842B04D0002700252BE007213D
:10772000F5E70227F9E7B5EBE30F29DA23689B6851
:107730000021204698472368DB68A5F15001C9B2B3
:10774000204698472368DB683946204698472368D7
:10775000DB6810212046984723689B68012120465A
:10776000984723685E69216A6368DAB205FB0311F2
:107770002046B0470135A368002BD4DA0733D2E79F
:10778000F8BD08B503290FD8DFE801F01102022087
:10779000036A4168826802FB01F2002A05DBD2100D
:1077A000FF21184600F040FE08BD0732F7E7036AE4
:1077B0004168826802FB01F2002A05DBD210002139
:1077C000184600F031FEEFE70732F7E7002207E046
:1077D000B2EBE30FE8D2016A8B5CDB438B540132DE
:1077E0004168836803FB01F3002BF1DA0733EFE70D
:1077F00010B5044603689B68002198472368DB683E
:10780000AE21204698472368DB68D521204698475B
:107810002368DB688021204698472368DB68A8211D
:10782000204698472368DB68A1680139C9B2204621
:1078300098472368DB68D321204698472368DB6894
:107840000021204698472368DB684021204698475E
:107850002368DB688D21204698472368DB68102168
:10786000204698472368DB682021204698472368F4
:10787000DB680021204698472368DB68A121204669
:1078800098472368DB68C821204698472368DB684F
:10789000DA21204698472368DB68A268202A34D082
:1078A0001221204698472368DB68812120469847AB
:1078B0002368DB689F21204698472368DB68D9212D
:1078C000204698472368DB68222120469847236892
:1078D000DB68DB21204698472368DB68402120468F
:1078E00098472368DB68A421204698472368DB6813
:1078F000A621204698472368DB68AF212046984799
:1079000000212046FFF73DFF10BD0221C9E72DE908
:10791000F04F85B001900C4615469DF83C2002774B
:107920001B1B1FB2BDF938B0ABEB050B0FFA8BFB7D
:10793000002F1DDB01230293BBF1000F20DB4FF072
:10794000010ABEB24FEA46081FFA88F81FFA8BF305
:107950004FEA43091FFA89F95F4530DDA9EB0606B6
:1079600036B24FF0000BCDF80C80DDF8088016E041
:107970003846FFF701FE07464FF0FF330293DBE77F
:107980005846FFF7F9FD83464FF0FF3AD9E74E44DA
:1079900036B2444424B20BF1010B1FFA8BFBBB45FA
:1079A00029DC01232A4621460198FFF705FE002E17
:1079B000EDDB039BF61A36B255442DB2E7E7A8EB90
:1079C000030636B2002705E0464436B255442DB2D0
:1079D0000137BFB25F450EDC01232A4621460198DC
:1079E000FFF7EAFD002EEFDBA6EB090636B2029B9D
:1079F0001C4424B2E8E705B0BDE8F08F2DE9F04F54
:107A000087B082460E46059203939DF84030037777
:107A10004B79013304930023019331E00BF1010B07
:107A20001FFA8BFB039B9B4526D2059B13F80B90FB
:107A3000049B03FB0BF81FFA88F8BAF8103098443F
:107A40001FFA88F80024B379A342E7D904EB0805AC
:107A5000ADB233681F68019B224649463046B8479D
:107A6000031C18BF0123BDF9082029B25046FFF7B7
:107A7000A3FD0134A4B2E6E7019B01339BB201935D
:107A80003379019A934207D9BAF8143013449BB260
:107A900002934FF0000BC5E7DAF81030049A03990F
:107AA00001FB0233CAF8103007B0BDE8F08F0000C8
:107AB000F0B59DF814C0069EBCF1FF0F0CD0581C09
:107AC000C0B2A0EB0C0C5FFA8CFC002E06DB00238E
:107AD00000240C54054608E01846F2E776420123DC
:107AE000F6E7013DEDB22E244C55CDB1954217D2AB
:107AF0006545F6D00D4F87FB0647F417C4EBA70486
:107B0000274604EB84044FEA440EA6EB0E04013D25
:107B1000EDB230344C553E46002FE6D1AC45E4D9A9
:107B20001BB1013DEDB22D234B55F0BD6766666676
:107B3000F0B587B005460E4617460E4A03AC07CA95
:107B400003C4227000228DF815200C9A0192009334
:107B50003B460A2203A92846FFF7AAFF9DF83430C6
:107B6000009383B203AA31462846FFF747FF07B0C8
:107B7000F0BD00BF08C90008012800D0704708B553
:107B80004FF6FF73994200D008BD024800F094F907
:107B9000FAE700BF2006002010B4016002714371B3
:107BA0009DF804308371BDF80830038110BC704724
:107BB0002DE9F04F85B00746B439048904FB01F183
:107BC000314C84FB01340C44C917C1EB64142F4DB4
:107BD0002146284600F09CF983462146284600F0BD
:107BE000CEF98246A4F5B4742146284600F090F9F7
:107BF000804602902146284600F0C1F90390BE79E4
:107C000006F102097600224B83FB063643465D42AD
:107C100044424FF00008B8F1020F32DC09FB0BF1CF
:107C2000491B1A4BD3F800E0B1FBFEF197F804C0F2
:107C30006144787909FB0AF2121BB2FBFEF2821A48
:107C400006FB0BF35B1BB3FBFEF3634406FB0AFC72
:107C5000ACEB040CBCFBFEFCA0EB0C004FF0030CE7
:107C6000CDF804C000B200901BB212B209B238685D
:107C7000FFF74DFE029B1D44039B1C4408F10108C5
:107C8000C9E705B0BDE8F08FB7600BB6200600204D
:107C9000565555552DE9F04F85B080460393BDF9F3
:107CA0003C304181828191FBF3F192FBF3FB03892C
:107CB0005802ABEB0102920090FBF2F9C3EB0363B5
:107CC0001F028D002FE007F13F0632E0DDF80CA027
:107CD00098F806C004FB0CF12E4B1B68B1FBF3F1C6
:107CE00098F804E0714498F8056000FB0CF2B2FBD0
:107CF000F3F2B21AACEB0A0C04FB0CF4B4FBF3F491
:107D0000744400FB0CF0B0FBF3F3F61A012301936B
:107D100036B2009623B212B209B2D8F80000FFF7CB
:107D2000F6FD4F440135B5EB8B0F2FDC3E46002F9F
:107D3000C9DBB6113146174800F0EAF8044631466F
:107D4000144800F01CF96A4205F0030302F0030234
:107D500058BF53420333062BBAD801A252F823F07E
:107D60007D7D0008857D00087D7D0008CD7C0008B4
:107D70007D7D0008857D00087D7D0008039B4FEA1E
:107D8000930AA5E7039B4FEA530AA1E705B0BDE8B4
:107D9000F08F00BF2006002008B54FF6FF710120CC
:107DA000FFF7EAFE08BD08B50346806A9B8D21B146
:107DB00001221946FAF72EFB08BD0022F9E710B59B
:107DC00004460122818E006BFAF724FB0120F9F7AB
:107DD000E7FD0022A18E206BFAF71CFB0A20F9F7C1
:107DE000DFFD0122A18E206BFAF714FB10BD10B548
:107DF00082B004468DF804100022818F806BFAF760
:107E000009FB0223012201A9606AFAF713FC01228F
:107E1000A18FA06BFAF7FEFA02B010BD70B5044650
:107E20000D4616460022818F806BFAF7F3FA642321
:107E300032462946606AFAF7FDFB0122A18FA06B4A
:107E4000FAF7E8FA70BD000010B50446024B036073
:107E5000FFF7ACFB204610BD20D4000810B5044647
:107E6000044B0360FFF7A2FB40212046FFF789FB8C
:107E7000204610BD20D4000830B583B00446069DCE
:107E80000095FFF781FB0B4B2360079B6362089B08
:107E9000A362BDF82430A3850A9B2363BDF82C3070
:107EA000A3860C9BA363BDF83430A387204603B0A0
:107EB00030BD00BF20D4000870B506464FF4807373
:107EC00003600024B4F5B47F18D22046F8F784FA92
:107ED00000220D4BF8F714FC09A3D3E90023F8F7AF
:107EE000E5FA03F045FB0022084BF8F7DFFA3519F5
:107EF000F8F7B4FD28710134A4B2E3E7304670BD51
:107F00006E861BF0F9210940008086400000704019
:107F1000002902DA01F5B461FAE7B1F5B46F02DBCA
:107F2000A1F5B461F9E7B1F5B47F15D3B1F5B47F2C
:107F300015D0A1F26912B2F5B47F12D3B1F5876FF3
:107F400014D0A1F2D123B3F5B37F12D8A1F53471C7
:107F5000014408794042704701440879704700683D
:107F60007047C1F534710144087970470068404298
:107F70007047C1F5B461014408794042704708B5C3
:107F8000C1F5B471FFF7C4FF08BD0000012800D09F
:107F900070474FF6FF739942FAD110B588B0134C71
:107FA0004022079203F1804303F601030693102158
:107FB000059104930821039102930D4B01930D4BFE
:107FC0000093842380212046FFF756FF0A4A0B497D
:107FD000204600F0D0F9B4230193202300936022BF
:107FE00021460748FFF7D8FD08B010BD9C070020C8
:107FF000F00D0020DC07002000000020497E000872
:108000008C07002010B582B0104C2046FFF7CFFA45
:108010002046FFF7EDFB00212046FFF7B2FB2D23A2
:1080200001930123009308234FF4B4720021084800
:10803000FFF730FE2046FFF743FB064B4FF02D3293
:10804000C3F80120A3F8052002B010BD9C07002052
:108050008C070020E80B00202DE9F043BBB08046E0
:1080600000219948FFF78DFB2D23019301230093F5
:1080700008234FF4B47200219448FFF70BFE944C90
:1080800094492046FFF772F9E37B33B1E069F9F7D1
:108090003FF8914B18600023E3738D4B1B78562BF0
:1080A00000F08E80884C002323616361884F8B4EE3
:1080B0000125009502237A1931462046FFF79EFCE0
:1080C000DFF8549200952B464A4631462046FFF78A
:1080D00095FC00950223FA1C31462046FFF78EFCE2
:1080E00000952B464A4631462046FFF787FC00950F
:1080F00002237A1D31462046FFF780FC764B196833
:10810000B43109B27148FFF753FD462323611923A7
:1081100063613B78412B5BD0012300930423704AB9
:1081200070496948FFF76AFC694B1B78412B5AD0AC
:10813000654C0026266108236361DFF8A0910125C4
:1081400000950523684A49462046FFF757FC2661FB
:10815000102363616549664B1868F8F7FDFD614FB0
:108160000195F8F7D5FF00902B46042239462046AA
:10817000FFF7DEFC266120236361009507235D4A3B
:1081800049462046FFF73AFC266128236361574998
:10819000594B1868F8F7E0FD0195F8F7B9FF009022
:1081A0002B46042239462046FFF7C2FCF9F7F2FBC2
:1081B000524B1B68C01A642823D83BB0BDE8F0833B
:1081C000434B4FF02D32C3F80120A3F8052069E797
:1081D0000195414B1B680093FF2303224149204630
:1081E000FFF7A6FCA0E73A4B186AF8F707F934A3A3
:1081F000D3E90023F8F784FAF8F750FC3C4B1860F9
:1082000096E7F9F7C7FB3D4B1860424602A90720E5
:10821000FEF7A8FD3A4B18600028CED101960096D3
:1082200033463246374908A8FEF76AFF0546012360
:108230003246AB4207DA3AA9194411F8C81C0A447D
:10824000D2B20133F5E7304908AB5819FEF758FFB1
:10825000291889B208A8FBF763FD1B4C002727618A
:10826000382363611D4E012500950223274A3146BC
:108270002046FFF7C3FB019500972B4604223146A9
:108280002046FFF755FC00950223214A314620463F
:10829000FFF7B4FB019500973B4605223146204687
:1082A000FFF746FC00952B461A4A31462046FFF759
:1082B000A5FB2046FFF704FA7FE700BFAFF300807D
:1082C0000AD7A3703D0AFD3F9C0700208C070020C1
:1082D000E80B002064190020DC0B002014060020AD
:1082E0003CD400080806002044D4000800002041C7
:1082F000400C00204CD400083C0C0020E00B002077
:10830000380C002054D400088CD4000894D4000801
:1083100098D400089CD4000838D4000808B54FF65B
:10832000FF710120FFF732FE08BD0000002103E0CD
:108330000B4B5B58435004310A480B4B42189A428E
:10834000F6D30A4A02E0002342F8043B084B9A4263
:10835000F9D3FAF7A3FC00F035F8F9F721F97047E3
:108360008CDA000800000020BC030020C0030020BD
:10837000E0210020FEE70B460146184600F000B859
:1083800010B5054C13462CB10A4601460220AFF346
:10839000008010BD2046FCE70000000008B5074B38
:1083A000044613B10021AFF30080054B1868836ABF
:1083B00003B19847204604F04BFA00BF00000000CC
:1083C000A4D5000870B500260C4D0D4C641BA410FC
:1083D000A64209D104F074FA00260A4D0A4C641B27
:1083E000A410A64205D170BD55F8043B984701364C
:1083F000EEE755F8043B98470136F2E778DA0008D3
:1084000078DA000878DA000888DA00080A4491422D
:1084100000F1FF3300D1704710B511F8014B9142C4
:1084200003F8014FF9D110BD03460244934200D135
:10843000704703F8011BF9E7F7B5016804463B29CB
:1084400011D93C22684601F02DFB019A636800991E
:10845000002A0B446360BBBF3C3203F1FF33226050
:108460002260B8BF636061683B2911D93C2268462D
:1084700001F018FB019AA3680099002A0B44A3603D
:10848000BBBF3C3203F1FF3362606260B8BFA360E0
:10849000A168172911D91822684601F003FB019A37
:1084A000E3680099002A0B44E360BBBF183203F174
:1084B000FF33A260A260B8BFE36021690B2911D924
:1084C0000C22684601F0EEFA019A63690099002ACD
:1084D0000B446361BBBF0C3203F1FF3322612261A5
:1084E000B8BF63616369990720D1642193FBF1F2FE
:1084F00001FB1232E2B94FF4C87103F26C7393FBC3
:10850000F1F201FB1233002B14BF1C231D23E26880
:10851000002A0FDC0B2664204FF4C875324FD4F8C4
:108520000CC0BCF1000F14DD03B0F0BD1C23EEE75E
:108530001D23ECE74FF0000C64254FF4C8762A4F5A
:10854000D4E90312012A2FD057F8220081422EDCF1
:10855000EAE7216901392161013114D16369591EAA
:108560008A07C4E9046117D191FBF0F200FB1211F4
:10857000A1B903F26B7393FBF5F205FB1233002BE9
:1085800014BF1C231D232269012A0CBF1A4657F869
:1085900022206244E260C2E71C23F4E71D23F2E7D5
:1085A0001C23CDE71D23CBE78B42BDDA18460132F1
:1085B000091A0C2AE1602261C2D163695A1C910731
:1085C000C4E904C2ECD192FBF5F105FB1122002AAB
:1085D000E8D103F26D7393FBF6F206FB1233002B26
:1085E00014BF1C231D23ABE7A8D500082DE9F04FCD
:1085F0008BB0064601F0D6FD4FF03C0A07463046E8
:10860000FFF71AFFD6E900230AFB03234FF4616A40
:10861000B068BC4A0AFB003AD6E9034352F823206B
:10862000013C012B1444756911DDA9070FD16422A7
:1086300095FBF2F302FB135343B94FF4C87205F2F2
:108640006C7191FBF2F302FB131303B9013444F68E
:10865000206205F51C5310339342F46100F27881D7
:10866000462D7EDD462340F26D1E64214FF4C87016
:108670009A0770D1B3FBF1F201FB1232002A6DD1DF
:1086800003F26C7CBCFBF0F200FB12C2002A14BFA8
:1086900072464FF4B77201339D421444E8D19A4BAD
:1086A0004FEAEA7BC3FB04ABCDE900AB01F06AF80B
:1086B00001F074F8954BD3F80090B9F1000F42D057
:1086C000D6F8209070697B68B9F1010F00F26C70E8
:1086D000C846A8BF4FF00108834240F08480D7E924
:1086E0001223D7F850C0D7F828E06046B2EB0E0A44
:1086F00063EBEE7BCDE90223DDE90023524573EB0A
:108700000B034FEAE071CDE906AB73DA3B6A1B1A43
:1087100004937B6A63EB01033968059300297AD0DF
:10872000DDE90401DDE900AB82457BEB010305DBFC
:10873000DDE9060182457BEB010374DBB9F1000F33
:108740004FF0000974DADDE900ABBB6A1AEB030AEB
:108750004BEBE37BB7E040F26D129CE74FF4B7724E
:1087600099E79CD0452340F26D1E64214FF4C870F8
:1087700012E062BB93FBF1F201FB123252BB03F237
:108780006C7C9CFBF0F200FB12C2002A14BF724604
:108790004FF4B772A41A013B9D4203F00302E8DBD9
:1087A000DAB9642295FBF2F302FB1353C3B94FF419
:1087B000C87205F26C7191FBF2F302FB1313002BEC
:1087C00040F26D1308BF4FF4B773E41A67E740F245
:1087D0006D12DFE74FF4B772DCE740F26D13F4E798
:1087E0004FF4B773F1E700F025FF00287FF477AF6F
:1087F000C1465BE0029BB3EB0C030893039B63EB66
:1088000001030993DDE908ABDDE90023524573EB71
:108810000B03EDDB7AE7DDE90401DDE900AB82451E
:108820007BEB010384DBB9F1000F43DB4FF001095F
:1088300088EA0908B8F1010F38D1B9F1000F55D015
:10884000AEEB0C03326830461A443260DDE90012A8
:10885000C91842EBE372CDE90012D6F80C80FFF79D
:10886000EBFDF268B2EB080220D0012A41DC901C3B
:10887000D8BF0122F3691444D31849D56A1E910761
:108880003AD1642192FBF1F301FB1323BBBB4FF4FC
:10889000C87205F26B7595FBF2F302FB1355002DC0
:1088A00040F26D1318BF4FF4B673F361B9F1010FC5
:1088B0007FF449AFDDE900AB4FF001093B6D1AEBE6
:1088C000030A4BEBE37B00F063FF0723043494FBC4
:1088D000F3F3C3EBC303E41A48BF0734C6F8209090
:1088E000B461504659460BB0BDE8F08FACEB0E03B7
:1088F000A8E74FF0FF32BDE74FF4B673D5E740F27B
:108900006D13D2E7D8D5000880510100600C00201B
:10891000AA0717D1642195FBF1F201FB1252A2B90B
:108920004FF4C87105F26C7595FBF1F201FB12551D
:10893000002D40F26D1208BF4FF4B7729342A8BFEA
:108940009B1AB2E740F26D12F8E74FF4B772F5E701
:108950004FF0FF3A4FF0FF3BC3E700BF2DE9F04176
:108960000F46904601F00EFF04460D46B8F1000F89
:1089700011D0C7F30A53C3F16B03002B0BDD0024A6
:108980001B0503F17F5505F5401522462B46F7F7E9
:108990008DFD04460D4620462946BDE8F0810000C5
:1089A0002DE9F04F1F460023A1B01C939C4B83463A
:1089B0001B680E46184617920493F7F7B3FB4FF067
:1089C000000804464FF000091B961B9A13780D2BE4
:1089D00032D8092B36D2002B3ED000230D931B9D9D
:1089E0002B78302B40F0AA806B78582B01D0782B55
:1089F00067D10D9B029701931CAB0093894A1DAB75
:108A00001BA9584601F0B2F810F00704064605D03D
:108A1000062C2BD1002301351B950D93179B002BA2
:108A200040F09D850D9BE3B1424609F1004310469D
:108A3000194621B0BDE8F08F2B2B06D02D2B13D07B
:108A4000202BCAD101321B92BFE700230D93531C88
:108A50001B935378002BC2D1179B1B96002B40F021
:108A60007C8542464B46E2E70123EFE71C9A3AB188
:108A700035211EA801F078FF1C99584601F0F0FB43
:108A8000013C042C06D8DFE804F00A0314170A009E
:108A9000DDE91E893107C1D549F00049BEE71D9ABD
:108AA000DDE91E8302F2334223F4801343EA0259C4
:108AB000F0E7DFF87491EDE76FF000494FF0FF3811
:108AC000E8E71B9B5A1C1B925B78302BF9D0002BDC
:108AD000A4D001234FF0000A0A22574605931B9B9E
:108AE000CDF818A008931B980578A5F13003D9B2EA
:108AF000092925D92246049902F074F870B30020A0
:108B00002B463C4602460490652B01D0452B13D1E1
:108B10001CB9059B03439FD000241B9E731C1B9311
:108B200073782B2B73D02D2B77D04FF0000CA3F143
:108B3000300109297ED91B9600259DE00023C9E755
:108B4000082FD8BF069900F10100D6BF02FB013300
:108B500002FB0A3A069301371B90C4E71B9B1A19C4
:108B60001B921B5D002F37D03C460490A3F13002CE
:108B7000092A12D90122C7E71B9B01305A1C1B92FC
:108B80005B78302BF8D0A3F13102082A00F2EC8494
:108B90000490002004461B9A0892303B00F1010229
:108BA00014D0049900EB040E1144049122460A21CA
:108BB000724513D12218082A04F1010404441CDC74
:108BC0000A22069902FB0133069300221B9B1046E2
:108BD000591C1B915B78C9E73846D2E7082A04DCA8
:108BE000069D4D4306950132E2E702F1010CBCF10E
:108BF000100FD8BF01FB0AFAF5E7102CDCBF0A22E0
:108C000002FB0A3AE1E700230122049381E74FF0D7
:108C1000000CB31C1B93B37889E74FF0010CF8E705
:108C2000A4D6000814D600080000F07F1B9B591C36
:108C30001B915B78302BF9D0A3F1310108293FF665
:108C40007BAF303B07931B9B09931B9B5D1C1B95C4
:108C50005B78A3F1300EBEF1090F31D909996D1A75
:108C6000082D44F61F6503DC07998D42A8BF0D4609
:108C7000BCF1000F00D06D42002C4ED1059901438C
:108C80007FF4CCAE002A7FF4E7AE4E2B25D01FDC5C
:108C9000492B7FF4E1AEA2491BA801F09DF9002801
:108CA0003FF4DAAE1B9B9F49013B1BA81B9301F0CD
:108CB00093F910B91B9B01331B93DFF88092ADE64B
:108CC0000A21079D01FB0535A5F130030793BCE799
:108CD000692BE0D06E2B7FF4BFAE93491BA801F047
:108CE0007BF900283FF4B8AE1B9B1B78282B0ED1D4
:108CF0001EAA8E491BA801F083F9052807D11F9BE6
:108D0000DDF8788043F0FF4949F4E00986E68848B9
:108D100001F01AFF8046894680E6049B002F08BFB9
:108D20002746EB1A102C069807932646A8BF102654
:108D3000F7F742FB092C8046894613DD7D4B03EB98
:108D4000C60353E91223F7F7B1FB80465046894624
:108D5000F7F732FB02460B4640464946F7F7F0F973
:108D6000804689460F2C36DC079B002B3FF456AE1D
:108D700022DD162B09DC6F4C424604EBC3044B4644
:108D8000D4E90001F7F792FBC4E7079AC4F1250381
:108D9000934220DB674DC4F10F0405EBC40142464A
:108DA000D1E900014B46F7F781FB079B1C1B05EB44
:108DB000C405D5E90023E5E7079B16330BDB049BCD
:108DC0005C4A5D1B02EBC505D5E9002340464946D8
:108DD000F7F796FC9EE7079BA4EB060A9A44BAF1C4
:108DE000000F75DD1AF00F030AD05249424601EB1D
:108DF000C301D1E900014B46F7F758FB804689468D
:108E00003AF00F0A52D0BAF59A7F27DD4FF0000AE8
:108E1000CDF810A0CDF820A0CDF818A022234FF057
:108E20000008DFF81891CBF80030089B002B3FF4C6
:108E3000F5AD1C99584601F013FA0699584601F011
:108E40000FFA0499584601F00BFA0899584601F0B8
:108E500007FA5146584601F003FADFE50023404681
:108E600049461E464FEA2A1ABAF1010F21DC0BB11E
:108E700080468946304BA9F1547903EBC606424639
:108E8000D6E900014B46F7F711FB2C4B0A460B4085
:108E90002B4980468B42B9D8A1F580118B4286BF01
:108EA0004FF0FF38DFF89C9002F1547900230593CE
:108EB00085E01AF0010F07D01F4B03EBC603D3E97F
:108EC0000023F7F7F3FA012301364FEA6A0ACBE7EA
:108ED000ECD0CAF1000A1AF00F020AD0154B404636
:108EE00003EBC2034946D3E90023F7F709FC8046A8
:108EF00089465FEA2A1AD9D0BAF11F0F24DD4FF054
:108F0000000ACDF810A0CDF820A0CDF818A022239B
:108F10004FF000084FF00009CBF8003085E700BFA4
:108F200008D600080BD6000811D6000828D600087D
:108F300034D8000848D7000820D700080000F07F88
:108F40000000A07CFFFFEF7F1AF0100318BF6A2318
:108F50004046059349460023B34E1AF0010F04D052
:108F6000D6E90023F7F7A2FA01235FEA6A0A06F1BD
:108F70000806F2D10BB180468946059BBBB1C9F307
:108F80000A53C3F16B03002B494610DD1F2B40F33E
:108F90002B81342BD8BF4FF0FF324FF00008CFBFEA
:108FA0004FF05C79203B02FA03F303EA0109002247
:108FB000002340464946F7F7E1FC00289FD1069B75
:108FC0003A46009308992346584601F09BF90890C9
:108FD00000283FF41BAF049B4FF0000A5D1B079B6A
:108FE000CDF810A0002BB4BF2B4600230E93079B97
:108FF00023EAE3731693089B5846596801F0FCF87E
:10900000069000283FF40AAF089B0C301A6903F160
:109010000C0102329200FFF7F9F91EAB01931DAB70
:10902000009342464B465846CDE90A8901F020FCA0
:109030001C9000283FF4F2AE0121584601F0F0F9EF
:109040000490034600283FF4E9AE1D9D1E9A002DB2
:10905000ABBF0E9B169BEE185C1B059BA8BF169C16
:10906000A5EB03051544714B05F1FF35B8BF0E9E06
:109070009D42C2F1360280F2C9805B1B1F2BA2EB1E
:1090800003024FF0010700F3B680002507FA03F34F
:109090000F93B718059BBE4214441C443346A8BF27
:1090A0003B46A342A8BF2346002BC2BFFF1AE41AC7
:1090B000F61A0E9B002B17DD1A460499584601F04C
:1090C00047FA049000283FF4A9AE01461C9A58467E
:1090D00001F0AFF9099000283FF4A0AE1C99584662
:1090E00001F0BEF8099B1C93002F00F39380079BAF
:1090F000002B08DD169A0699584601F029FA0690C9
:1091000000283FF48BAE002C08DD22460699584615
:1091100001F06CFA069000283FF480AE002E08DDC6
:1091200032460499584601F061FA049000283FF451
:1091300075AE069A1C99584601F0C5FA8246002879
:109140003FF46CAE0024C3680499C4600C9301F032
:10915000A0FAA04270DA0C9B53EA080340F0968014
:10916000C9F31303002B40F0918029F000431B0D3D
:109170001B05B3F1D66F40F28980DAF8143023B9B9
:10918000DAF81030012B40F3818051460122584615
:1091900001F02CFA0499824601F07BFA002875DD73
:1091A00005994B46224A002900F0918002EA090104
:1091B000B1F1D66F00F38B80B1F15C7F7FF7A7AE82
:1091C00000231C4A4046CDE914324946DDE9142308
:1091D000F7F76CF90B46034308BF22238046894604
:1091E00008BFCBF8003024E64FF0FF3202FA03F359
:1091F00003EA0808DBE6C5F17F4505F57F0505F5BF
:109200007B45E23507FA05F50F9742E70123002574
:109210000F933EE73A461C99584601F0E7F91C9037
:1092200000287FF464AFF9E540D6000802FCFFFF98
:109230000000F07F00005039CDF8249066D10C9AE0
:10924000C9F313035AB39C4A93422CD1059B404661
:1092500003B34B46994A4FF0FF311A40B2F1D46F35
:109260001BD8120DC2F16B0301FA03F398421AD115
:10927000934B099A9A4202D101303FF4CFAD4FF09F
:1092800000088E4B099A1A4002F58019059B002BA5
:1092900096D1CEE54FF0FF33E8E70B46E6E753EA19
:1092A00008033FF47DAFE5B1099B1D42EED00C9B56
:1092B000059A40464946C3B1FFF750FB02460B46AC
:1092C000DDE90A01F6F73CFF80468946DEE71340F8
:1092D000A3F580136FEA13594FF0FF386FEA09596D
:1092E000D4E70F9B13EA080FE0E7FFF737FB0246CE
:1092F0000B46DDE90A01F6F721FF00220023804634
:109300008946F7F73BFB0028C0D000E60499504699
:1093100001F0FCFA00224FF0804306460F46F7F7B3
:1093200041FB002875D00C9B002B47D00026654FD1
:10933000644D099B23F000431B0D1B050F930F9AEF
:10934000614B9A4240F0C880DDE90A23CDE914233D
:10935000099B4046A3F15479494601F013FA0246AD
:109360000B4630463946F7F7A1F842464B46F6F72A
:10937000E7FE0B465149554A1940914280465ED955
:109380000B9B02F15472934203D10A9B01333FF4C9
:1093900045AD4FF0FF38DFF828911C99584600F092
:1093A0005FFF0699584600F05BFF0499584600F0AD
:1093B00057FF5146584600F053FF1CE6B8F1000F26
:1093C00019D1099BC3F31303E3B900223D4B304687
:1093D0003946F7F7DDFAC8B900223D4B3046394629
:1093E000F7F764F804460D4605F100431894199305
:1093F000DDE918679DE7B8F1010F03D1099B002B48
:109400003FF485AD0026334F002491E70C9C304D8E
:10941000EAE72F4B002230463946F7F747F80C9B16
:1094200004460D4633B901F1004310901193DDE974
:1094300010677EE702460B46CDE91023F7E703F1FC
:109440005479059B002BA8D129F000431B0D0F9ADE
:109450001B059A42A1D12046294603F0FBF9F6F7F5
:10946000F7FF02460B4620462946F6F767FEC9F38A
:1094700013030C9A43EA0803134304460D4666D0CF
:1094800009A3D3E90023F7F783FA00287FF4D1ACCE
:1094900007A3D3E9002320462946F7F797FA0028C7
:1094A0003FF47BAFC5E400BF9535A094FFFFDF3FDD
:1094B00035E5AF350000E03FFFFF0F000000F07F13
:1094C000FFFFEF7F0000F03F0000E07FFFFF9F7C89
:1094D0000000E03F0000F0BF059B13B30F9BB3F10A
:1094E000D46F1ED826A3D3E9002320462946F7F7D8
:1094F00059FA90B129462046F7F7B0FA002808BF7C
:109500000120F6F759FF0C9B04460D46D3B901F133
:10951000004312901393DDE912670F9A07F1D663A7
:109520009F1ADDE90A0101F02DF902460B4630468B
:109530003946F6F7BBFFDDE90A23F6F701FE804660
:1095400089467EE702460B46CDE91223E3E70EA3E8
:10955000D3E90023F7F71CFAA1E700230D931B9B27
:10956000179A1360FFF75EBA652B3FF44CAB452B9F
:109570003FF449AB0122FFF781BB00BFAFF300808E
:109580000000C0FFFFFFDF419535A094FFFFCF3FF4
:109590002DE9F041224E0A46224B01463068FFF782
:1095A000FFF902460B4605460C46F7F719FA68B173
:1095B000002C1D4806DA01F0DDFA00F100473846BC
:1095C000BDE8F081BDE8F04101F0D4BA214628465B
:1095D000F7F764FA20F00048074614494046F7F7C9
:1095E00081FD0028EBD111494046F7F75DFD0028C9
:1095F000E5D124F000444FF0FF320D4B28462146C0
:10960000F7F7EEF940B94FF0FF32094B28462146F3
:10961000F7F7C8F90028D2D0222233681A60CEE7C3
:10962000800100204C02002034D80008FFFF7F7F1B
:10963000FFFFEF7F2DE9F74F804600F0B3FD40F2CA
:10964000B173984540F397806FF4F66340F26D1262
:1096500043449B10A8F2B27502FB05356FF063021C
:10966000A8F26D7393FBF2F36FF4C8621D444FF4DC
:10967000C8734244B2FBF3F298FBF3F7154464223B
:1096800003FB178798FBF2F6B7FA87FC04464FF006
:10969000070E02FB168608F00303C0F804804FEAA9
:1096A0005C1C00F1500B0093227A63694A2A28D18E
:1096B0000099EA1801B906B90FBB3B2BD4BF0023B0
:1096C000012313445A1EA3692C49283401FB02329A
:1096D000236813441A46DB1744E90223A345E3D168
:1096E000D0E90845D0E91223944275EB0303B4BFD7
:1096F000012300230360012003B0BDE8F08F0023A5
:10970000DFE7442A01D1EA18DDE7009A6ABB002EA0
:109710000CBFE0464FF001084FF0300AE2684FF00E
:10972000000901922A4616490AFB0818A8F1040804
:10973000019909F10109494558F829A017DC02F1FE
:10974000040898FBFEF9C9EBC909A8EB0909B3EBBA
:109750000909236948BF09F10709013BC3EBC303AA
:109760004B44534505DA1A44ADE7E046D4E752448A
:10977000DEE7073BF5E70020BEE700BF80510100B0
:10978000BCD60008014800F011BD00BFD721002061
:10979000014800F00DBD00BFD7210020014B186823
:1097A00000F002B8800100202DE9F04F8DB007468F
:1097B00000F0F8FCAF490546384600F0EBFCAE4E31
:1097C000044670B9AD4BAE4A1860AE4B1860AE4B54
:1097D0003068C3E9002200F0F5FC34600DB0BDE84C
:1097E000F08F316800295FD1306800F0EBFC204633
:1097F000F6F798FC411C384601F04CF9306000281F
:1098000057D123780AAE3A2B08BF013433469F4A1A
:109810009F49204601F0B2F90028DFDD0A9BE718D6
:10982000E35C2D2B49D14FF0FF3401374FF0000896
:109830000DF1200A0DF11E0B0396CDE9016ACDF85A
:1098400000B0334607AA93493846ADF81E80ADF8FC
:10985000208001F093F94045C0DD3C21BDF81E3069
:10986000BDF82020DFF8389201FB03224FF461613C
:10987000BDF81C3001FB03235C43844BAC62824C7B
:109880004A4623600A9B82491F443846334601F00A
:1098900075F9404516DC2368AA6A6360774B1A6045
:1098A000784BC3F8008099E7F6F732FC00289BD18B
:1098B00094E7214601F08EF9A3E72B2B08BF01376F
:1098C0000124B3E70A9BC4F80490FC18FB5C2D2B21
:1098D00040F08C804FF0FF3701340023CDE902A621
:1098E000ADF81C30ADF81E30ADF820300A93CDE94C
:1098F00000B6334607AA6749204601F03FF9002821
:1099000079DCAF6AA7F561672F654FF000092F4634
:109910000A9B1C4423782C2B08BF013494F8008048
:10992000B8F14D0F79D10DF12603CDE9016309ABF3
:109930000093039633460DF122025749204601F069
:109940001DF903287FF44AAFBDF822104B1E0B2BE4
:109950003FF644AFBDF82420531E042B3FF63EAF24
:10996000BDF82630062B3FF639AFC7E9031287F85A
:1099700008807B610A9B04EB03080223ADF81C30CE
:109980000023ADF81E30ADF820300A9398F800306F
:109990002F2B09D1CDE902A6CDE900B6334607AA9F
:1099A0003E49404601F0EAF83C21BDF81E30BDF8C2
:1099B0002020283701FB03224FF46161BDF81C30E1
:1099C00001FB032347F8103C0A9C4444B9F1000F03
:1099D00020D06868FFF72EFEAA6A284B1A602B6D0C
:1099E0009B1A18BF0123274A1360F7E62B2B08BFE9
:1099F0000134012771E73C21BDF81E30BDF820205D
:109A000001FB03224FF46161BDF81C3001FB03230D
:109A10005F4379E74FF001097CE7B8F14A0F0ABFCD
:109A20004346442301340A220BA92046059301F042
:109A300063F9DDF82C80ADF82600A045059B14D114
:109A40004D23B9F1000F07D12B7203210223C5F872
:109A50001490C5E9031390E785F830300B220123F9
:109A6000C5E90D230023EB6387E780B23B72786181
:109A700083E700BF68D600085C0C0020640C00205F
:109A80006BD60008600C0020E40100204F0C002081
:109A90006FD6000892D600087ED6000891D600083E
:109AA000440C002010B591FBF2F4002902FB1413C2
:109AB00006DB002B01DA01349B1AC0E9004310BD1C
:109AC000002BC4BF04F1FF349B18F6E7F0B506691C
:109AD0004B119E4200F1140431DD11F01F0104EB23
:109AE000860604EB830208D12146B2420B4611D20E
:109AF00052F8043B41F8043BF7E754F8235023465F
:109B0000C1F1200CCD400432964217460DD81D609D
:109B100005B10433A342A3EB040208BF00234FEABC
:109B2000A202026108BF4361F0BD3F6807FA0CF76B
:109B30003D4343F8045B52F8045BCD40E4E7234621
:109B4000E8E7A0F13003092B02D82038C0B27047F3
:109B5000A0F16103052B01D84738F7E7A0F14103D5
:109B6000052B01D82738F1E7002070472DE9F04F89
:109B70008BB00693B74B02901B688B4618469046F5
:109B80000393F6F7CFFA039BDBF80020034413F8A6
:109B9000013C01900793931CC2F1FF2202F57F0262
:109BA000FE3202EB030A1F4613F8010B3028F8D0EF
:109BB000FFF7C7FF0446002867D1019A039938468A
:109BC00001F010F8002863D1019BF85CFE18FFF744
:109BD000B8FF00285FD0334618781F46302803F1BD
:109BE0000103F9D0FFF7ADFFB0FA80F534464FF02E
:109BF000010A6D093A46164630780132FFF7A1FF97
:109C00000028F8D1019A0399304600F0EBFF50B9D3
:109C100054B9019BF4182246164630780132FFF7FA
:109C200090FF0028F8D10CB1A41BA4003378502B6E
:109C300001D0702B3DD173782B2B2ED02D2B30D013
:109C40004FF00009711C0878FFF77BFF431EDBB261
:109C5000182B2ED8A0F1100211F8010FFFF771FF99
:109C6000431EDBB2182B1FD9B9F1000F00D05242AE
:109C70001444CBF80010F5B1BAF1000F14BF00275F
:109C8000062738460BB0BDE8F08F00252C46B1E71B
:109C90003E460125CAE70446FBE74FF00009B11C28
:109CA000D1E74FF00109FAE70A2303FB0202103A59
:109CB000D2E73146DDE72946F31B013B072B4FDC9A
:109CC000029800F099FA4FF0000B0546DA46019B26
:109CD00000F11409C3F10103CDF810900893B742C5
:109CE00041D3049840F804ABA0EB09008010286130
:109CF0004701504600F044FBD8F800603F1AB742D5
:109D000063DDBF1B3946284600F048FE8246A8B1F5
:109D10004FF0010A7B1E591103F01F0259F8211060
:109D20000AFA02F20A4209D0534505DDB91E284657
:109D300000F034FE002845D14FF0020A394628468B
:109D4000FFF7C4FE3C44D8F80830A3424BDA29465A
:109D5000029800F085FA0023149AA327136090E775
:109D600001315B10AAE7731E0593079A16F8013CB0
:109D7000934217D0BBF1200F06D1049B43F804ABEC
:109D80004FF0000AD346049316F8010CFFF7D9FEF2
:109D900000F00F0000FA0BF04AEA000A0BF1040B86
:109DA000059B0DE0059B089A1344BB42E2D318467D
:109DB000019A0399099300F015FF099B0028D9D156
:109DC0001E468CE74FF0030AB8E709DAF71B29466D
:109DD0003A46029800F00AFC0546E41B00F114091B
:109DE0004FF0000AAFE7D8F80400A0426EDD041B74
:109DF000A64231DCD8F80C30022B22D0032B24D021
:109E0000012B15D1A64213D1012E0BD1D8F8043065
:109E1000069A6227136001232B61C9F80030149B56
:109E20001D602EE7711E284600F0B8FD0028EDD118
:109E30002946029800F014FA0023149A5027136060
:109E40001FE7159B002BF3D1E0E7159B002BDDD11D
:109E5000EEE700BFA4D60008671EBAF1000F32D1AA
:109E600027B13946284600F099FD824601237A1130
:109E700007F01F0703FA07F759F8223021461F425F
:109E80004FF00207284618BF4AF0020A361BFFF7B8
:109E90001DFED8F80440BAF1000F48D0D8F80C30B5
:109EA000022B15D0032B17D0012B09D11AF0020F6A
:109EB00006D0D9F800304AEA030A1AF0010F0ED191
:109EC00047F0100733E04FF0010ACFE70127E2E740
:109ED000159BC3F101031593159B002BF0D04FF098
:109EE000000CD5F8109005F114034FEA890A03EB32
:109EF0000A01184653F8042BB2F1FF3F1CD001327F
:109F00000260022F05F1140338D1D8F80020013A7D
:109F1000B2420AD10122711153F8213006F01F0616
:109F200002FA06F61E4218BF174647F02007149B98
:109F30001D60069B1C60A4E6994243F804CCD8D867
:109F4000AB68994512DB69680298013100F054F959
:109F500083462A6905F10C01023292000C30FEF7AB
:109F600055FA2946029800F07BF95D462B695A1C88
:109F70002A61012205EB83035A61C2E72A694A4537
:109F80000BDD01212846FFF7A1FDD8F80830013488
:109F9000A342FFF6DCAE0127C7E716F01F06FAD092
:109FA0009A445AF8040C00F0EBF9C6F12006B042CE
:109FB000E7DBF0E7C2F10802920070B5C2F12006BB
:109FC0004368046803FA06F52C43D340046040F864
:109FD000043F8842F4D370BD30B50368013311F8F3
:109FE000014B14B90360012030BD13F8012BA2F11D
:109FF0004105192D98BF2032A242F0D00020F3E78E
:10A000002DE9F04F00250B6882465F1102EB8707B0
:10A0100013F01F0318BF04373E1F9046B146344665
:10A02000AB4687B00168019347F8045C02954A7813
:10A030004B1C039342B3104605910492FFF781FD38
:10A04000002843D1049A0599202A18D8029B9B45E1
:10A0500013DD4C4506D2072D04DC2A46494620462E
:10A06000FFF7A8FF444544D90023A4F1040944F8AC
:10A07000043C1D464C46CDF808B00399D7E7292A81
:10A080004AD10231CAF80010BBF1000F44D04C4550
:10A0900006D2072D04DC2A4649462046FFF78AFFF0
:10A0A000444528D9434654F8042BA64243F8042BD0
:10A0B000F9D2002243F8042B9E42FBD233681BB92D
:10A0C000464527D101233360052026E00135082DC0
:10A0D0000BF1010B06DD4445CFD90023012544F8DF
:10A0E000043C043C226800F00F0040EA02102060AB
:10A0F000C3E70825C1E7019B002BDFD04FF0FF32FB
:10A10000C3F1200322FA03F357F8042C1A4047F84E
:10A11000042CD3E7043ED1E7042007B0BDE8F08F5C
:10A120002DE9F84F06468A46174600F0FDFD184B0C
:10A130001C68994634B15346984613F8012B3AB13E
:10A140003D2AF9D1304600F0F5FD0020BDE8F88F3A
:10A15000A8EB0A08A34654F8040B0028F2D04246A4
:10A16000514600F03FFD0028F4D154F8043C03EBC5
:10A17000080513F808303D2BECD1D9F800303046F3
:10A18000ABEB03039B103B6000F0D4FD681CDDE7E4
:10A19000B803002007B501AAFFF7C2FF03B05DF8BE
:10A1A00004FB000000487047F00100207047704732
:10A1B00070477047024B0146186800F06BBC00BF47
:10A1C00080010020024B0146186800F017BC00BF58
:10A1D0008001002082B001B901A942B14BB11378CE
:10A1E0000B601278101C18BF012002B07047104697
:10A1F000FBE76FF00100F8E770B5456A04460E46CC
:10A200003DB91020FFF7D6FFC0E901556062056037
:10A21000C560656AEB6883B1636ADB6853F8260042
:10A22000B8B9012101FA06F56A1D9200204600F036
:10A23000D6FB60B1C0E901650EE021220421204671
:10A2400000F0CDFB636AE860DB68002BE4D10020FE
:10A2500070BD026843F826200023C0E90333F7E706
:10A2600070B5446A06460D463CB91020FFF7A2FFC0
:10A27000C0E9014470620460C4603DB1736A6A68F9
:10A28000DB6853F82210296043F8225070BD2DE995
:10A29000F0411F4606460C4600230D6901F1140CDF
:10A2A000DCF80000013381B202FB0171000C0F0CDD
:10A2B00002FB007089B201EB00419D424FEA10475A
:10A2C0004CF8041BECDCD7B1A368AB4212DC61682C
:10A2D00030460131FFF790FF8046226904F10C01FE
:10A2E000023292000C30FEF791F821463046FFF71B
:10A2F000B7FF444604EB850301355F6125612046C5
:10A30000BDE8F0812DE9F843154609221F460833C0
:10A310000C4693FBF2F30646012200219A4220DB11
:10A320003046FFF769FF089B092D43614FF0010399
:10A33000036119DD04F10909C8462C4418F8013BF2
:10A340000146303B0A223046FFF7A1FFA045F5D178
:10A35000A5F108044C442D1B6319BB4207DBBDE883
:10A36000F88352000131D9E70A340925F3E714F8DC
:10A37000013B0146303B0A223046FFF788FFEBE7FE
:10A38000020C12040346CAB90304102013F07F4FD5
:10A3900004BF1B02083013F0704F04BF1B010430D0
:10A3A00013F0404F04BF9B000230002B05DB13F07D
:10A3B000804F00F1010008BF202070470020E5E732
:10A3C0000368014613F007020BD0DA0724D498077C
:10A3D00049BF5B089B0801200B605CBF0B6002203B
:10A3E000704798B2B0B910201B0C13F0FF0F04BFD8
:10A3F0001B0A08301A0704BF1B0904309A0704BF60
:10A400009B080230DA0703D45B0800F1010005D095
:10A410000B6070471046E8E7002070472020704727
:10A4200010B50C460121FFF7E7FE012244610261ED
:10A4300010BD2DE9F74F90460A69D8F810300C4648
:10A440009A42BEBF0B46444698462769D8F81090FA
:10A45000A368616807EB0906B342B8BF0131FFF793
:10A46000CBFE00F114052B46002205EB860E73454A
:10A4700016D304F1140308F1140203EB870702EB6F
:10A4800089030093009B019293420CD8002E03DDB8
:10A490005EF8043D002B59D0066103B0BDE8F08F93
:10A4A00043F8042BE3E7B2F800A0BAF1000F23D081
:10A4B000AC464FF0000804F1140959F8041BDCF80D
:10A4C00000B08BB21FFA8BFB0AFB03B34FEA114BB0
:10A4D000DCF8001043444FEA11480AFB0B8101EB02
:10A4E00013419BB243EA01434F454FEA11484CF8F0
:10A4F000043BE2D8CCF80080019B0432B3F8029010
:10A50000B9F1000F20D0AC464FF0000A2B6804F1DF
:10A510001408B8F80010BCF802B09BB209FB01B1F6
:10A520008A4443EA0A434CF8043B58F8043BBCF81D
:10A5300000101B0C09FB0313474503EB1A434FEABA
:10A54000134AE6D8CCF8003004359BE7013E9DE77E
:10A550002DE9F843154612F0030206460F4607D0D0
:10A56000214C013A002354F82220FFF790FE0746C1
:10A57000AD1035D0746A3CB91020FFF71BFEC0E95E
:10A58000014470620460C460D6F82480D8F80840A2
:10A590004CB940F271213046FFF742FF00230446D8
:10A5A000C8F8080003604FF00008EB070AD53946E9
:10A5B00022463046FFF73DFF814639463046FFF7D9
:10A5C0004FFE4F466D100BD0206838B92246214609
:10A5D0003046FFF72EFF2060C0F800800446E4E715
:10A5E0003846BDE8F88300BF10D800082DE9F047D1
:10A5F0000C460746164623694FEA621A0AEB03091E
:10A600004968A36809F10105AB4233DB3846FFF71F
:10A61000F3FD0023804600F1140100F110021846FA
:10A6200053452ADB20692AEAEA7A04F1140316F07A
:10A630001F0201EB8A0103EB800C22D00020C2F143
:10A64000200E1E689640304341F8040B53F8040B6B
:10A650009C4520FA0EF0F4D8086008B109F1020513
:10A66000013D3846C8F810502146FFF7F9FD404635
:10A67000BDE8F08701315B00C6E742F8040F013303
:10A68000CEE7043953F8042B9C4541F8042FF9D840
:10A69000E6E703690A6930B59B1A0CD192001430C1
:10A6A00014318418114454F8045D51F8042D954276
:10A6B00003D005D30123184630BDA042F3D3FAE7F7
:10A6C0004FF0FF33F7E72DE9F0470D4607461146F7
:10A6D00028461446FFF7DDFF061E08D131463846EE
:10A6E000FFF78AFD0123C0E90436BDE8F087A4BF67
:10A6F00023462C4638466168A6BF1D460026012623
:10A70000FFF77AFD4FF0000EC6602B69266904F151
:10A71000140205F1140902EB860709EB830800F126
:10A72000140152F804AB59F8045B1FFA8AF373441E
:10A73000ACB21B1B2C0CC4EB1A4404EB23449BB29D
:10A740004FEA244EC84543EA0444944641F8044B7A
:10A75000E7D8BC4504D351F8043D83B10661C4E792
:10A760005CF8044BA2B27244131403EB144392B28C
:10A7700042EA03424FEA234E41F8042BE9E7013E47
:10A78000E9E700000F4B0B40A3F15073002B02DDF3
:10A790000020194670475B421B15132B4FF0000039
:10A7A0004FF0000104DC4FF4002242FA03F170473D
:10A7B000143B1E2BD6BF4FF00042012322FA03F3B5
:10A7C000184670470000F07F2DE9F843076900F153
:10A7D000140909EB870757F8046CA7F10408304601
:10A7E000FFF7CEFDC0F120030A280B601F4917DCDC
:10A7F000C14528BF0022C0F10B0C26FA0CF338BF6C
:10A8000057F8082C43EA010500F1150306FA03F393
:10A8100022FA0CF243EA020420462946BDE8F883F6
:10A82000C1453ABFA7F1080857F8082C0022B0F13B
:10A830000B0316D0C3F1200722FA07F1C84506FA28
:10A8400003F646EA010694BF002158F8041C46F0BE
:10A850007F5502FA03F0F94045F4401540EA01043F
:10A86000DAE746EA01051446D6E700BF0000F03FEC
:10A870002DE9F3411C46DDE9086501219046FFF70B
:10A88000BBFCC4F31302C4F30A5407462CBB019269
:10A89000B8F1000226D068460092FFF791FD0099BA
:10A8A000F0B1019AC0F1200302FA03F30B43C24056
:10A8B0007B610192019B002B14BF02210121BB612E
:10A8C0003961C4B1A4F2334404443460C0F13500AA
:10A8D0002860384602B0BDE8F08142F48012D6E725
:10A8E0007961E7E701A8FFF76BFD0121019B396161
:10A8F0007B612030E5E7A0F2324007EB8103306056
:10A900001869FFF73DFDC0EB4110E1E72DE9F74F76
:10A91000884669468146FFF757FF8B4606460F4635
:10A92000404601A9FFF750FFD9F81030D8F81020A1
:10A930000D46A3EB020CDDE900329B1A03EB4C132E
:10A94000002BD5BF0A463A46C3EB033302EB035B49
:10A95000D8BF02EB03552B46024659463046F5F761
:10A96000CFFE03B0BDE8F08F013910B5491114696D
:10A97000013102F1140300EB810103EB8404A342D3
:10A98000024603D300238A4205D310BD53F8042B9B
:10A9900040F8042BF3E742F8043BF4E700F114021B
:10A9A00000694B11984210B511DB0ADD11F01F014F
:10A9B00007D052F8234024FA01F000FA01F18C424A
:10A9C0000BD102EB8303934203D8002010BD034652
:10A9D000F7E753F8041D0029F5D00120F6E738B554
:10A9E00002FB01F4214600F055F8054618B1224655
:10A9F0000021FDF719FD284638BD000038B5054691
:10AA0000002943D051F8043C0C1F002BB8BFE418B8
:10AA100000F096F91E4A1368104633B9636014605B
:10AA20002846BDE8384000F091B9A3420BD921680F
:10AA30006218934201BF1A685B6852182260636013
:10AA40000460EDE713465A680AB1A242FAD91968C0
:10AA50005818A0420BD1206801445818824219604E
:10AA6000DED110685268014419605A60D8E702D9F3
:10AA70000C232B60D4E7206821188A4201BF11689B
:10AA800052680918216062605C60C9E738BD00BF88
:10AA9000680C0020F8B5CD1C25F0030508350C2DF9
:10AAA00038BF0C25002D064601DBA94203D90C2333
:10AAB00033600020F8BD00F043F921490A681446CC
:10AAC0009CB9204F3B6823B92146304600F042F83C
:10AAD00038602946304600F03DF8431C23D10C2352
:10AAE0003046336000F032F9E3E723685B1B17D48C
:10AAF0000B2B03D923601C44256004E06368A24249
:10AB00000CBF0B605360304600F020F904F10B00DD
:10AB1000231D20F00700C21ACCD01B1AA350C9E78E
:10AB200022466468CCE7C41C24F00304A042E3D0AE
:10AB3000211A304600F00EF80130DDD1CFE700BF1A
:10AB4000680C00206C0C002000200149704700BFF9
:10AB50000000F87F38B50023054C05460846236001
:10AB600001F068FE431C02D1236803B12B6038BD9D
:10AB7000DC210020004870470000C07F0EB44FF475
:10AB8000017230B59CB01FAC54F8045BADF81420D2
:10AB900002900690F5F7C6FA0B4B03900B93002337
:10ABA0000F9314934FF6FF7307900848ADF81630D3
:10ABB0002A46234602A90068019400F027F91CB038
:10ABC000BDE8304003B07047D1AB000880010020E1
:10ABD00000207047034611F8012B03F8012B002ACF
:10ABE000F9D1704710B56AB10139841810F8013BEA
:10ABF00011F8012F934203D1A04201D0002BF5D1CF
:10AC0000981A10BD1046FCE72DE9F0438646084629
:10AC1000374F054615F8014BE65D16F0080631D1B1
:10AC20002D2C31D14FF001082C78851C002B5AD0E7
:10AC3000102B09D1302C07D1287800F0DF005828DC
:10AC40004CD110236C7802354FF0FF3CBCFBF3FC79
:10AC5000002603FB0CF930466FEA0909A4F130071E
:10AC6000092F18D83C46A34224DD002E1FDB844563
:10AC70001DD301D1A1451ADB012600FB034015F8C5
:10AC8000014BEBE72846C4E72B2C08BF2C78B046D5
:10AC900008BF851CCAE7A4F14107192F01D8373C2A
:10ACA000E1E7A4F16107192F04D8573CDBE74FF027
:10ACB000FF36E4E7002E07DA22234FF0FF30CEF80C
:10ACC000003042B9BDE8F083B8F1000F00D0404237
:10ACD000002AF7D006B1691E1160F3E73024002B7B
:10ACE000B2D10823B0E7302CA6D00A23ACE700BFCE
:10ACF000A1D40008FFF788BF13460A460146024860
:10AD00000068FFF781BF00BF8001002049B1FF2A22
:10AD10008BBF8A230A700360012088BF4FF0FF3089
:10AD200070470846704700000148FFF740BA00BF6F
:10AD3000D22100200148FFF73CBA00BFD2210020F9
:10AD40000148FFF734BA00BFD42100200148FFF7C3
:10AD500030BA00BFD421002038B54B1C144603D1B3
:10AD60004FF0FF35284638BD9389CDB223F020033C
:10AD70009381636B52688BB1A36B934208DD2368A8
:10AD80005A1E226003F8015C636801336360E9E7DF
:10AD9000214600F079FB0028F1D0E1E72169236822
:10ADA00051B1994208D213F8011CA94204D1013BC8
:10ADB000013223606260D5E7C4E90F3204F1440335
:10ADC00063630323A363234603F8465F23600123E1
:10ADD000DCE710B50C46496B69B104F144039942B4
:10ADE00001D0FFF70BFE0020236C6063636013B19A
:10ADF000E36B236010BD23694FF0FF302360002315
:10AE00006360A38943F02003A381F3E72DE9F04FAA
:10AE10000C4600210646ADF5237DCDE944119A4943
:10AE20000DF10408A0919949994FDFF86892CDF887
:10AE30001881A191009392F800A0BAF1000F00F0E0
:10AE400021811AF80730551C13F0080319D06368E4
:10AE5000002B0FDD23681A78BA5C120701D42A464A
:10AE6000E9E7459A01330132459262682360013A6D
:10AE70006260ECE7A19B2146304698470028E9D064
:10AE8000EDE7BAF1250F7FD14193439353782A2BF5
:10AE900004BF1023951C4FF00A0208BF4193AB4634
:10AEA0001BF8011BA1F13003092B21D9032279489A
:10AEB00000F022FB38B1A0EB090301205D46984069
:10AEC000419B1843419015F8013B672B48D8652BEF
:10AED00080F09E80472B12D8452B80F09980002B64
:10AEE0006BD0252B50D0032347930A23429316E0BF
:10AEF000439B5D4602FB0313303B4393CFE75B2B41
:10AF000067D027D8582BEED1419A42F40072419273
:10AF100010226F2B34BF03230423429247936368AC
:10AF2000002B77DD419B590604D423681A78BA5C5C
:10AF3000120776D4479B022B00F386806B4622468D
:10AF400041A9304600F0AAF8012800F09B800228B1
:10AF500085D12FE0632B47D0642BC4D10A22D8E7D8
:10AF6000702B2DD008D86E2B44D02ED8692BBAD197
:10AF7000002342930323D1E7752BEFD0782BC3D066
:10AF8000732BB0D10223C9E76368002B0CDD236863
:10AF90001A78524576D1013362682360459B013AA5
:10AFA0000133626045935AE7A19B2146304698479A
:10AFB0000028ECD0449800285AD14FF0FF305DE0D3
:10AFC000419A42F0200241929EE7082342930423D3
:10AFD000A4E72946404600F0ABF9419B054643F003
:10AFE00040034193012399E7419B43F04003419380
:10AFF000002393E74198C3063FF531AF009B459A84
:10B00000191D00911B68C0074CBF1A801A6026E703
:10B01000052383E7A19B214630469847002881D02D
:10B02000C8E7459A013245926268013A002A626097
:10B0300002DD0133236078E7A19B21463046984723
:10B0400000283FF472AFB5E7042B06DC6B462246BE
:10B0500041A9304600F07AF876E70F4B002B3FF419
:10B06000FEAE6B46224641A93046AFF300806BE747
:10B07000A38913F0400F18BF4FF0FF300DF5237D6B
:10B08000BDE8F08F4498F9E759AD0008D3AD00084A
:10B09000A1D400081CD80008000000002DE9F843E6
:10B0A00015468A6880460C4632B98A69002A0CBF68
:10B0B00001224FF0FF328A6000272268DFF8889073
:10B0C000D1065FBF1A68111D19601668A06988B1A2
:10B0D000012807D12B681A7863699B5C53B927BB99
:10B0E000BDE8F883022820D12B681B7813F80930BB
:10B0F0001B071AD423680137DA065EBF2B681B785A
:10B1000006F8013B2A686B6801322A60A268013B9D
:10B11000013A6B60A26042B1002BD7DCD4F88031D9
:10B120002946404698470028D0D0236813F01003E2
:10B1300005D1E2680132E260A26902B1337023698D
:10B1400000201F442761CBE7A1D400082DE9F04F70
:10B150000C469946724B87B08246164693E8070024
:10B1600003AB83E807006F4BA1696F4A27460329A9
:10B1700018BF1A46A36801925A1EB2F5AE7F81BF6E
:10B180006FF4AE7503EB050840F25D13A36057F84A
:10B190001C3B98BF4FF000083D464FF0000B43F4B6
:10B1A00050632360316803AB0222097853F82B0007
:10B1B00000F0A2F928B3BBF1010F59D162682AB996
:10B1C00008232268636042F400722260226822F43D
:10B1D000A0622260A268511EA16092B13268511C27
:10B1E0003160127805F8012B7268013A002A72600A
:10B1F00007DCD4F88021314650469047002840F0C3
:10B2000085800BF1010BBBF1030FCBD163680BB948
:10B210000A236360636845496069C91A00F088F8C9
:10B220004FF0000BA3682268002B3DD031686069A5
:10B2300091F800C010F80C00002835D0BCF1300F98
:10B2400024D1100522D50BF1010BB8F1000F03D06A
:10B25000013308F1FF38A3607368013B002B736072
:10B260001BDD336801333360A368013BA360D9E77A
:10B27000BBF1020FAED1226802F4C061B1F5007FCC
:10B28000BFD1102342F480726360A2E722F41062FF
:10B2900022600B7805F8013BDEE7D4F880313146B7
:10B2A000504698470028DFD02368D9050DD5BD4208
:10B2B00009D915F8011C05F1FF38D4F87C31324664
:10B2C000504698474546BD4228D0226812F01002E9
:10B2D00013D12A70636839465046019EB047D9F8A9
:10B2E000003021681A1DC9F8002011F0200F1B68DA
:10B2F0000FD01860E3680133E3600020ED1BAB441E
:10B3000025695D44256107B0BDE8F08F4FF0000B63
:10B31000CAE7CA074CBF18801860EBE70120F2E7C4
:10B3200014C90008F5AC000885B4000830D800083E
:10B3300070B50B78441E5E2B13BF4A1C8A1C4B78D9
:10B34000002108BF012100F1FF0504F8011FAC42F4
:10B35000FBD113B9013A104670BD81F00104C45409
:10B36000511C11F8015C4E1E2D2D0A4606D05D2D94
:10B37000F1D00DB93246EEE72B46F0E70E785D2EA0
:10B38000FAD0B342F8DC01339E42C454FBDC0231F4
:10B39000E7E700002DE9F04786460846384F0546A6
:10B3A00015F8014BE65D16F0080634D12D2C34D18A
:10B3B0004FF001082C78851C002B5CD0102B09D194
:10B3C000302C07D1287800F0DF0058284ED1102308
:10B3D0006C780235B8F1000F14BF4FF0004C6FF0DD
:10B3E000004C0027BCFBF3F9384603FB19CAA4F153
:10B3F0003006092E18D83446A34224DD7E1C07D01F
:10B4000081451DD301D1A2451ADB012700FB034072
:10B4100015F8014BEBE72846C1E72B2C08BF2C7829
:10B42000B04608BF851CC7E7A4F14106192E01D814
:10B43000373CE1E7A4F16106192E04D8573CDBE75D
:10B440004FF0FF37E4E77B1C06D122236046CEF89D
:10B45000003042B9BDE8F087B8F1000F00D040429B
:10B46000002AF7D007B1691E1160F3E73024002BE2
:10B47000B0D10823AEE7302CA4D00A23AAE700BF3E
:10B48000A1D40008FFF786BF2DE9F0410C46496BB7
:10B4900004F1440399421BD14FF48061FFF7FAFA9B
:10B4A00018B94FF0FF30BDE8F0814FF48063A3631B
:10B4B00094F84630606380F8FF3394F8453000F22A
:10B4C000FD30437094F84430037020600020EAE7B8
:10B4D000A66B77003A4600F01DF805460028E0D03C
:10B4E00000EB0608014632464046FCF78FFFC4F8E1
:10B4F0000080C4E90D57E9E710B5C9B20244904293
:10B50000034601D1002303E01C7801308C42F6D1C0
:10B51000184610BDF8B5074614460E4621B9114627
:10B52000BDE8F840FFF7B6BA22B9FFF767FA25463B
:10B530002846F8BD00F014F8A0420FD22146384644
:10B54000FFF7A8FA05460028F2D031462246FCF75C
:10B550005DFF31463846FFF751FAE9E73546E7E740
:10B5600051F8043C181F002BBCBF0B58C018704783
:10B5700030B5214A21F00043934287B01BDD1F4ABA
:10B58000934205DD02460B46F4F7D8FD07B030BD07
:10B5900002AA00F035F800F00300012813D00228B9
:10B5A0001FD0DDE90423A8B1DDE9020100F044FA6F
:10B5B00001F10041EAE7002400220023009400F09A
:10B5C0007FFF07B030BDDDE90423DDE9020100F0B3
:10B5D00033FADBE70124DDE90201009400F070FF9B
:10B5E000D4E70124DDE90423DDE90201009400F041
:10B5F00067FF01F10041C9E7FB21E93FFFFFEF7F52
:10B600002DE9F04FBE4C21F00045A5428FB040F32C
:10B6100082801446BB4A0E46954226DCAEA3D3E98F
:10B620000023002940F3B381F4F788FDB64B0646AA
:10B630009D420F4600F08480A9A3D3E90023F4F7CC
:10B640007DFD02460B4630463946C4E90023F4F737
:10B6500075FDA3A3D3E90023F4F770FD0127C4E926
:10B66000020138460FB0BDE8F08FA84A954240F37A
:10B670008780A74A954259DC2F15A7F21647A5EBFC
:10B68000075189468046F5F7C1F9F4F7A5FE8246D1
:10B690008B464046494652465B46CDE908ABF4F737
:10B6A0004DFD00229B4BF4F701FF89468046F5F7DC
:10B6B000ADF90546F4F790FE02460B464046494672
:10B6C000CDE90A23F4F73AFD0022924BF4F7EEFE9F
:10B6D00000220023CDE90C01F5F750F9002800F015
:10B6E000F680002D0CBF0123022302208A493A462E
:10B6F000CDE90001214608A800F0C2FA002E074655
:10B70000AFDA6268E36802F1004203F100434742A6
:10B710006260E360A5E7002700240025C2E900017C
:10B720003846C2E902450FB0BDE8F08F02460B462D
:10B73000F4F704FD0027C4E90201C4E9000190E721
:10B7400069A3D3E90023F4F7F9FC69A3D3E9002343
:10B7500006460F46F4F7F2FC02460B463046C4E9B3
:10B7600000233946F4F7EAFC61A3D3E90023F4F798
:10B77000E5FC0127C4E9020138460FB0BDE8F08FAF
:10B7800000F054FF5CA3D3E9002380468946F4F718
:10B790008DFE0022614BF4F7D3FCF5F737F907462D
:10B7A000F4F71AFE4CA3D3E9002382468B46CDE979
:10B7B00004ABF4F77BFE02460B4640464946F4F7DD
:10B7C000BDFC47A3D3E90023CDE902015046594609
:10B7D000F4F76CFE1F2F8046894602460B46DDE9D2
:10B7E000020128DCF4F7AAFC4D4B7A1E53F82230F4
:10B7F0008346AB428A4622D05A465346C4E90023C8
:10B80000DDE902015A465346F4F798FC42464B469E
:10B81000F4F794FC02460B46002EC4E90223BFF65F
:10B8200020AF0AF1004301F10041C4E900B3C4E9CB
:10B8300002017F4215E7F4F781FC83468A462D1505
:10B84000CAF30A53EB1A102BD6DD27A3D3E9002342
:10B85000DDE90401F4F72AFE8046894602460B46DC
:10B86000DDE90201F4F76AFC82468B4602460B468C
:10B87000DDE90201F4F762FC42464B46F4F75EFC58
:10B880001BA3D3E9002380468946DDE90401F4F7D0
:10B890000DFE42464B46F4F751FC0B4602468046ED
:10B8A000894650465946CDE906ABF4F747FCC1F34B
:10B8B0000A53ED1A312D83468A4633DC02460B4685
:10B8C000DDE90601C4E90023CDE9020198E703237D
:10B8D0000BE700BFAFF3008000004054FB21F93FAD
:10B8E0003163621A61B4D03D0000601A61B4D03D8A
:10B8F0007370032E8A19A33B83C8C96D305FE43F80
:10B90000FB21E93F7BD90240FB21F93FFB21394173
:10B91000FFFFEF7F000070411CD900080000E03FEE
:10B920009CD8000838A3D3E90023DDE90401F4F72B
:10B93000BDFD8046894602460B46DDE90601F4F767
:10B94000FDFB82468B4602460B46DDE90601CDE94A
:10B9500002ABF4F7F3FB42464B46F4F7EFFB2CA3A4
:10B96000D3E9002380468946DDE90401F4F79EFD12
:10B9700042464B46F4F7E2FB02460B4680468946B8
:10B9800050465946F4F7DAFB83468A4634E7F4F723
:10B99000D7FB274B06469D420F4616D01EA3D3E980
:10B9A0000023F4F7CDFB02460B4630463946C4E986
:10B9B0000023F4F7C3FB18A3D3E90023F4F7C0FB7B
:10B9C0004FF0FF37C4E902014BE615A3D3E900238A
:10B9D000F4F7B6FB14A3D3E900230F460646F4F7A9
:10B9E000AFFB02460B4630463946C4E90023F4F764
:10B9F000A5FB0DA3D3E90023F4F7A2FB4FF0FF371B
:10BA0000C4E902012DE600BF0000002E8A19A33B05
:10BA1000C14920259A837B393163621A61B4D03DD4
:10BA20000000601A61B4D03D7370032E8A19A33BE5
:10BA3000FB21F93F000000002DE9F04F21F0004606
:10BA4000B6F1795F85B00C4692469B4605466BDAA7
:10BA5000F4F7DCFF002800F0E7802A46234628465A
:10BA60002146F4F723FD74A3D3E9002380468946D9
:10BA7000F4F71CFD72A3D3E90023F4F761FB4246FF
:10BA80004B46F4F713FD70A3D3E90023F4F756FBFC
:10BA900042464B46F4F70AFD6DA3D3E90023F4F7C1
:10BAA0004FFB42464B46F4F701FD6BA3D3E900235D
:10BAB000F4F744FB42464B46F4F7F8FC68A3D3E99D
:10BAC0000023F4F73DFB42464B46F4F7EFFCCDE98B
:10BAD00000010022644B40464946F4F7E7FCDDE9EB
:10BAE000002306460F4640464946F4F7DFFC52461F
:10BAF000804689465B4628462146F4F7D7FC024635
:10BB00000B4640464946F4F719FB02460B463046C1
:10BB10003946F4F713FB02460B4600205349F4F76D
:10BB20000DFB05B0BDE8F08F02460B46F4F7BEFCF6
:10BB300041A3D3E9002380468946F4F7B7FC40A32C
:10BB4000D3E90023F4F7FCFA42464B46F4F7AEFC87
:10BB50003DA3D3E90023F4F7F1FA42464B46F4F74C
:10BB6000A5FC3BA3D3E90023F4F7EAFA42464B468F
:10BB7000F4F79CFC38A3D3E90023F4F7DFFA42463C
:10BB80004B46F4F793FC36A3D3E90023F4F7D8FA35
:10BB90004B464246F4F78AFC354BCDE900019E4204
:10BBA00097DD344B00229E4238DCA6F500130020BE
:10BBB0002E4916461F46F4F7C1FACDE902010022CC
:10BBC000294B40464946F4F771FC32463B46F4F7B0
:10BBD000B5FADDE9002306460F4640464946F4F72C
:10BBE00065FC5246804689465B4628462146F4F766
:10BBF0005DFC02460B4640464946F4F79FFA024672
:10BC00000B4630463946F4F799FA02460B46DDE911
:10BC10000201F4F793FA05B0BDE8F08F164B002649
:10BC2000CDE90223154FCAE70020104905B0BDE851
:10BC3000F08F00BFAFF30080D43888BEE9FAA8BD0A
:10BC4000C4B1B4BD9EEE213EAD529C804F7E923E6B
:10BC50009015CB19A001FA3E7751C1166CC1563F21
:10BC60004C5555555555A53F0000E03F0000F03FAD
:10BC70003233D33F0000E93F0000E73F0000D23FEE
:10BC80002DE9F04F1C46ADF5197D0B91611E08930F
:10BC90000391B54BA29912F1140F53F821300746C6
:10BCA0000593C0F2C982B149D31E81FB0301DB17A2
:10BCB000C3EBA10307930133A3EB8303DB00D3188A
:10BCC0000693079A039BD61A059A12EB03091BD415
:10BCD00009F1010900240025B1440DF18008DDF8C7
:10BCE0008CA208E05AF82600F4F776FB01364E45A0
:10BCF000E8E8020108D0002EF4DA20462946013691
:10BD00004E45E8E80201F6D1059B002BC0F2B8834E
:10BD1000089BA7F10802DB0002EB0308049220AAAB
:10BD200002EB030A0293059B72AA02EBC30B0DF50B
:10BD3000E079039B002BC0F29A815546002600272C
:10BD4000049C75E90223F4E90201F4F7AFFB024613
:10BD50000B4630463946F4F7F3F9444506460F469C
:10BD6000EFD1E9E80267D9450AF1080AE1D1029961
:10BD70000498059B014401938B469B000BA9A3F1FA
:10BD80000802CB180A930CAB13440993019A98A9A3
:10BD900001EBC203002A53E9284529DD0DF5E07ABD
:10BDA0000DF130090AEBC2080022714B20462946EA
:10BDB000F4F77CFBF4F72AFEF4F70EFB00226D4B40
:10BDC00006460F46F4F772FB02460B46204629460C
:10BDD000F4F7B4F9F4F71AFE78E9022349F8040BF2
:10BDE00039463046F4F7ACF9D04504460D46DBD170
:10BDF000DDF81890204629464A4600F0A1FC0022B2
:10BE00004FF07F5304460D46F4F750FB00F014FC4E
:10BE10000022594BF4F74AFB02460B4620462946BE
:10BE2000F4F78CF904460D46F4F7F0FD8046F4F77C
:10BE3000D3FA02460B46204629464C46F4F77EF9D3
:10BE4000002C06460F4640F39980019BC9F1180269
:10BE5000581E0CAB53F82030C9F1170543FA02F114
:10BE600001FA02F29B1A43FA05F50CAA002D42F8DA
:10BE70002030884400F38C8000220023304639466D
:10BE8000F4F77CFD002800F09F82019B059A03F1E6
:10BE9000FF394A4510DC002203F18043013B0CA925
:10BEA0000A9801EB830353F80419834242EA010222
:10BEB000F9D1002A40F0E580059B0CAA013B52F81D
:10BEC0002330002B40F0CE800123099A52F8041948
:10BED00001330029FAD001994A1C9146CB180293EC
:10BEE000079B089902EB030A019B0AF1804A0B4465
:10BEF0001D4620AB03EBC505A39B0AF1FF3A03EBFC
:10BF00008A0A70AB03EBC20301935AF8040FF4F7EB
:10BF100063FAA846039BE8E80201002B20DB049C9F
:10BF200000260027083D01E075E80201F4E902233C
:10BF3000F4F7BCFA02460B4630463946F4F700F9EE
:10BF40005C4506460F46EFD1019B09F10109E3E884
:10BF500002670193029B45469945D6DD019315E79B
:10BF600000260027F0E700BF68DA0008ABAAAA2A7B
:10BF70000000703E000070410000204069D1019B2C
:10BF80000CAA013B52F82350ED15002D7FF774AF3A
:10BF9000019B08F10108002B40F314820C9C002C3B
:10BFA0003AD1019B012B09D001220CA951F8044F71
:10BFB000531C9CBB1A46019B9342F7D1069B002B56
:10BFC0000EDD012B00F01B81022B09D1019B0CA976
:10BFD0005A1E0CAB53F82230C3F3150341F822303C
:10BFE000022D7FF449AF32463B4600209849F4F7D2
:10BFF000A5F806460F46002C3FF43EAF069A0020F7
:10C00000934900F09DFB02460B4630463946F4F753
:10C0100095F806460F462FE7012300220CA9C4F12C
:10C02000807441F822400199994210DD0CAC0CAAB1
:10C0300052F823206FF07F4004EB830304EB81016F
:10C0400000E01A68821A43F8042B8B42F9D10124CC
:10C05000B4E700227F4BF4F7AFFC002840F0DA8011
:10C06000054609E7019B5A1C9146029238E70026D3
:10C070000027E9E80267D9450AF1080A7FF459AEBA
:10C0800075E6069A0CAB53F82930183ACDF81C80A7
:10C090000495069273B9019B0CA903F18043023BFE
:10C0A00001EB830353F8041909F1FF39183A002909
:10C0B000F8D00692069A0020654900F041FBB9F1DC
:10C0C000000F04460D46C0F2E2814FF0000A4FEA2D
:10C0D000C90370AA02EB0308069309F101060CAB31
:10C0E000DFF874B108F1080703EB860656F8040D73
:10C0F000F4F772F922462B46F4F7D8F95B4667E964
:10C100000201524620462946F4F7D0F90CAB9E4274
:10C1100004460D46EAD1CDF80890DDF8149048ABFE
:10C12000B9F1000F0393C34601934FF0000A2BDBD4
:10C1300045A3D3E90023DFF824815D4600260027CC
:10C14000002403E0544510DCF8E80223F5E802017E
:10C15000F4F7ACF902460B4630463946F3F7F0FFE8
:10C160000134A14506460F46ECDA019B029AE3E84A
:10C17000026792450193ABF1080B0AF1010306D067
:10C18000B9F1000F9A46D3DA00260027EDE7A29B0B
:10C19000DDF80890032B2BD8DFE813F0F400E30060
:10C1A000E300640000252C46DDE9480123462A46C9
:10C1B000F3F7C4FF049B002B40F0428123462A463C
:10C1C0000B9CB9F1000FC4E900230CDD012648AF38
:10C1D000F7E902230136F3F7B3FFB145F8DA049B20
:10C1E0000BB101F100410B4602460B99C1E9022354
:10C1F000079B03F007000DF5197DBDE8F08F019B4B
:10C200000CA95A1E0CAB53F82230C3F3160341F8A5
:10C210002230E5E6019B08F10108002BC8BF02258A
:10C220003FF7BCAE32463B4600200949F3F786FF94
:10C23000022506460F461FE600216FF017030791FF
:10C240003DE500BFAFF3008000000040FB21F93F57
:10C250000000F03F0000E03F0000703E30DA0008D0
:10C2600048AB0393B9F1000F40F32381039A4FEADF
:10C27000C9030193D3189846D3E900AB58E9026784
:10C2800052465B4630463946F3F75AFF04460D46A0
:10C2900002460B4630463946F3F750FF5B4652469E
:10C2A000F3F74EFFC8E9000168E90245039BA24687
:10C2B0004345AB46E2D1B9F1010F40F3FA80019B4F
:10C2C000039A13441C46D3E900AB1D4655E9028985
:10C2D00052465B4640464946F3F732FF06460F4654
:10C2E00002460B4640464946F3F728FF5B46524656
:10C2F000F3F726FFC5E9000165E902674AABAB42E7
:10C30000B246BB46E2D100239C46039A083402F1B0
:10C310001005184674E902236146F3F711FFA542A0
:10C3200003468C46F5D1039A1146D2E90082D1E941
:10C3300002E90499002940F08D801846464674466B
:10C3400017464D4661460B9BC3E90401C3E90067EC
:10C35000C3E90245079B03F007000DF5197DBDE811
:10C36000F08F00252C46069E039F08363E44284643
:10C3700076E902232146F3F7E3FEB74205460C4671
:10C38000F5D111E700231C46069D039E0835354470
:10C39000184675E902232146F3F7D2FEAE42034662
:10C3A0000C46F5D1049A0AB104F10044184621461E
:10C3B0000B9BC3E90001079B03F007000DF5197DF6
:10C3C000BDE8F08F0024F9E53946069F30467A42F1
:10C3D0000495CDF81C8000F0B3F90022364B0446DA
:10C3E0000D46F4F7E9FA08B30022344B20462946FB
:10C3F000F4F75CF8F4F70AFB0646F3F7EDFF0022CA
:10C400002D4BF4F753F802460B4620462946F3F726
:10C4100095FEF4F7FBFA019B0CAA03F1010918370A
:10C4200042F82300069742F8296043E62046294651
:10C43000F4F7ECFA019B0CAA994642F8230039E67E
:10C440000B9B04F10044B9F1000FC3E900543FF71E
:10C45000BDAEC6E60B9C09F100402361079B02F1CB
:10C4600000420CF10041E06003F00700626061618E
:10C47000C4F80080C4F808E00DF5197DBDE8F08F20
:10C48000A7F108030493089BDB0002936FE4A29BCF
:10C49000032B3FF6ADAE01A252F823F0ADC4000865
:10C4A000A5C10008A5C1000861C2000800231C4600
:10C4B00078E700239C4636E7000070410000703E9C
:10C4C0002DE9F04F21F00046B6F1795F85B00C46BA
:10C4D00090469946054604DAF4F798FA002800F0E9
:10C4E00085802A46234628462146F3F7DFFF064685
:10C4F0000F4602460B4628462146F3F7D7FF3EA3D8
:10C50000D3E9002382468B4630463946F3F7CEFF07
:10C510003BA3D3E90023F3F711FE32463B46F3F782
:10C52000C5FF39A3D3E90023F3F70AFE32463B46A1
:10C53000F3F7BCFF36A3D3E90023F3F7FFFD324640
:10C540003B46F3F7B3FF34A3D3E90023F3F7F8FD39
:10C550000E9BCDE900019BB30022334B4046494678
:10C56000F3F7A4FFDDE90023CDE902015046594667
:10C57000F3F79CFF02460B46DDE90201F3F7DEFD0F
:10C5800032463B46F3F792FF42464B46F3F7D6FD61
:10C5900023A3D3E9002306460F4650465946F3F736
:10C5A00085FF02460B4630463946F3F7C9FD024681
:10C5B0000B4628462146F3F7C1FD05B0BDE8F08FD4
:10C5C00002460B4630463946F3F770FF14A3D3E911
:10C5D0000023F3F7B3FD52465B46F3F767FF2A46A5
:10C5E0002346F3F7ADFD05B0BDE8F08F28462146A0
:10C5F00005B0BDE8F08F00BF7CD5CF5A3AD9E53DF4
:10C60000EB9C2B8AE6E55A3E7DFEB157E31DC73E03
:10C61000D561C119A0012A3FA6F810111111813F5F
:10C62000495555555555C53F0000E03F21F00043A1
:10C630001946704700000000C1F30A522DE9F0418D
:10C64000A2F2FF36132E0B460D460446074631DC98
:10C65000002E1FDB384A42FA06F808EA01020243BC
:10C660002DD033A3D3E90023F3F76AFD0022002382
:10C67000F4F7ACF948B1002D04DA4FF4801343FA13
:10C6800006F63544002725EA08053C46294620469B
:10C69000BDE8F08126A3D3E90023F3F751FD002282
:10C6A0000023F4F793F90028EFD0002D29DB0027B1
:10C6B0003D46EAE7332E06DDB6F5806F1CD01946FD
:10C6C0002046BDE8F0814FF0FF38A2F2134228FA6D
:10C6D00002F818EA000FF2D015A3D3E90023F3F70C
:10C6E0002FFD00220023F4F771F90028CDD0002D92
:10C6F00010DB27EA0807C8E70246F3F721FD0446E6
:10C70000DEE725F000430D4A1F43002F18BF1546F2
:10C710000027BAE7142E08D00123C6F1340603FA25
:10C7200006F6371928BFED18E3E70135E1E700BF4A
:10C730009C7500883CE4377EFFFF0F000000F0BFCF
:10C74000F8B5C1F30A5304460D460E46174673BBAF
:10C75000034621F00046334328D0314B0022F3F743
:10C76000A5FE304B04469F420D461ADB0E46C1F330
:10C770000A53363B40F2FE723B44934220DC002BCE
:10C780003DDC13F1350F2CDA4CF250339F4217DCAD
:10C7900005F0004343F0D27141F4B731224841F033
:10C7A0001F011BA3D3E90023F3F780FEF8BD40F27D
:10C7B000FF729342DED102460B46F3F7C1FCF8BD8F
:10C7C00005F0004444F0FC4141F45F1141F4105184
:10C7D00011A3D3E90023154841F03C01F3F766FEAD
:10C7E000F8BD26F0FF4626F4E006363346EA035548
:10C7F0002046294600220E4BF3F758FEF8BD26F0DE
:10C80000FF4626F4E00646EA035520462946F8BDD1
:10C8100059F3F8C21F6EA5019C7500883CE4377E71
:10C8200000005043B03CFFFF59F3F8C29C750088EC
:10C830000000903C044A05491368002B08BF0B46D2
:10C840001844106018467047740C0020E021002046
:10C85000FEE700BFF8B50022002307460E46F4F7B6
:10C8600097F828B938463146BDE8F84000F00AB8D4
:10C87000384606F1004100F005F8404261EB410105
:10C88000F8BD00BFD0B500220B4B06460F46F3F7AC
:10C890000DFEF4F7E3F80446F3F78EFD0022074B94
:10C8A000F3F704FE02460B4630463946F3F746FCE2
:10C8B000F4F7D4F82146D0BD0000F03D0000F0416F
:10C8C000F8B500BFF8BC08BC9E467047F8B500BF7D
:08C8D000F8BC08BC9E4670474D
:10C8D80002030405060708090A0B0C0D0E0F1010B9
:10C8E8000102000002030405060708090A0B0C0DE3
:10C8F8000E0F1010010200000001020408100000D1
:10C9080020202020202020200000000032D800080D
:10C9180035D8000838D800080000000000000000E2
:10C9280001020304060708090000000001020304CD
:10C9380043444320436F6E666967000043444320C5
:10C94800496E7465726661636500000053544D69F1
:10C9580063726F656C656374726F6E6963730000F0
:10C9680053544D3332205669727475616C20436F8D
:10C978006D506F7274000000286E756C6C29000091
:10C98800000000000000006F00000007000700140E
:10C998007F147F142E2AFF2A3A231308646236492B
:10C9A8005620500000070000001C224100004122D0
:10C9B8001C0014083E081408083E080800503000FF
:10C9C8000008080808080060600000201008040239
:10C9D8003E5149453E00427F40004261514946214F
:10C9E80041454B311814127F1027454545393C4ABB
:10C9F800494930017109050336494949360649490B
:10CA0800291E003636000000563600000814224160
:10CA180000141414141400412214080201510906C8
:10CA28003E415D494E7E0909097E7F494949363EA6
:10CA3800414141227F4141413E7F494949417F0966
:10CA48000909013E4149497A7F0808087F00417F6A
:10CA580041002040413F017F081422417F4040406F
:10CA6800407F020C027F7F0408107F3E4141413E17
:10CA78007F090909063E4151215E7F091929464669
:10CA88004949493101017F01013F4040403F0F3092
:10CA980040300F3F4030403F63140814630708706C
:10CAA8000807615149454300007F4100020408100E
:10CAB8002000417F00000402010204404040404041
:10CAC800000003040020545454787F484444383804
:10CAD80044444444384444487F3854545418087EE5
:10CAE8000901020C5252523E7F0804047800447D2A
:10CAF80040002040443D00007F10284400417F4012
:10CB0800007C041804787C080404783844444438C9
:10CB18007C14141408081414147C7C0804040848B1
:10CB280054545420043F4440203C4040207C1C2066
:10CB380040201C3C4030403C44281028440C5050B5
:10CB4800503C4464544C44000836414100007F0086
:10CB5800004141360800080C081808552A552A557E
:10CB680000060906000000000000000000000000A8
:10CB780000000000000000000000000000000000AD
:10CB8800000000000000000000000000000000009D
:10CB9800000000000000000000000000000000008D
:10CBA800000000000000000000000000000000007D
:10CBB80000000000000000000C0000000000000061
:10CBC800000000C00003000000000000000000009A
:10CBD800000000000000000000000000000000004D
:10CBE80000C0C00C6C103880070C603000010000D9
:10CBF8000000006078E0C0071FE0F883877F78E0D6
:10CC0800010000000000001F00C0E0073C3EF8E7FC
:10CC18001F3C86F1039F710638E7181E7EE0E10786
:10CC28001EFE1966D8C0CE1DEE1F1E06F08003003A
:10CC380018006000008001000F0006C00083011E7C
:10CC480000000000000000000000000000000000DC
:10CC5800000038307000000000C0C00C641044C0F0
:10CC68000F0C30600001000000000030FCF0E08F85
:10CC78003FE0F8C38F7FFCF0030000000000803F16
:10CC880078E0E11F7FFEF8E71F7F86F1039F3906F2
:10CC980038E7183FFEF1E31F3FFE19E6DCC0CC1869
:10CCA800E61F0604C0C00700300060000080018055
:10CCB8000F0006C00083011E0000000000000000F5
:10CCC800001800000000000000000C30C000000048
:10CCD80000C0C00C667C44C0080C3060600D0000C9
:10CCE80000000030CCD1209860F018C00870863958
:10CCF8000700000000008030FCE0611843C618609F
:10CD0800004386C10098190638E7183386316398BE
:10CD1800213018C6CCC0FC38071C060CC0E00E0039
:10CD280000006000008001800100060000800118FA
:10CD380000000000000000000018000000000000D3
:10CD480000000C30C000000000C0C08CFF7E44C052
:10CD5800000C3060C0070C000000001886C10018E5
:10CD680060D81860003086190600000001200030E5
:10CD7800CEE1619801861960800186C100980D0690
:10CD8800F8E7996186196698013018C6CCCC7830D6
:10CD9800030E0608C0701C0000E063073EB8E1E11E
:10CDA8000F6EF6F0C083391878630F1E76E0C61E42
:10CDB8003FFE1866D8C0CE39E71F0C30C00000000F
:10CDC80000C00080FF163886010018C0C0070C009C
:10CDD8000000001886C1001860C8F8610738861975
:10CDE80006030CE0F9E7011887E1619801861960EC
:10CDF800800186C100980F06F867996186196698C0
:10CE0800033018C68C6D78F003060618C0000000C1
:10CE180000F0E70F7FFCF1E30F7FFEF1C0831D18E0
:10CE2800F8E71F3FFEF0C79F7FFE18E6DCC0CC3056
:10CE3800E71F0C30C000000000C00000321E80C197
:10CE4800030018C0600D0C000000000CB6C1000CF7
:10CE58003ECCF8E30F18FC3807030C78F887071C5A
:10CE6800F331E38F0186F9E38F01FEC100980F06C5
:10CE7800D8669B61FE19E60F1F3018C68C6D30E02E
:10CE880001070610C00000000010E69C43CE19867A
:10CE980081738EC100830D18D8E69873CE39C78187
:10CEA800411818C6CCCC7830030C0C30C0C0110027
:10CEB80000C00000337C7040370018C000817F003C
:10CEC8000000000CB6C100063EC608E71C18FCF0BE
:10CED80007030C0E00001C06FB31E38F0186F9E303
:10CEE8008F79FEC100980F06D8669B617E18E60F01
:10CEF8003E3018C68C6D30C080030630C00000007C
:10CF080000C067980186F987816186C10083071888
:10CF1800D86698618619C6801F1818C68C4C787018
:10CF280003060C30C0E01F0000C000C07FF08C6317
:10CF3800360018C000817F00F001000C86C1000394
:10CF480070FE0166180C86E10600000E00001C0643
:10CF58009BF1639801861960807986C1009819064B
:10CF6800D8669A610618660E70301886876D78C084
:10CF780080010620C000000000F067980186F9874C
:10CF8800816186C100830F18D86698618619C6002A
:10CF98003F1818C68C6D30E00303033000230E00E1
:10CFA800000000C07FD040643C0018C000000C00A6
:10CFB800F001000686C1800160FE0166180C86013A
:10CFC80006000078F8870706FBF163980186196068
:10CFD800806186C10098390618669E610618661C2D
:10CFE80060301886877378C0C0010660C0000000F2
:10CFF8000038669801861980816186C100831D18F2
:10D00800D86698618619C60070181886877F78E0F8
:10D0180081010C30C00000000000000019D240E47B
:10D028001C0018C000000C3000000306CCC1C080F2
:10D0380060C008E71C06861103030CE0F9E701004D
:10D04800F331631843C61860006386C1209831061F
:10D0580018661C3306306798603038878773CCC0F1
:10D06800E0000640C00000000018E79C43CE398469
:10D07800817386C100831918D8669873CE39C78022
:10D0880060181887877378C0C1000C30C000000092
:10D0980000C0008019FE40C41F00306000000C3042
:10D0A80000000303FCF8E79F7FC0F8C30F06FEF1FA
:10D0B80003030C00012000060638E71F7FFEF8670F
:10D0C800007F86F1E39F71FE19661C3F06F06398A6
:10D0D8007F30F0838773CCC0E01F06C0C00000001B
:10D0E80000F8E70F7FFCF187017F86F9078331F8A5
:10D0F800D866183FFEF0C7807FF8F8870733CCC0A2
:10D10800E11F0C30C000000000C00080097C808353
:10D118003F003060000000300000030378F8E71F8C
:10D128001FC0F081070378E001030C00000000062F
:10D138008E18E60F3C3EF867003C86F1C38761FE17
:10D1480019661C1E06E061381F30E0818773CEC166
:10D15800E01F0680C000000000F066073EB8E183CB
:10D16800016E86F9078371F0D866181E76E0C6004E
:10D178003FF0F0060333CEC1E01F0C30C0000000C2
:10D1880000000000001000000000306000000030C7
:10D198000000800100000000000000000000000006
:10D1A80000000C0000000000FC010000000000006E
:10D1B8000000000000000000000000000000030064
:10D1C800000000000000000000000680C100000010
:10D1D80000000000000000000061000000030000E3
:10D1E800000000000600060000000000000000C06B
:10D1F80000000C30C000000000000000001000001B
:10D20800000060300000001800000000000000006E
:10D218000000000000000000000006000000000000
:10D22800F8000000000000000000000000000000FE
:10D2380000000000000002000000000000000000E4
:10D2480000001E00F00000000000000000000000C8
:10D25800007F0000E0030000000000000600060058
:10D26800000000000000007000000C30C00000004A
:10D2780000000000000000000000000000000000A6
:10D288000000000000000000000000000000000096
:10D298000000000000000000000000000000000086
:10D2A8000000000000000000000000000000000076
:10D2B8000000000000000000000000000000000066
:10D2C8000000000000000000003E0000E001000037
:10D2D80000000000060006000000000000000070CA
:10D2E800000038307000000000000000000000005E
:10D2F8000000000000000000000000000000000026
:10D308000000000000000000000000000000000015
:10D318000000000000000000000000000000000005
:10D3280000000000000000000000000000000000F5
:10D33800000000000000C0FF000000000000000026
:10D3480000000000000000000000000000000000D5
:10D358000000000000000000000000300000000095
:10D3680000000000000000000000000000000000B5
:10D3780000000000000000000000000000000000A5
:10D388000000000000000000000000000000000095
:10D398000000000000000000000000000000000085
:10D3A8000000000000000000000000000000000075
:10D3B8000000000000000000000000000000000065
:10D3C8000000000000000000000000000000000055
:10D3D8000000000000000000000000000000000045
:10D3E8009D74000800000000000000003974000867
:10D3F8000000000000000000000000000000000025
:10D40800857500088575000885750008857500080C
:10D418000000000000000000497E00085D7E000852
:10D42800A77D0008EF7D0008BF7D00081D7E00086D
:10D438003A0000004750533F0000000053706565F4
:10D44800640000004176657261676500244D4A58A2
:10D4580044522C432C256C642E2530326C642C43AA
:10D468002C41697254656D702C502C2530316C64D8
:10D478002E2530356C642C422C41697250726573CC
:10D48800000000002A253032580A0000540000002D
:10D498002050000020000000002020202020202014
:10D4A800202028282828282020202020202020204C
:10D4B800202020202020202020881010101010105C
:10D4C80010101010101010101004040404040404A8
:10D4D8000404041010101010101041414141414142
:10D4E8000101010101010101010101010101010124
:10D4F8000101010110101010101042424242424234
:10D5080002020202020202020202020202020202F3
:10D51800020202021010101020000000000000009B
:10D5280000000000000000000000000000000000F3
:10D5380000000000000000000000000000000000E3
:10D5480000000000000000000000000000000000D3
:10D5580000000000000000000000000000000000C3
:10D5680000000000000000000000000000000000B3
:10D5780000000000000000000000000000000000A3
:10D588000000000000000000000000000000000093
:10D5980000000000000000000000000084010020DE
:10D5A8001F0000001C0000001F0000001E000000FB
:10D5B8001F0000001E0000001F0000001F000000E8
:10D5C8001E0000001F0000001E0000001F000000D9
:10D5D800000000001F0000003B0000005A0000008F
:10D5E8007800000097000000B5000000D40000009B
:10D5F800F300000011010000300100004E0100009E
:10D608006E6600696E69747900616E00350000000D
:10D61800CEFBFFFFCB03000001000000000000006C
:10D6280034000000CEFBFFFFCB0300000100000028
:10D638000000000000000000BC89D897B2D29C3CD2
:10D6480033A7A8D523F649393DA7F444FD0FA532E1
:10D658009D978CCF08BA5B25436FAC642806681188
:10D66800545A00474D54002531305B5E302D392C1B
:10D678002B2D5D256E004D256875256E2E25687548
:10D68800256E2E256875256E002F256875256E3A3E
:10D69800256875256E3A256875256E00B0D6000890
:10D6A80034D80008480200202E004300504F534948
:10D6B800580000001F0000001C0000001F000000B0
:10D6C8001E0000001F0000001E0000001F000000D8
:10D6D8001F0000001E0000001F0000001E000000C8
:10D6E8001F0000001F0000001D0000001F000000B8
:10D6F8001E0000001F0000001E0000001F000000A8
:10D708001F0000001E0000001F0000001E00000097
:10D718001F000000000000000080E03779C341438B
:10D72800176E05B5B5B89346F5F93FE9034F384D7F
:10D73800321D30F94877825A3CBF737FDD4F15752B
:10D74800000000000000F03F00000000000024403E
:10D7580000000000000059400000000000408F4019
:10D76800000000000088C34000000000006AF84084
:10D778000000000080842E4100000000D0126341A8
:10D788000000000084D797410000000065CDCD411E
:10D79800000000205FA00242000000E876483742FF
:10D7A800000000A2941A6D42000040E59C30A2429D
:10D7B8000000901EC4BCD64200003426F56B0C4312
:10D7C8000080E03779C3414300A0D88557347643B9
:10D7D80000C84E676DC1AB43003D9160E458E1431A
:10D7E800408CB5781DAF154450EFE2D6E41A4B448F
:10D7F80092D54D06CFF08044F64AE1C7022DB544D4
:10D80800B49DD9794378EA44050000001900000066
:10D818007D000000686C4C00412D46612D6638394A
:10D8280030313233343536375D002B2D003030003F
:10D838007858000000000000000000000000000010
:10D8480000000000000000000000000000000000D0
:10D8580000000000000000000000000000000000C0
:10D8680000000000000000000000000000000000B0
:10D8780000000000000000000000000000000000A0
:10D888000000000000000000000000000000000090
:10D8980000000000FB21F93FFB2109407CD9124020
:10D8A800FB2119407A6A1F407CD92240BBFD2540E4
:10D8B800FB2129403A462C407A6A2F405C47314088
:10D8C8007CD932409C6B3440BBFD3540DB8F374000
:10D8D800FB2139401BB43A403A463C405AD83D40B7
:10D8E8007A6A3F404C7E40405C4741406C10424061
:10D8F8007CD942408CA243409C6B4440AC344540A8
:10D90800BBFD4540CBC64640DB8F4740EB584840FF
:10D91800FB21494083F9A200444E6E00FC29150002
:10D92800D1572700DD34F50062DBC0003C99950033
:10D93800419043006351FE00BBDEAB00B761C500F8
:10D948003A6E2400D24D42004906E00009EA2E0052
:10D958001C92D100EB1DFE0029B11C00E83EA70077
:10D96800F535820044BB2E009CE98400B426700083
:10D97800417E5F00D6913900538339009CF4390009
:10D988008B5F840028F9BD00F81F3B00DEFF97007D
:10D998000F980500112FEF000A5A8B006D1F6D00BC
:10D9A800CF7E360009CB2700464FB7009E663F0062
:10D9B8002DEA5F00BA277500E5EBC7003D7BF10053
:10D9C800F739070092528A00FB6BEA001FB15F002B
:10D9D800085D8D00300356007BFC4600F0AB6B0001
:10D9E80020BCCF0036F49A00E3A91D005E619100C7
:10D9F800081BE60085996500A0145F008D4068004B
:10DA080080D8FF0027734D0006063100CA5615005E
:10DA1800C9A873007BE260006B8CC00000000000A6
:10DA280000000040FB21F93F000000002D44743E37
:10DA3800000000809846F83C0000006051CC783B1C
:10DA480000000080831BF0390000004020257A3850
:10DA5800000000802282E336000000001DF36935D3
:10DA6800020000000300000004000000060000009F
:10DA7800C51100085D750008997D00081D83000820
:04DA88009D110008E4
:10DA8C000000000001000000100000000024F40061
:10DA9C00B53B0008C13B0008713C00084D3C000838
:10DAAC00393C00088D3C0008B13C00081201000212
:10DABC0002020040830440570002010203010000EF
:10DACC00040309041A030000000000000000000019
:10DADC00000000000000000000000000000000003A
:10DAEC00F93C0008D53C0008D93C0008DD3C000896
:10DAFC000D5E0008CB5D0008F15C00080000000022
:10DB0C001F5C0008A75C0008795C0008000000009E
:10DB1C000000000000000000555C0008495C000893
:10DB2C00615C00086D5C000809024300020100C042
:10DB3C003209040000010202010005240010010555
:10DB4C0024010001042402020524060001070582B9
:10DB5C000308001009040100020A00000007050177
:10DB6C00024000000705810240000000090243004A
:10DB7C00020100C032090400000102020100052468
:10DB8C0000100105240100010424020205240600F2
:10DB9C00010705820308001009040100020A0000B5
:10DBAC0000070501020002000705810200020000C7
:10DBBC000A060002000000400100000009074300B3
:10DBCC00020104C032090400000102020100052414
:10DBDC0000100105240100010424020205240600A2
:10DBEC00010705820308001009040100020A000065
:10DBFC0000070501024000000705810240000000FB
:10DC0C0084010020000000005CD800087CD80008CB
:10DC1C003CD80008000000000000000000000000DC
:10DC2C0000000000000000000000000000000000E8
:10DC3C0000000000000000000000000000000000D8
:10DC4C0000000000000000000000000000000000C8
:10DC5C0000000000000000000000000000000000B8
:10DC6C00000000006BD600086BD600080000000016
:10DC7C0001000000000000004A000000000000004D
:10DC8C000000000000000000000000000000000088
:10DC9C000000000000000000000000000000000078
:10DCAC004A0000000000000000000000000000001E
:10DCBC000000000000000000000000000000000058
:10DCCC000000000000000000FF0000004300000006
:10DCDC000000000000000000000000000000000038
:10DCEC0000000000000000000000000043000000E5
:10DCFC000000000000000000000000000000000018
:10DD0C0000000000000000000000000043000000C4
:10DD1C0000000000000000000000000000000000F7
:10DD2C0000000000000000000000000043000000A4
:10DD3C0000000000000000000000000000000000D7
:10DD4C000000000000000000000000004300000084
:10DD5C0000000000000000000000000000000000B7
:10DD6C000000000000000000000000004300000064
:10DD7C000000000000000000000000000000000097
:10DD8C000000000000000000000000004300000044
:10DD9C000000000000000000000000000000000077
:10DDAC000000000000000000000000000DAD0008A5
:10DDBC00D5A1000800000000A0D40008B0D60008CF
:10DDCC0034D8000834D8000834D8000834D80008F7
:10DDDC0034D8000834D8000834D8000834D80008E7
:10DDEC0034D80008FFFFFFFFFFFFFFFFFFFFFFFF1F
:10DDFC00FFFF0000010041534349490000000000AF
:10DE0C000000000000000000000000000000000006
:10DE1C00000000000000415343494900000000008D
:10DE2C0000000000000000000000000000000000E6
:0CDE3C000000000000000000700C00203E
:040000050800832D3F
:00000001FF
